:100000000C94B7370C94BC3A0C94E73A0C94123B1E
:100010000C943D3B0C94683B0C94933B0C94BE3B7E
:100020000C94E93B0C94E8370C94E8370C94E837CF
:100030000C94E8370C94E8370C94E8370C94E837C4
:100040000C94E8370D948D310C94E8370C94E83714
:100050000C94E8370C94E8370D946B240C94EA3731
:100060000C94E8370D941C000D94C8000C94E837EC
:100070000C94E8370C94E8370C94E8370C94E83784
:100080000C94E8370C94E8370C94E8370C94E83774
:100090000C94E8370C94E8370C94E8370C94E83764
:1000A0000C94E8370C94E8370C94E8370C94E83754
:1000B0000C94E8370C94E8370C94E8370C94E83744
:1000C0000C94E8370C94E8370C94E8370C94E83734
:1000D0000C94E8370C94E8370C94E8370C94E83724
:1000E0000C94E837323937393C3946395039C939F7
:1000F0005A3962396A3974397E3988399739A13960
:10010000C939AB39B539BF39ED39F039DF39E339A0
:10011000E939273AF439F839FE39023A063A0C3A05
:10012000103A143A273A1A3A1E3A223A326940698A
:1001300051695F696E697C698B699969237B2B7B47
:10014000347B3F7B477B4F7B587B6F7B9D7B9D7BCD
:100150009D7B9D7B9D7B9D7B9D7B9D7B9D7B9D7BDF
:100160008E7B917B947B9A7BAD7CB07CB37CB67CA0
:10017000B97CD97CBC7CBF7CC27CC57CC87CCB7C78
:10018000CE7CD67C20822E823D824E825C826A8228
:1001900079828B82328637863A8649864C865486A7
:1001A0006486648664865D86F18B0B8C208C3A8C29
:1001B0004F8C698C868C7F8C1C901F9022902A908B
:1001C0002D9032903590389040906D927B928C9229
:1001D0009A92A992B792C692D4923C964A965B960E
:1001E0006996789686969596A3964C9751975497CC
:1001F00057975E9761976797709A789A839A8B9AC8
:10020000949A9C9AA59AAC9AB59AC89ACCA7CCA76E
:10021000CCA7CCA7D7A7D7A700A800A8E1A7E4A799
:1002200000A8CCA7E7A7EAA7EFA7F6A74FA858A86A
:1002300069A862A871A878A880A880A894B7A2B776
:10024000B3B7C1B7D0B7DEB7EDB7FBB7B2B8BFB879
:10025000CEB8DBB8EAB8F7B806B95CD461D461D4DB
:1002600061D494D494D470D476D494D480D480D4EB
:1002700094D494D494D48ED404FE02FE26FE23FE9D
:1002800021FE58FE55FE53FEB1FE7FFE7CFE7AFE37
:10029000DF02B103AD03E703AD02BB039502BB036D
:1002A00025037302BB0387028D03CB03A1038902DD
:1002B0002B03B503DB023D03FF02FF027B02FF02BB
:1002C00063032103BF03FD0293023103DD026703D1
:1002D000B703E5021F030F030F0381030F039B0204
:1002E0008D02BB02D102DB03AF03A702E3039F022F
:1002F0009B03ED027D027D0243037D02E90333038C
:10030000D703B903A1029503A9034D038B03BF02D1
:10031000190315031503750215039D024B0377039B
:10032000C503E702C502AB021303B3025B03070375
:10033000170317031703170355039703A703D503E1
:1003400065032D030303BD037503C703C703C70379
:10035000C703C9028502EB027303B1020D03F70262
:100360004103EF02CD03CD03CD03CD037B03710326
:100370006D031103E50383039702C302D303F30262
:10038000F302F302F3025103D70283029D039903A0
:100390007702C9038F03FB028302090383029902D8
:1003A000830237039102790229037903C1034903C8
:1003B000CF03C1023B03930305035D039F03D902EF
:1003C0001B03CD02B5020503F9020503A5020503CF
:1003D00057038703D302C702D502DD03CF02DF0331
:1003E00059030103E1038B02CB02F5022F03B30390
:1003F0006B03E9028B02AF028B02BD028B027F030B
:1004000047036103D103E30281028F02B7021D0398
:100410005F03EB035303A3037F026F0323039103E3
:1004200045035303F1025303D90353036903C30381
:10043000B9024F03E1027D033F030B038503A503CC
:10044000084AD73B3BCE016E84BCBFFDC12F3D6C3B
:1004500074319ABD56833DDA3D00C77F11BED9E4A1
:10046000BB4C3E916BAAAABE000000803F05A84C81
:10047000CDB2D44EB93836A9020C50B9918688084D
:100480003CA6AAAA2ABE000000803F08000000BEC9
:10049000922449123EABAAAA2ABECDCCCC4C3E0037
:1004A000000080BEABAAAAAA3E00000000BF000068
:1004B00000803F0000000000084178D3BB4387D193
:1004C000133D190E3CC3BD4282AD2B3E68EC8276D3
:1004D000BED98FE1A93E4C80EFFFBE01C4FF7F3F34
:1004E0000000000000000D9485000D94540D0D9443
:1004F00030110D94B5110D943A0C0D940E0D0D9410
:100500008A150D9416150D9445120D94940F0D94A3
:100510008B000D94210C0D945D150D94A20C0D947F
:1005200021150D94A0110D94720C0D947D000D9465
:1005300096100D9483110D949D0C0D94590D0D94EE
:10054000E70C0D942E0D0D9408920D94EB120D9462
:10055000DD0C0D94B8970D944E0E0D9479000D940A
:1005600064140D94C20F0D94640E0D94C5120D9475
:1005700030150D940F160D94AB0C0D9477140D944B
:100580004A0D0D942A120D94A1100D94430E0D9452
:100590003B130D944B0F0D94F9130D94B2120D945F
:1005A00095130D94CB0C0D9429130D947D130D947C
:1005B00014110D9489120D94300C0D947F0C0D9430
:1005C0004F000D945C160D9409150D948E0C0D942E
:1005D000380E0D9451140D94A00F0D94F10C0D9440
:1005E00006100D94CF150D94DA100D9406140D9489
:1005F000E40F0D94D8120D9463110D946D0C0D94AD
:10060000520C0D94C5130D941B0F0D94D1130D9422
:100610007A0E0D9473110D9474160D94D30F0D94DE
:10062000B00C0D9475100D94590E0D946C0D0D9425
:10063000AE0E0D944F0D0D9498120D943F150D9420
:10064000930C0D94440C0D949C150D9481000D9405
:1006500059030D94C1110D94260C0D940A0F0D949D
:1006600015140D94770C0D94000D0D94232D0D94FD
:1006700094110D944E6D0D9439120D94350C0D940A
:100680006C160D94F50F0D94F60C0D94C1150D9488
:100690009D140D9412120D945E0D0D94400D0D9449
:1006A0001A160D94B3100D9494160D94850E0D9496
:1006B000FF120D94B3130D946F0E0D946D120D94E3
:1006C00051150D94B5140D943F0C0D94F90E0D9425
:1006D000840C0D94EC150D943E140D9466100D943D
:1006E00094150D945D100D94B10F0D943D0F0D9464
:1006F000670D0D9400120D9414100D9464160D9452
:100700008B140D94980C0D948B100D947C160D94F5
:1007100011130D942F560D94450D0D940F0C0D943F
:1007200053110D94B3150D9464120D94330D0D9463
:10073000CC0E0D9424110D94EC0C0D941A110D9403
:100740007A120D94190C0D9482150D948B160D943C
:10075000D70E0D943B0D0D94AE940D9466000D9440
:10076000D50C0D9455000D9424140D942B0C0D9460
:10077000890C0D94290D0D948E000D942C0F0D9461
:100780004D0C0D940A120D94FB150D94330E0D941F
:10079000750F0D943C110D94140C0D943E100D9496
:1007A0001E120D94C7140D94AB100D94E80E0D9409
:1007B000090D0D94DD150D94D00C0D948A130D9434
:1007C000A4130D94F0130D94E20C0D9480100D946D
:1007D00071000D94FB0C0D947C154E414E494E4911
:1007E0005459494E46CDCCCC3D0AD7233C17B7D1FE
:1007F0003877CC2B329595E6241FB14F0A000020A4
:10080000410000C84200401C4620BCBE4CCA1B0E22
:100810005AAEC59D7400407A10F35A00A0724E186B
:10082000090010A5D4E80000E87648170000E40BA2
:1008300054020000CA9A3B000000E1F50500008068
:10084000969800000040420F000000A086010000C2
:1008500000102700000000E8030000000064000012
:100860000000000A00000000000100000000002C51
:1008700076D888DC674F0823DFC1DFAE59E1B1B716
:1008800096E5E3E453C63AE651997696E8E6C284E3
:1008900026EB898C9B62ED407C6FFCEFBC9C9F40FB
:1008A000F2BAA56FA5F490055A2AF75C936B6CF920
:1008B000676DC11BFCE0E40D47FEF520E6B500D0F6
:1008C000ED902E0300943577050080841E0800000B
:1008D000204E0A000000C80C333333330F986E12D9
:1008E000831141EF8D2114893BE65516CFFEE6DBDF
:1008F00018D1844B381BF77C1D901DA4BBE4242029
:100900003284725E228100C9F124ECA1E53D27000A
:10091000000A0B02090C0D0E080703040100000079
:1009200000000000000000000000000000000000C7
:100930000000000000000000000000121110000084
:1009400000000000000000000000000000000000A7
:1009500000000000000102102020080810204010B4
:100960002040800201020108040201010204081073
:100970002040808040201008040201800402018091
:1009800040201008040201080402010102040810BA
:10099000204080010204081020408005050505075D
:1009A0000508080808020202020A0A0808040404EA
:1009B0000401010101010101010303030303030316
:1009C00003040707070C0C0C0C0C0C0C0C020202A5
:1009D0000206060606060606060B0B0B0B0B0B0B98
:1009E0000B000020002300260029002C002F0032DD
:1009F000000001000003010601090100002200259A
:100A00000028002B002E00310034000201000005F8
:100A10000108010B0100002100240027002A002DFD
:100A2000003000330001010000040107010A0154F5
:100A3000696D656F7574206F6E20444C5F43616310
:100A400068653A3A576169745F556E74696C5F49BD
:100A5000646C6528290A0000FF00000A0B0F1A19B0
:100A60001F1A0A0F0E121809120B1118181818184D
:100A700018181818180A0A15171614251B1B1A1C03
:100A800017161C1D0C171A16231D1C1A1D1B1A1ACB
:100A90001C1B241B1A190C120C12150D17181618F2
:100AA000160F18180A0B160A24181818180F160E05
:100AB0001815201515160F0A0F1D0A080810100D1D
:100AC0001114161D261014191C24313F536C0000FC
:100AD00000070AA9C2000B26AEC2000C26B0C20055
:100AE0000518B2C2000910B3C2000A10B9C200084A
:100AF0001080C341000D81C341010D82C341020D2D
:100B000083C341030D84C341040D85C341050D8793
:100B1000C343060D88C345000D89C345010D8AC333
:100B200045020D8BC345040D8CC34900068DC34996
:100B300001068EC34902068FC349040691C34E03C2
:100B40000F92C34F000E93C34F010E94C34F020E7A
:100B500095C34F030E96C34F040E99C355000E9ACA
:100B6000C355010E9BC355020E9CC355040E9DC375
:100B700059010DA0C361000CA1C361010CA2C361A6
:100B8000020CA3C361030CA4C361040CA5C36105DB
:100B90000CA7C363060CA8C365000CA9C365010CB0
:100BA000AAC365020CABC365040CACC3690005ADF8
:100BB000C3690105AEC3690205AFC3690405B1C3CA
:100BC0006E030CB2C36F000CB3C36F010CB4C36FE0
:100BD000020CB5C36F030CB6C36F040CB9C3750028
:100BE0000CBAC375010CBBC375020CBCC375040CF5
:100BF000BDC379010BBFC379040B7600010801EE78
:100C000001E5110001AF01FF01201000010C01FFFF
:100C100001D01000010101DF01F91100012E01FFD7
:100C200001501000010301FF01F21100015F01FDFD
:100C30001100010601990140FF00FF00A4007B00A4
:100C4000019E01EE01500F00010501FF01F81000A7
:100C5000012F01FF01A0100001CF01FC10000109CC
:100C600001FF01D11000014F01FE01200F00010121
:100C700001EF01F31000010701AA0140FF00FF008E
:100C8000A500790001CF01FC1000010702FF0160FF
:100C90000F00012F02FF01F20F0001CF01F6016FDB
:100CA00001FB0E00010601FF01A0010A01FF016026
:100CB0000D00011F01FD0100010101DF01F10D0027
:100CC00001BF01F30200013F01FB0C000102019989
:100CD00001500200010501990120FF00FF00A20060
:100CE0007C0001110D00010901FF01C3020001FF99
:100CF00001800C0001AF02FF0150010101FF016002
:100D00000B00010201FF01D901FF01F7010701FFFB
:100D100001400B00010701FF0120013E02FF01FD20
:100D20000C00010901FE0100010201DF01FF01F4D5
:100D30000C00010701A80200010601980120FF0034
:100D4000FF00B6008A000244020002440D0002FFC8
:100D50000110010102FF0D0002FF0110010102FF5D
:100D60000D0002FF0110010102FF0D0002CC011075
:100D7000010102CCFF00FF00C9002D00011301306A
:100D80001000012B02FF01A10E00010201EF02FF82
:100D900001FD01100D00010D01FF0194015A01FF39
:100DA00001B00D00014F01F70200019F01F20D009B
:100DB000018F01F00200012F01F60D00018F01E00B
:100DC0000200010F01F70D00017F01F20200014F47
:100DD00001F50D00012F01FC0110010201DF01F0FE
:100DE0000D00010801FF01FB01CF01FF01600E00B2
:100DF000019F02FF01F80F000103019C01C90130AE
:100E0000FF00FF00A400FF00FF00EE00010601FF4D
:100E10000120110001CF01C01100013F01F61100B6
:100E2000010F01FB1100013F01FD0E00010701D977
:100E3000018901FF01FB0E00010703FF01F30E0012
:100E4000010401BD01EE01D901202F00FF00320095
:100E50000101019901961000010101FF01F9100043
:100E6000010101FF01F91000010101FF01F910006A
:100E7000010101FF01F91000010101FF01F910005A
:100E8000010101FF01F91000010101FF01F910004A
:100E9000010101FF01F91000010101FF01F910003A
:100EA000010101FF01F91000010101FF01F910002A
:100EB000010101FF01F91000010101FF01F910001A
:100EC000010101FF01F91000010101FF01F910000A
:100ED000010101FF01F91000010101FF01F91000FA
:100EE000010101FF01F91000010101FF01F91000EA
:100EF000010101FF01F91000010101FF01F91000DA
:100F0000010101FF01F9CD00990001010136019BAA
:100F100001BB01200E00013F03FF01200E00013F35
:100F200001FE01BE01FF01200E0001140110010BA2
:100F300001FF01201000010B01FF01201000010B37
:100F400001FF01201000010B01FF01201000010B27
:100F500001FF01201000010B01FF01201000010B17
:100F600001FF01201000010B01FF01201000010B07
:100F700001FF01201000010B01FF01201000010BF7
:100F800001FF01200F000111011C01FF01310111BE
:100F90000D00010D05FF01400C00010D05FF014092
:100FA0000C0001010522FF00C200880001011000B1
:100FB000011601AE01FF01FD01920E0005FF016067
:100FC0000D0001FE01840122015C01FF01F30D000F
:100FD0000150030001CF01FA1100015F01FC110073
:100FE000015F01FB110001CF01F41000010801FFB6
:100FF00001A01000016F01FE01100F00010501FFAB
:1010000001E21000015F01FF01300F00010501FF47
:1010100001E31000016F01FE01200F00010801FF34
:1010200001D1100001AF01FD014303330C000101A8
:1010300006FF0C00010106FF0D000622FF00C200A2
:101040008800010101100F00013901CE02FF01B536
:101050000E00017F04FF01B00D00016B017301223E
:10106000013801FF01F91100015F01FF1100010FBB
:1010700001FF1100014F01FC1000012701FF01F3E6
:101080000E00010C02FF01FA01200E00010C02FF0C
:1010900001FB01400E0001010123014901FF01F69E
:1010A0001100013F01FF01101000010B01FF015071
:1010B0001000010A01FF01601000011E01FF014044
:1010C0000C0001A40200010501DF01FD0D0002FF7B
:1010D00001DE02FF01E30D0001AE03FF01E9011093
:1010E0000E00012401550152FF00C400A0000101BF
:1010F0000145017601430E00012801DF03FF01E9EC
:1011000001400B00011902FF01DB01AB01CE01FF21
:1011100001FB01300900010301EF01FB0150030055
:10112000013801FF01F70900016F01FC01300500E2
:10113000011901FF01A00700010501FF01A007003F
:10114000015F01FB0700013F01F803000146018830
:10115000016501100100010301FF0180060001EF9C
:1011600001A001000101019F03FF01FC01600100DA
:10117000014F01F40500010801FD0200014E02FFCC
:1011800001ED01EF01FF01B00100010801FD0500C3
:10119000011F01F40100010401FF01FE01610100D2
:1011A0000101014A01A0020001EF01600400016F8A
:1011B00001C00100010E01FF01C10700017F01B064
:1011C000040001BF01600100017F01FF0110070061
:1011D000011F01F0040001FF0120010001DF01F9FE
:1011E0000800010D01F40300010101FE01000101ED
:1011F00001FF01F40800010A01F60300010301FDEB
:101200000100010201FF01F10800010801F80300DB
:10121000010401FC0100010301FF01F008000107C6
:1012200001F90300010301FD0100010201FF01F1C9
:101230000800010801F80300010101FE010001019D
:1012400001FF01F30800010901F7040001FF01108B
:10125000010001DF01F80800010C01F5040001BFE5
:1012600001600100018F01FE01100700011F01F163
:101270000400016F01B00100011F01FF01B0070070
:10128000016F01C00400011F01F40100010501FF0D
:1012900001FD01500200012901A0020001EF0160DF
:1012A0000400010801FD0200016F02FF01DB01CE15
:1012B00001FF01B00100010701FD0500010101EF7F
:1012C00001900100010201BF03FF01FE0170010056
:1012D000014F01F40600014F01F70200010101581E
:1012E000019A018601300100010201EF0180060030
:1012F000010601FF01900700014F01FB0800016F8B
:1013000001FC01300500011801FF01B008000104D3
:1013100001EF01FA01400300012701EF01F80A0083
:10132000011902FF01CA019A01BE01FF01FC01304F
:101330000B00012901DF03FF01FA01400D0001024A
:10134000014601760153C500A00001020146017665
:1013500001530E00012801DF03FF01EA01400B00E9
:10136000011902FF01CB019A01CE01FF01FC0130FE
:101370000900010401EF01FA01400300013801FFF7
:1013800001F80900016F01FC01300500011801FF9F
:1013900001A00700010601FF01900700014F01FBBA
:1013A0000700013F01F7010001130233013203007E
:1013B000010201FF0180060001EF01A00100017F91
:1013C00003FF01FD01810200014F01F50500010845
:1013D00001FD0200017F01FF01DD01EF01FF01FEC0
:1013E00001300100010801FE0500011F01F40200A7
:1013F000017F01FA0200013C01FF01D0020001EF70
:1014000001600400016F01C00200017F01FA0200C7
:10141000010201FF01F30200017F01B0040001BFDE
:1014200001600200017F01FA030001FF01F40200E4
:10143000011F01F0040001FF01100200017F01FA09
:10144000030001FF01F20200010C01F5030001019C
:1014500001FE0300017F01FA0200010801FF01E023
:101460000200010A01F60300010301FD0300017FF0
:1014700001FD0188019A01EF01FE0130020001081F
:1014800001F80300010401FC0300017F03FF01FEDA
:1014900001910300010701F90300010301FD0300AD
:1014A000017F01FC017801DF01FD0120030001083B
:1014B00001F80300010101FE0300017F01FA0100B0
:1014C000010B01FF01C00300010901F6040001FF47
:1014D00001100200017F01FA020001DF01F80300A0
:1014E000010C01F5040001BF01600200017F01FA57
:1014F0000200014F01FF01300200011F01F1040051
:10150000016F01C00200017F01FA0200010901FF21
:1015100001D00200016F01B00400011F01F40200BC
:10152000017F01FA0200010101EF01F7020001EF62
:1015300001600400010801FD0200017F01FA0300BF
:10154000016F01FF0120010801FE060001EF01A06B
:101550000100015A01A60300010901AA0160014F1F
:1015600001F40600013F01F80800010301FF0180BA
:101570000600010501FF01900700014F01FB080073
:10158000016F01FC01300500011901FF01A00800F5
:10159000010401EF01FA01400300013801EF01F8F5
:1015A0000A00011902FF01CB019A01CE01FF01FCE3
:1015B00001300B00012801DF03FF01EA01400D00AB
:1015C0000102014501760143C500004C696E656169
:1015D0007220416476616E63650052756E6F75743A
:1015E0002053656E736F720046696C616D656E7431
:1015F000004261636B0020002B002D000031303071
:10160000003130003100302E31002E3031002E30CC
:1016100030310000496E6372656D656E7400486F0D
:101620006D6500416C6C005A0059005800426163BE
:101630006B0052756E6F757420320052756E6F7547
:10164000742031005A2050726F6265005A204D6933
:101650006E005A204D61780059204D696E00592066
:101660004D61780058204D696E0058204D6178001A
:10167000456E6473746F7073004261636B006D41FB
:101680000045005A005900580043757272656E7427
:101690007300506C6561736520776169742E2E2E1E
:1016A00000BC80D76FAF80D871C87FD971B77FD8A1
:1016B0006FBC80D76FFFFFCB83F66FCD840B703E7E
:1016C0008406725B83F471FFFFA97CF86F1A7DF5C5
:1016D00071377C0772A77B0D70A97CF86FA97CF825
:1016E0006FFFFFCD876870C7889270BA877C72DF02
:1016F000865872FFFFA8786B7097795A72BA787E15
:1017000072AD779570A8786B70A8786B70FFFFA7A3
:101710008B2C71958C6A71108B39733F8A0373FF20
:10172000FFCE742F713576077364753C73DE736D6D
:1017300071CE742F71CE742F71FFFF478F3F7223CC
:10174000908E722D8E3A746B8DF473FFFF2D714263
:10175000720973F77348723D74507092722D714222
:10176000722D714272FFFF9B929A735C93FA730021
:101770009178755A902775FFFFDC6D9D7322702755
:1017800075746F7C75166DFF73DC6D9D73DC6D9DDC
:1017900073FFFF899533753496A4757E93ED76E8D3
:1017A000928B76FFFFEB6A39758D6D9076FB6CF04E
:1017B00076406AA975EB6A3975FFFF0B9807779A2F
:1017C000988477979592781A952578FFFF6A680C28
:1017D000775B6B2A78DF6A9778DD6788776A680CB1
:1017E000776A680C77FFFF129A0A797E9A9179409E
:1017F000975E7AE196E879FFFF64660F799669ED66
:10180000793769637AF965967964660F7964660F4A
:1018100079FFFF919B327BDB9BC17B7098487C31C9
:1018200098CC7BFFFFE664377B4768D07B07684C2A
:101830007C9D64C57BE664377BE664377BFFFF8273
:101840009C727DA79C067E2599467E0399C57DFFE7
:10185000FFF763787D7667C97D5667497ED3630A53
:101860007EF763787DF763787DFFFFE09CC07FE0C3
:101870009C558057994D805799CB7FFFFF9D63C53D
:101880007F2667CE7F266751809D635A809D63C502
:101890007FFFFF2799D181AA9C1082879CA2820793
:1018A0009952822799D1812799D181FFFF5767D516
:1018B0008177675682F963A782D4631482FFFF772A
:1018C00098CF83E29B5584999BE38438984C847726
:1018D00098CF83FFFF0868D38348685084E764E8A3
:1018E000849E645A84FFFF4997B985889A84861D2F
:1018F0009A0C87EB962E864997B9854997B985FF4B
:10190000FF3869BD859769348665661087F96589F2
:1019100086FFFFA2958587A598928818980F89273A
:1019200095F287A2958587A2958587FFFFDF6A8A52
:10193000875B6BF8876A681589DC679788FFFFF714
:101940006C30898D6D9189EB6AE98A406A798AFFEA
:10195000FF809332894596728A9995E38AF5928D34
:101960008980933289FFFF1091A18A6F931F8CAAFF
:1019700092808C6490F78A1091A18A1091A18AFFBD
:10198000FF736FA58A2170FB8AED6D8C8C176D2318
:101990008CFFFF3E8EE18B37908B8D598FDC8D7CD9
:1019A0008D278C3E8EE18B3E8EE18BFFFF5972EBD3
:1019B0008B1B73318C4071E78D6470978DFFFF2115
:1019C0008BE38CA98CB28EBA8BEF8E518A188D2145
:1019D0008BE38C218BE38CFFFF7675EB8C487620B4
:1019E0008DE074F88EF273BB8EFFFFCD87A18DDC86
:1019F000888B8FE087B58FF086C68DCD87A18DCD82
:101A000087A18DFFFFCC78A88DA879CB8DBC78BB42
:101A10008FC077928FFFFF5084198EE2841490E07C
:101A20008329906C832C8E5084198E5084198EFFDC
:101A3000FF487C1C8E2B7D2E8EBD7C2C90BB7B1793
:101A400090FFFFBE80498ED1804A90CC7F4A90D9CA
:101A50007F498EBE80498EFFFF7682D675AF83FEAA
:101A60007536842876AE846176428506771285BA0B
:101A7000775784457835838B7818838278D882604D
:101A8000781E83307853832378E683F977648490D3
:101A9000777A841A771584B776B6839176518376F0
:101AA000767F826276BB8187766181AF762381DA29
:101AB00076E5801A77C5804D77B880C177D180EE02
:101AC0007707811478CC816B787F8318796484835D
:101AD00079C084B2792D85FD799D85BC7A8E857912
:101AE0007B4585257CD984C57C69844D7D3B84CD2F
:101AF0007D5585A87DD385677D0D87A07CE087C057
:101B00007B0D885B7B6D88467AB3889B79CC887027
:101B1000793A89EA789589A878018A6F78F88A1FD6
:101B200078A68BFD770C8CEF77968CFB771D8D1547
:101B300078598D2678408E8978DB8E2579FC8E7BCE
:101B400079FF8ED479718E7B7A588DD27A238CDE90
:101B50007AFF8A977AF58A817AEF8A4E7A688B5271
:101B60007A968B5F7A398C877A338D7F7A078E3FAE
:101B70007A668ECB79638E8579438E3F79C68DC622
:101B800078FA8C76787E8C5F78188C5778848B7492
:101B900078228B8F787D8ACA782E8AF978F08930FE
:101BA00079A389A5797989C07A7C899C7B7289F22D
:101BB0007BCC88327DB7874C7E6586527F60865AA3
:101BC0007F8F87017FAE88C27EFD899E7E8D8BC60A
:101BD0007E408C0E7FB68C687F1D8DD77FFA8DBDC1
:101BE00080A88E6E81348FD4818A8FF981DA8F0A32
:101BF00082AB900F822091FF81A591DC81F491B896
:101C0000812C92988188922B817D92AB8052926830
:101C1000801C9233807491EB7F9990EB7FCF8F295A
:101C2000805D8F8D80478FA480D48EA480C58E70F8
:101C300080658FE67F6D90927FA491907FA892F748
:101C40007FFC9243803193908049933D81D192E310
:101C50008164922782E5915B825D918082D3909628
:101C600082A08F9A822C8F8682E78E7382788E4A2A
:101C700082A98DD481B98C2781688B2C80228B011D
:101C800080C38AE77F508AF47FFD886880A4871D1F
:101C9000819E872D810489F181D48985827C8A4344
:101CA00083948A31844E8AA184E8890E852F89E540
:101CB00085B088E586C0885787F2888D872789ADEB
:101CC00087BF8A21880E8B1E88708B11881B8CD64B
:101CD000879B8C7687C48C3D87D38C0587A28CA389
:101CE00086068C6286398B4F86778A6286F9894DA3
:101CF00086108A0686668AF785358BDC85508CFDD2
:101D0000853C8D6386948D0A877D8D5F873A8DB87B
:101D100087B18C2D88C18B8C88308BA7888D8AAE3B
:101D200088EE8998886E897E8869882D88EE87EA92
:101D300087A487A8878E8785874D87E3865D873749
:101D400086FD87668405875A83B8865983A484589C
:101D500083207F1B85137F4D861680F9868E81D860
:101D6000873B8269887282C9887682158966823D3E
:101D700089FB81D8899781218A1981628AA7808A03
:101D80008A1680AA8ADC7EAE8AC57D638A557D2943
:101D90008AFA7CE589AD7C39891B7D9588007E2592
:101DA00088277F0088667F0F88697F5088497E7307
:101DB000889A7DC9884F7D3E898B7DB289D87DE622
:101DC00089367E108A027F408ADB7F348A468016FD
:101DD0008A9180F589A580EB89FE80AB8926818177
:101DE00089598118894F81E6882881B8889480565E
:101DF00088FC7E9687747DE7863D7DC586D87C7499
:101E000086987C0586A07C36857C7DE683077E5798
:101E100083ED7D5B83CC793E8462794884CB7750B7
:101E200084F37638843E761E840275FE836C74FDDE
:101E300083E4730A84CE7244849B725784E671B73C
:101E400084B571EB849B713B859B715885D471E09F
:101E500085B0724286D4736186B3741686AD74D72A
:101E600084B274B384B5749B841E7596843B75B834
:101E700084C5756E856D755A86D074B886FA73EA16
:101E8000865072CF86E7703F867E70C8855F704946
:101E9000857570CC84AC707584CD705284FF719C54
:101EA00083877276836A733A83437419831E75112C
:101EB00083AC762783C4774183107840839F79135E
:101EC000832A7AEA82247B8182E47B0C82EC7BB1D8
:101ED000815E7AC8810978ED815177F8816476EF67
:101EE000817175B481BB7441818374F98008742F4A
:101EF00080D973EB7F5973507FA072C47E9E718925
:101F00007E7470A87E1570CC7ED06FF87EA36F199A
:101F10007F6B6FBB7F936F1780A76F3280D76F5A2D
:101F200080DF70928005725A809E72CB7FB372BC44
:101F30007F0973A67F3B73DE7FF9724B806D72A7BA
:101F400080E670FB800D70EC80486FA880FC6E739B
:101F500080C16E2680936ECC7FD46ED87E546F7213
:101F60007ECB6F3A7E0B70257EAB71ED7D56733E56
:101F70007E7274F47E3675BD7FDA7575802876B60C
:101F8000807B76D880D976EF805577FC808178D5B4
:101F90008031799380007A1E809B799B7D9A78D8D6
:101FA0007CC077E57B8377557B8777B97AAE776797
:101FB0007AE6771D7A1E78CD795E7809795378C0F4
:101FC0007823788B78087875784976E877B67469DD
:101FD000788874B37872740179D2746F79D8759AED
:101FE00079EE7671794A777A795177B479A076F07B
:101FF00079E4750A7A5474E179AF73867969730963
:1020000079747391789D733C78B6731E78B7746851
:10201000775D762C77ED7769773279FC7779793649
:1020200078B8797B78DF7912799879147A6779B4FE
:102030007A6A79D87AC579607B9D7AE97B727B4729
:102040007CBA7ED67B0682A87CFA822E7C9183B4F1
:102050007BF683407B1384D07ADD83717A8A83395F
:102060007A9682B779F380FA7816808A78B47F33CB
:10207000788D7FDF77927FA977B37F1877F67FC25D
:102080007636808A7697804A76DF802A763C81058C
:10209000767582D57548807A52DE8ADE5CB275DE4E
:1020A0005CFFFF4880F64FD971205EB88E205E48F5
:1020B00080F64FFFFF36448E8DCC4EF297A039F25A
:1020C00097FFFF36440A8BC8353499A5523499FFDF
:1020D000FF3DBC8E8DD4C6F297A7B1F297FFFF3DAE
:1020E000BC0A8BCEAD3499ACCA3499FFFF458078D9
:1020F000676D7FA7679D7E9F68497DEA69417B8107
:102100006A08793A6A26772C69EA755A6805754C27
:10211000684A749968F573A86945731A6B9371F8E6
:102120006B4D6F086CFA6C456B616BA36A7D6AB787
:102130006AEB691D6B1D6A346C226AB86DE568CD67
:102140006EB966336F1764C56E39625C6E656191F6
:102150006E0861096FC161187082629671CF61D19A
:1021600072E55F8473385D80734B5B6573975AB714
:1021700073745A3874905B2075E85C7176CB5CBBE5
:1021800077435BB078B6581479D75644794F56AD3B
:102190007967562F7ADA57E37AB759F37B315A3792
:1021A0007D27595D7EE0561E7F2955937FD7540DBC
:1021B0008029558780E056FD802659BE81305AE53A
:1021C00082B5592884D85738856456EB854C566DAE
:1021D00086D456D786B25808873F5B6B87C65C604B
:1021E00088E35CAA898B5BFC8A6D5AE38B915A6504
:1021F0008C445BB78C325D9C8CDE5F988CC7614BE6
:102200008D7A62878EB9610590FF6014915C618B55
:10221000912F62C0910E645891B066EA90DC6850CC
:1022200091186A6692126AE993E0690195726A6789
:1022300095566B7B95EE6CD994436F1794887128F3
:102240009439730695E97378963E748797F874D439
:1022500097DD75C6971A77F496FB78E695357BA1DE
:10226000953D7D3796917E8297607F7A983880AAD7
:10227000980F817B98DF818297338338963B85A1C5
:10228000957587E7955689F596928AC897788BD683
:1022900097328C8997888C7A96378D0895E98E2AA3
:1022A000942F911A948393DD941B957F95FF956BE2
:1022B00095909605956096ED9359966A92979754E6
:1022C00091C399EF90659C5D91439EC691179F9134
:1022D00091749F1991BB9E0A90FA9D8C8EAE9E516F
:1022E0008D98A09E8C45A3A28C31A5BE8CE5A56BD4
:1022F0008C09A6EA8BECA4028B94A3B189B2A367E4
:10230000883AA57287C6A70E87A5A9DE862DAA756D
:102310008614AAF285A2A83F85C5A62E844BA6EBFB
:102320008255A7C5819CA9048152AB8F80A6AB15AD
:102330008052AB9B7F9CA9257F55A7647E4CA63E0F
:102340007DC7A6FA7BA5A8EA7A18AA377A31AAB57A
:1023500079A9A94B79CAA71B793CA5B778B6A3C1BF
:10236000779AA37776F1A426750EA63F74EBA5BDE8
:102370007338A56B734BA387739EA08A73B49ED6E4
:1023800072029E9B71C49E1D707E9F0E6F209F9651
:102390006E4E9E616E6E9CCA6ECB99376FA097D2BF
:1023A0006E6496BC6D6B96386C9B96216B0B96BBDE
:1023B0006A2695A66A8E93486B3B910B6CF48EFA55
:1023C0006B438D1D6B948CAA693F8C9B68858B4DEC
:1023D000689E8A5C6862892E6981873C6A4685822C
:1023E0006A3F83EA69EC81A0681C81A86745807810
:1023F0006745807867FFFF4780A06AC881FA6A68EE
:1024000082D56BC881AF6C4780096DC67EAF6C27E3
:102410007ED56BC67EFA6A4780A06A4780A06AFFB5
:10242000FF3E80196E7C86716E658C756FD7911B2F
:1024300071AD965B73BC9A2C76A29D4C795F9FA27E
:102440007CF39F11805E9F8083A19DD586BA9AF60A
:1024500089AB96C78CD691088F658CAD907C86B180
:10246000913D800992007AB1911674AD90A66E08E4
:102470008FD069C78CD6650A8AEE62F48625619B87
:1024800083896011802461887CED622E79D665197C
:1024900076CF695B73A56E1B711674756F007A71C8
:1024A0006E3E80196E3E80196EFFFF3E80B26E5AFE
:1024B0007A046FB274F86F4B6F94718F6AC773A20E
:1024C000668176D56386792662BF7C976111802606
:1024D000626383D5639C86A266A2898F6A5B8C4BFC
:1024E0006F8E8EB2742B905A7A1E913D8070913E01
:1024F00080709121861E91CA8B2B9030918E8EED2B
:10250000955B8CCF99AB89A79C9C86559E6783E58C
:102510009E1180559EBB7CA79C8679CF997776EDDE
:1025200095C77330919471CA8BF86F2186046F3E02
:1025300080B26E3E80B26EFFFFBC80D76FAF80D896
:1025400071C87FD971B77FD86FBC80D76FBC80D777
:102550006FFFFFCB83F66FCD840B703E8406725BFA
:1025600083F471FFFFA97CF86F1A7DF571377C0742
:1025700072A77B0D70A97CF86FA97CF86FFFFFCD67
:10258000876870C7889270BA877C72DF865872FF3E
:10259000FFA8786B7097795A72BA787E72AD77958A
:1025A00070A8786B70A8786B70FFFF00678A7080E6
:1025B00068E5702069BF7180689972FF66F4727F68
:1025C000659972E064BF717F65E47000678A70008E
:1025D000678A70FFFF8D998C700E9BE670AE9BC072
:1025E000710E9B9B728D99F6720D989B726E97C1BE
:1025F000710D98E7708D998C708D998C70FFFFA785
:102600008B2C71958C6A71108B39733F8A0373A779
:102610008B2C71FFFFCE742F713576077364753C78
:1026200073DE736D71CE742F71CE742F71FFFF47FF
:102630008F3F7223908E722D8E3A746B8DF4734798
:102640008F3F72FFFF2D7142720873F77348723D1E
:1026500074507092722D7142722D714272FFFF3E62
:1026600080F6721B89F4739A90CC769F950B7B5EF3
:102670009711809F9517859A9057891B892E8C3EBC
:10268000802B8D61772E8CE26F5789DD6A17851E4E
:10269000691180DD6A0B7BE26FCC766177F4733E63
:1026A00080F6723E80F672FFFF3E808F73C877819E
:1026B00074A0703877D76B467B2C6A1180D76BDC9F
:1026C00084A170EA88C977A18B3E80938CB488A1DD
:1026D0008BDB8FEA88A594DD8450961180A5944603
:1026E0007BDB8F3877B48881743E808F733E808F18
:1026F00073FFFF9B929A735C93FA73009178755AFB
:1027000090277575915E74FFFFDC6D9D73227027B5
:1027100075746F7C75166DFF73DC6D9D73DC6D9D3C
:1027200073FFFF899533753496A4757E93ED76E833
:10273000928B76FFFFEB6A39758D6D9076FB6CF0AE
:1027400076EC6CFA76ED6B7476406AA975456AA7EB
:1027500075EB6A3975EB6A3975FFFF0B9807779A45
:10276000988477979592781A952578FFFF6A680C78
:10277000775B6B2A78DF6A9778DD6788776A680C01
:10278000776A680C77FFFF129A0A797E9A917940EE
:10279000975E7AE196E879129A0A79FFFF64660FEC
:1027A000799669ED793769637AF965967964660F88
:1027B0007964660F79FFFF919B327BDB9BC17B7055
:1027C00098487C3198CB7BFFFFE664377B4768D025
:1027D0007B07684C7C9D64C57BE664377BE6643789
:1027E0007BFFFF829C727DA79C067E2599467E0317
:1027F00099C57DFFFFF763787D7667C97D56674988
:102800007ED3630A7EF763787DF763787DFFFF8769
:102810005CDB7E085E357FA85E0F80085EE98087FE
:102820005C4481855C4481065BE980675A0F8006C1
:102830005B357F875CDB7E875CDB7EFFFF02A4DE8F
:102840007E83A5387F23A6118023A6138083A5EC61
:102850008002A4478181A2ED80E2A1138081A23889
:102860007F02A4DE7E02A4DE7EFFFFE09CC07FE04C
:102870009C558057994D805799CB7FFFFF9D63C52D
:102880007F2667CE7F266751809D635A809D63C5F2
:102890007F9D63C57FFFFF2799D181AA9C10828706
:1028A0009CA282079952822799D1812799D181FFD1
:1028B000FF5767D58177675582F963A782D4631480
:1028C00082FFFF7798CF83E29B5584999BE38438FE
:1028D000984C847798CF837798CF83FFFF0868D38D
:1028E0008348685084E764E8849E645A84FFFF4903
:1028F00097B985889A84861D9A0C87EB962E86490F
:1029000097B9854997B985FFFF3869BD85976934BF
:102910008665661087F9658986FFFFA2958587A57C
:1029200098928818980F892795F287A2958587A293
:10293000958587FFFFDF6A8A875B6BF8876A681473
:1029400089DC679788DF6A8A87FFFFF76C2F898D9C
:102950006D9189EB6AE98A406A798AFFFF80933238
:10296000894596728A3E96778A9995E38AF5928D83
:10297000898093328980933289FFFF1091A18A6FF9
:10298000931F8CAA92808C6490F78A1091A18A1070
:1029900091A18AFFFF736FA58A2170FB8A357004AD
:1029A0008BED6D8B8CE16D878C176D238CFFFF3E5B
:1029B0008EE18B37908B8D598FDC8D7C8D278C3EF3
:1029C0008EE18B3E8EE18BFFFF5972EB8B1B7331D7
:1029D0008C4071E78D6470978DFFFF218BE38CA98C
:1029E0008CB28EBA8BEF8E518A188D218BE38C219D
:1029F0008BE38CFFFF7675EB8C4876208DE074F8C6
:102A00008EF273BB8EFFFFF3662F8D74688A8D7D07
:102A1000688F8D8668948D26696E8E8768488F05CD
:102A200067A28F8465498F7F65458F70653E8F7380
:102A3000653E8FD364638E7365898DF3662F8DF346
:102A4000662F8DFFFF9399318D139B8C8DB49B6600
:102A50008E169B408F93999A8F1498408F74976627
:102A60008E12988C8D9399318D9399318DFFFFCD76
:102A700087A18DDC888B8FE087B58FF086C68DCDE2
:102A800087A18DCD87A18DFFFFCD78A88DA879CBAB
:102A90008DBC78BB8FC177928FFFFF5084198EE277
:102AA000841490E08329906C832C8E5084198E506E
:102AB00084198EFFFF487C1C8E2B7D2E8EBD7C2CB6
:102AC00090BB7B1790487C1C8EFFFFBF80498ED245
:102AD000804A90CC7F4A90D97F498EBF80498EBF73
:102AE00080498EFFFF4F802193D0817A9371825568
:102AF00094D1812F9551808A95CF7E30952F7E5627
:102B000094CE7E7B934F8021934F802193FFFF488B
:102B100080D946BC27BA9DD3D8BA9DFFFF4880C94B
:102B20004B2E954A60626B4A60FFFFD268CE62BF4F
:102B300097CE62BAB9278439A2369B165E369BB609
:102B4000464684D268CE62FFFF3EBC9F863BD136AC
:102B50009B42A7369BFFFF3144BE860E59369B54DD
:102B60002F369B3144BE86D5D820A5A5D863A52E87
:102B7000D87FA548D37FA5D1D298A5A0D2D9A5A0AA
:102B8000D27AAF74D2BEAF02D2DAAF37CDDAAFBFEE
:102B9000CCBEAF8FCC7AAF8FCCD9A563CC98A5F142
:102BA000CB7FA50BC77FA594C663A564C620A5648B
:102BB000C68CA20BC72CA22ED82CA2A5D848A2D571
:102BC000D88CA2FFFF38B18CAC52B98CAC52B97F13
:102BD000A538B17FA5FFFF27BF21A457BF76A46DFD
:102BE000BFD0A46DBF36AD57BF90AD27BFE6ADFADD
:102BF000BBB2AF60BBCFAFBDBADAAFCEAFDAAF30EA
:102C0000AFCFAF9AAEB2AF6EABE6AD39AB90AD28F9
:102C1000AB36AD28ABD0A439AB76A46EAB21A49A69
:102C2000AE55A230AF39A2CEAF2CA2BDBA2CA26055
:102C3000BB39A2FABB55A2FFFFA493DCACEA9CDC33
:102C4000ACEA9C34AAA49334AAA493DCACFFFFA4FE
:102C50009396A7EA9C96A7EA9C25A5A49325A5FF91
:102C6000FF27A221A458A278A46EA2D5A46EA20028
:102C7000A74FA257A704A2A5A789A0B8A861A0033F
:102C8000A992A049A9FCA143AA4BA291AA6EA2E8CD
:102C9000AA6EA236AD58A290AD27A2E6ADFC9EB2B8
:102CA000AF619ECFAFBE9DDAAFD08EDAAF288E7AFD
:102CB000AF288E8CA2598E48A2D08E2CA2BE9D2CFD
:102CC000A2619E39A2FC9E55A2FFFF3C8502A5177A
:102CD0008557A5C984A2A59479C8AC9484C8AC0AC8
:102CE00085E4AC3C8527AD3C857AAF0A85BEAF94C0
:102CF00084DAAF7173DAAFC9727AAFC97209ADE81D
:102D000072B2AC337364ACA57E3EA5A6733EA52F0C
:102D10007322A5FE72DFA4FE728CA22F7348A2A6B6
:102D2000732CA294842CA20A8548A23C858CA2FF15
:102D3000FF686B87ACDB6BA3AC076CE6AC076C7A07
:102D4000AFDB6BBEAF686BDAAF845CDAAFDC5B7AAB
:102D5000AFDC5B8CA2845C2CA246612CA2EE618C61
:102D6000A2EE612DAC1E626EAC956287ACFFFFC611
:102D70005248A2F7528CA2F75245ADEE5245ADDC57
:102D8000529BADB152E6AD854FB2AFEA4ECFAF47E1
:102D90004EDAAF5943DAAFBA42CFAF2442B2AFF8FE
:102DA0003EE6ADC33E90ADB23E36ADB23E8CA2E241
:102DB0003E48A25A3F2CA21B442CA2934448A2C3D3
:102DC000448CA2C3442DACF44471AC6B458CAC3E36
:102DD0004C8CACB14C71ACDD4C2DACDD4C8CA20DEF
:102DE0004D48A2854D2CA24F522CA2FFFF48378799
:102DF000ACBB37A3ACE737E6ACE7377AAFBB37BE3F
:102E0000AF4837DAAF6428DAAFBC277AAFBC278C7B
:102E1000A264282CA2262D2CA2CD2D8CA2CD2D2D46
:102E2000ACFE2D6EAC752E87AC9FDB0CAC6FDA2D33
:102E3000AC70D991ACC0D823AD85D8CFADC0D87A0D
:102E4000AE70D90CAF6FDA6FAF9FDB8FAFCEDC6F98
:102E5000AFD0DD0CAF7DDE7BAEB9DECFAD7DDE2247
:102E6000ADD0DD91ACCEDC2DACFFFF9FDBC3ABFE64
:102E7000DCEAAB28DE5EACF1DE06AD36DFCFADF1CD
:102E8000DE95AE28DE3EAFFEDCB1AF9FDBD8AF3FB4
:102E9000DAB1AF16D93EAF49D895AE08D8CFAD4913
:102EA000D806AD16D95EAC3FDAEAABFFFF7DDBE6B4
:102EB000ACE4DAE6ACE4DAA9AD7DDBA9AD3BDC94A9
:102EC000AD71DC48AD3BDCFDACFFFF85DB9EACCBE0
:102ED000DCC8AC37DD47ADF6DCACAD3EDCDEAD8545
:102EE000DCFFADE8DC4EAE92DDEAAEBDDCEAAE1E44
:102EF000DC58AEA7DB03AE36DBEFADE4DAEFADE4D2
:102F0000DAEAAE26DAEAAE26DA9EAC4880D946BCCA
:102F100027BA9DD3D8BA9D00436C69636B20736F49
:102F2000756E647300496E746572666163652053E3
:102F30006F756E647300536F756E6420766F6C7579
:102F40006D65005072696E74206572726F72005008
:102F500072696E742066696E697368656400507288
:102F6000696E74207374617274696E670042616384
:102F70006B004E6F00596573004C6F6164696E673A
:102F80002073657474696E672066726F6D204545A5
:102F900050524F4D0A0057726974696E672073650D
:102FA0007474696E6720746F20454550524F4D0A06
:102FB00000496E7465726661636520536F756E6457
:102FC0007300426F6F742073637265656E005363A4
:102FD0007265656E206C6F636B00536F756E642055
:102FE000766F6C756D65004C43442062726967684A
:102FF000746E65737300496E7465726661636520F3
:1030000053657474696E6773004261636B004E6F41
:10301000005965730047323800473238205A00475C
:1030200032382059004732382058006D6D00450075
:103030005A00590058004D6F766520417869730039
:103040004C696E65617220416476616E636500490A
:103050006E746572666163652053657474696E672A
:103060007300446973706C617900486F6D6520531B
:10307000656E736500526573746F72652044656692
:1030800061756C747300456E6473746F7073004384
:10309000757272656E7473004261636B6C61736804
:1030A000004A65726B00416363656C6572617469A7
:1030B0006F6E0056656C6F6369747900546F6F6C46
:1030C000204F6666736574730053746570732F6D5B
:1030D0006D004261636B004F6B6179004E6F005968
:1030E000657300546F7563682074686520646F743D
:1030F0007320746F2063616C696272617465005241
:10310000656C6561736520746F20626567696E2008
:1031100073637265656E2063616C69627261746964
:103120006F6E006D6D2F73C2B200416D61782045E6
:103130003100416D6178205A00416D61782059005D
:10314000416D6178205800416363656C65726174FC
:10315000696F6E00313233343536373839300071AB
:10316000776572747975696F7000617364666768FA
:103170006A6B6C20007A786376626E6D213F3C004A
:10318000456E7465722050617373636F64653A00B5
:1031900053656C6563742050617373636F64653A43
:1031A0000050617373636F6465206163636570745D
:1031B0006564210057726F6E672070617373636F6F
:1031C0006465210043616E6E6F74206F70656E20C0
:1031D000535441525455502E41564900506C65612C
:1031E000736520646F206E6F742072756E20746832
:1031F0006973207465737420756E617474656E6490
:103200006564206173206974206D61792063617544
:10321000736520796F7572207072696E74657220A3
:10322000746F206D616C66756E6374696F6E2E00CD
:10323000446576656C6F706572204D656E750053E0
:10324000686F7720416C6C20576964676574730000
:1032500053747265737320546573740053686F7789
:1032600020546F7563682052656769737465727363
:1032700000506C617920536F6E6700506C6179204B
:10328000566964656F2066726F6D204D6564696173
:1032900000506C617920566964656F2066726F6DAD
:1032A0002053504920466C617368004C6F61642064
:1032B000566964656F20746F2053504920466C61D5
:1032C00073680045726173652053504920466C61F4
:1032D0007368004261636B004732380A47302058F8
:1032E000313135205A35302046363030300A4D34B1
:1032F00030300A4D3138205820590041626F7574C2
:1033000020746F206D6F766520746F20686F6D6517
:1033100020706F736974696F6E2E20456E737572BD
:10332000652074686520746F7020616E6420746815
:103330006520626564206F6620746865207072691C
:103340006E7465722061726520636C6561722E0A0D
:103350000A436F6E74696E75653F004730205831BF
:1033600030302059313030205A313030204636301C
:1033700030300A54300A47342053310A473020583D
:103380003135302059313530205A3135300047320F
:1033900038005465737420333A205072696E746536
:1033A000722077696C6C20726573746172742E0080
:1033B0005465737420323A205072696E74657220BD
:1033C00077696C6C20726573746172742E00546539
:1033D000737420313A20537472657373207465736B
:1033E00074696E672E2E2E004D3530300045786999
:1033F00074004E75646765204E6F7A7A6C65006D57
:103400006D005A0059005800446F6E6520706C6161
:1034100079696E6720766964656F0A0054696D6525
:103420006F757420706C6179696E67207669646568
:103430006F0A005374617274696E6720746F207034
:103440006C617920626F6F7420766964656F0A0021
:103450005374617274696E6720746F20706C617947
:1034600020535441525455502E4156490A0053544A
:1034700041525455502E41564900473131320A4D80
:10348000313137204C6576656C696E672058204174
:103490007869730A4732380A47302058313730206C
:1034A0005937352046393939390A4730205A3520BD
:1034B00046363030300A4739310A4D3231312053E7
:1034C000300A4D3430300A4D393036205A363030DB
:1034D0000A4730205A2D313520463530300A4730E2
:1034E000205A3520463530300A4D3430300A4739BD
:1034F000300A4D393036205A3936300A4D323131A2
:103500002053310A473238205A300A4D31313720A2
:103510004C6576656C696E6720646F6E652E0A4730
:10352000302058313135205A353020463630303051
:103530000A4D3430300A4D3138205820590041624C
:103540006F757420746F206175746F2D6C6576656E
:103550006C20616E642072652D686F6D6520706CE3
:10356000756E6765722E2052656D6F766520737972
:1035700072696E6765207072696F7220746F207057
:10358000726F63656564696E672E0A0A436F6E74B5
:10359000696E75653F00253364255320282553291E
:1035A00000253364202F2025336425530025336400
:1035B0002553202F202553002533642553006964AB
:1035C0006C6500C2B043004D313137204C657665E3
:1035D0006C696E67205820417869730A4732380A4F
:1035E000473020583137302059373520463939395E
:1035F000390A4730205A352046363030300A4739AC
:10360000310A4D3231312053300A4D3430300A4DB9
:10361000393036205A3630300A4730205A2D31356D
:1036200020463530300A4730205A35204635303074
:103630000A4D3430300A4739300A4D393036205A75
:103640003936300A4D3231312053310A4732382071
:103650005A300A4D313137204C6576656C696E679A
:1036600020646F6E652E00473131320047302045AF
:10367000302046313230004265642054656D7065FB
:10368000726174757265004175746F2D6C65766535
:103690006C205820417869730052656C65617365D0
:1036A000205820616E64205920417869730052616E
:1036B00069736520506C756E676572004D6F766535
:1036C00020746F20486F6D65004D61696E204D65F7
:1036D0006E7500496E74657266616365205365742A
:1036E00074696E67730041626F7574205072696E01
:1036F00074657200416476616E636564205365741D
:1037000074696E6773004261636B0073742F6D6D33
:103710000045005A005900580053746570732F6DAE
:103720006D0043616368656453637265656E3A3A20
:1037300073746F72654261636B67726F756E642834
:1037400029206661696C65643A206E6F7420656E2D
:103750006F75676820444C206361636865207370EF
:103760006163650A0046696C616D656E742055730E
:103770006564004C6F6E67657374205072696E7477
:1037800000546F74616C205072696E742054696DBE
:103790006500546F74616C205072696E74730050D0
:1037A00072696E7420436F756E74005072696E7426
:1037B0006572205374617469737469637300426144
:1037C000636B006D6D2F7300566D6178204531007D
:1037D000566D6178205A00566D6178205900566DFB
:1037E000617820580056656C6F63697479004730C2
:1037F0002045302046313230004265642054656DEA
:1038000070657261747572650052656C656173658F
:10381000205820616E6420592041786973005261FC
:1038200069736520506C756E676572004D6F7665C3
:1038300020746F20486F6D65005072696E74204D62
:10384000656E75004E75646765204E6F7A7A6C659B
:10385000005072696E742053706565640042616344
:103860006B00506C65617365207265736574005000
:1038700052494E5445522048414C5445440025007D
:103880006D6D005A0059005800436F727265637481
:10389000696F6E00536D6F6F7468696E6700426187
:1038A000636B6C6173680053616D706C6520576960
:1038B00064676574730053686F7720677269643A50
:1038C000006E6FFF79657300310032004261636BF7
:1038D0000041726520796F75207375726520796F6C
:1038E000752077616E7420746F2063616E63656C00
:1038F00020746865207072696E743F0042656420B0
:1039000054656D706572617475726500436F6F6C9C
:10391000646F776E2028416C6C204F66662900C268
:10392000B04300426564005370656564005072697D
:103930006E742053706565640025004261636B00FE
:1039400030782530386C580030782530386C580085
:1039500030782530386C580030782530386C580075
:1039600030782530386C580030782530386C580065
:10397000544F5543485F58464F524D5F4100544F96
:103980005543485F58464F524D5F4200544F554390
:10399000485F58464F524D5F4300544F5543485F70
:1039A00058464F524D5F4400544F5543485F584668
:1039B0004F524D5F4500544F5543485F58464F5254
:1039C0004D5F46000000000000004C756C7A426FAD
:1039D000742042696F004669726D77617265206676
:1039E0006F7220746F6F6C686561643A0A25730AA0
:1039F0000A00C2A9203230313920416C657068203C
:103A00004F626A656374732C20496E632E0A0A77CD
:103A100077772E6C756C7A626F742E636F6D004FC2
:103A20006B6179005374617274207072696E74698D
:103A30006E672025733F005072696E742073746145
:103A40007274696E6700473238205A004D31370072
:103A5000426564004D38342058590046696E65202F
:103A60006D6F74696F6E005072696E74696E670075
:103A70004D65646961004D656E75004E6F00596556
:103A80007300018181800181818000C0C0C000C0BD
:103A9000C0C0006060600060606000C0C0C000C066
:103AA000C0C0018181800181818003030300030381
:103AB00003000606060006060600030303000303D0
:103AC0000300018181800181818000000000FFFFEF
:103AD000FFFFFFFFFFFFC0000003FFFFFFFFB1C9B3
:103AE0001E3290D91E3290D900207FE10020A0D153
:103AF000F116C2C10020B1C90020B1C91E32B1C93E
:103B00002D3B90D92D3B90D94B4D7FE14B4DA0D112
:103B10005A56C2C14B4DB1C94B4DB1C92D3B109C3A
:103B2000D2C6A3E4D2C6A3E416D3109C16D3A71A18
:103B3000D2C68793D2C6879316D3A71A16D3641713
:103B4000281235612812356184266417842664178B
:103B50006F4635616F463561CB5A6417CB5A64178F
:103B60004C2C35614C2C3561A8406417A8404FB9E6
:103B7000AA25D89D3A35B6A43A35B6A4C94471B23F
:103B8000C94471B2023D2CC0023D2CC0C944E7CDEE
:103B9000C944E7CD3A35C5D43A3528CA362F28CAA4
:103BA000AB274BC3AB274BC3532BC9D6CC8053BBDE
:103BB0005B9031C25B9031C2EB9FECCFEB9FECCFBF
:103BC0002398A7DD2398A7DDEB9F62EBEB9F62EBC9
:103BD0005B9040F25B90A3E7588AA3E7CD82C6E0F2
:103BE000CD82C6E074865A6417809E5FA180BA5B5E
:103BF0001B8211594A840A58F7860A58318970592C
:103C0000988A495C988AB05D3189B05D03873C5ED3
:103C10008E85AA5F5F84C56194835A644A83F06687
:103C200094830C695F847A6A8D85076B0387076BC1
:103C3000238FC857238F1E55C38F045445910454B6
:103C40008F9C1E55119EC857B19EEE70B19E987301
:103C5000119EB2748F9CB27445919873C38FEE70AD
:103C6000238FAC70FA86A56F4A84FD6C1B8217699E
:103C7000A180C77A4B0FC77A4A135B854A135B85CD
:103C80004919C77A4919C77A404B5B85404D5B8516
:103C90003F53E2883F53E2883C65698C3C67698CFE
:103CA0003F53F08F3F53F08F404D859A404B859A9C
:103CB0004919F08F4919F08F4A13859A4A13859A4A
:103CC0004B0FC77A4B0FC283AA42C283FF432C8D8E
:103CD000FF432C8DAA42FFFFC283543DC283AA3EFC
:103CE0002C8DAA3E2C8D543DFFFFC283FF37C2832B
:103CF00054392C8D54392C8DFF37FFFFC283AA32E3
:103D0000C283FF332C8DFF332C8DAA32FFFFC28379
:103D1000542DC283AA2E2C8DAA2E2C8D542DFFFF3C
:103D2000C283FF27C28355292C8D55292C8DFF274F
:103D3000FFFFC283AA22C283FF232C8DFF232C8D79
:103D4000AA22FFFFC77A4B0FC77A4A135B854A1333
:103D50005B854919C77A4919C77A404B5B85404D45
:103D60005B853F53E2883F53E2883C65698C3C6742
:103D7000698C3F53F08F3F53F08F404D859A404BF5
:103D8000859A4919F08F4919F08F4A13859A4A1379
:103D9000859A4B0FFFFFE2884A13698C4A13698C9E
:103DA0004919E2884919E2884A13FFFF4D7E491BF1
:103DB000FE96491BFE964149698C404BE288404B78
:103DC0004D7E41494D7E491B1D7D0F4AFC870E4C9F
:103DD000F48C0E4C01980F4A0198A21A1D7DA21A6C
:103DE0001D7D0F4A6675B38DC96E8C9522938C9597
:103DF000D48F79999EA8A0910E9DC789C099B38D43
:103E00006675B38D3D51B38DA04A8C9547268C9530
:103E1000F82279996917A0913330C789E42CB38DC2
:103E20003D51B38D725DC7899F6FC789DA7C157A62
:103E3000F085157A617A3D729761157AAD6A157AC7
:103E4000725DC789375079996462799929552AA991
:103E50003F5E2AA9754503B1E6392AA9FC422AA981
:103E600037507999B1C9A48D90D9A48D90D9867B0A
:103E70007FE1867BA0D17772C2C1867BB1C9867B88
:103E8000B1C9A48DB1C9B39690D9B39690D9D0A831
:103E90007FE1D0A8A0D1DFB1C2C1D0A8B1C9D0A85C
:103EA000B1C9B3964D35303000446F20796F75201D
:103EB0007769736820746F20736176652074686514
:103EC00073652073657474696E6773206173206411
:103ED000656661756C74733F0053657474696E67D1
:103EE0007320736176656421004D35303200417274
:103EF0006520796F7520737572653F204375737403
:103F00006F6D697A6174696F6E732077696C6C206C
:103F10006265206C6F73742E0053657474696E67EC
:103F20007320726573746F72656420746F206465AA
:103F30006661756C74004B004C696E65617220415E
:103F40006476616E63650053504920666C617368E6
:103F5000206572617365640045726173696E672ED6
:103F60002E2E0041726520796F7520737572653F42
:103F70002053504920666C6173682077696C6C200F
:103F80006265206572617365642E006D6D2F73002C
:103F900045005A00590058004A65726B0053657419
:103FA000204D6178696D756D006D6D2F73C2B20023
:103FB00052657472616374696F6E005472617665E4
:103FC0006C005072696E74696E6700416363656C62
:103FD00065726174696F6E00486F6D652053656E20
:103FE0007365005A00590058004361636865645363
:103FF000637265656E3A3A73746F72654261636BA2
:1040000067726F756E642829206661696C65643A11
:10401000206E6F7420656E6F75676820444C206356
:10402000616368652073706163650A004D656E7534
:10403000004261636B0043616E63656C0025303242
:10404000646820253032646D0046696E6973686566
:10405000642E005072696E74696E672E2E2E0000F9
:1040600043616C69627261746500546F75636820A6
:1040700053637265656E0056204F66667365740003
:1040800048204F666673657400446973706C61798B
:104090000043616368656453637265656E3A3A73A1
:1040A000746F72654261636B67726F756E64282905
:1040B000206661696C65643A206E6F7420656E6F6E
:1040C00075676820444C2063616368652073706184
:1040D00063650A00506C6561736520776169742EB1
:1040E0002E2E0098C31D9B99C3D06D9D66C06A9A01
:1040F000C39CC39EC398C3C58099C356816E806F0D
:10410000809AC39CC39EC398C31D9B99C303AAAC4A
:10411000A9D1B4B2A706A8BCA798C31D9B99C38A0E
:104120009B83CA46909AC39CC3099098C31D9B99D0
:10413000C38A9B2BCA6C979AC39CC3409798C31D94
:104140009B99C38A9BD3C9DB7C9AC39CC3A17C98EF
:10415000C32BB599C3A47F7AC927B59AC39CC398CA
:104160007F98C32BB599C3A47F7AC90C939AC39C3B
:10417000C30E9398C31D9B99C3A47F9D66E7B59A10
:10418000C39CC3F0B598C31D9B99C3A47F9D669E35
:10419000B59AC39CC3A7B598C309A699C3A47F9D2C
:1041A0006635A69AC39CC37BA698C31D9B99C3A4DE
:1041B0007F9D66D3A09AC39CC3DCA098C31D9B9926
:1041C000C36BC321C903C39AC39CC3987F98C3DD43
:1041D000A499C38A9B9D66F9A49AC39CC3E6A4983C
:1041E000C31D9B99C38A9B9D664F949AC39CC37FB2
:1041F0009398C3188B99C3938CC9C8238B9AC3DB3C
:104200008B8B8C98C3677A99C3787C1C7C717A9A63
:10421000C30B7B455F98C32D5F99C38A9B71C8CF41
:10422000919AC35392455F98C32D5F99C38A9B1996
:10423000C89A689AC31869455F98C32D5F99C38A65
:104240009BC1C734B99AC3B6B9455F98C32D5F996E
:10425000C38A9B69C7AE999AC3549A455F98C32D88
:104260005F99C38A9B11C7B5A19AC3F5A1455F9811
:10427000C32D5F99C38A9BB9C69E959AC322964562
:104280005F98C32D5F99C38A9B61C682819AC306DA
:1042900082455F98C32D5F99C38A9B09C633B89A3C
:1042A000C398B8455F98C32D5F99C38A9BB1C5F683
:1042B000B69AC37AB7455F98C32D5F99C38A9B5955
:1042C000C5DC5C9AC39CC3F45B98C32D5F99C38A19
:1042D0009B01C522B69AC367B6455F98C32D5F9907
:1042E000C38A9BA9C403A19AC354A1455F98C3FC88
:1042F000D30ED4E4D851C4EAD4D1D499D449D4EF5C
:1043000074F07499C3D6797E79B7772C759CC3FE07
:104310007498C39F6E99C362730C73BD70C96E9C11
:10432000C3A56E98C3BD8299C38A9BEF842B839AE1
:10433000C39CC3898598C396CD99C352CEF8C33C1C
:10434000D19AC39CC3A9CD98C3E266E766F4669D83
:104350006604679AC39CC3EA6698C31D9B99C3B45D
:10436000C15BC1BCC09AC39CC31CBB98C31D9B99B5
:10437000C3A47F9D66F7879AC39CC3008898C31D1A
:104380009B99C3A47F9D66958E9AC39CC39E8E986D
:10439000C31D9B99C38A9B9D6666869AC39CC32650
:1043A0008698C31D9B99C3A47F9D66BDB69AC39C86
:1043B000C3C6B698C3FB9B99C3189D9D666B9D01B0
:1043C0009C9CC39EC398C31D9B99C38A9B9D6650AA
:1043D000A29AC39CC346A298C3BB8999C30D8A9D68
:1043E00066428A9AC39CC38C8998C3B08C99C38A4D
:1043F0009B9D66B78C9AC39CC39EC398C32D5F993F
:10440000C38A9BA0C3DFC19AC351C2455F436163A6
:1044100068656453637265656E3A3A73746F72656A
:104420004261636B67726F756E64282920666169EB
:104430006C65643A206E6F7420656E6F75676820D6
:10444000444C2063616368652073706163650A0092
:10445000003C003E0050616765202564206F6620A7
:104460002564003E20005072696E74004F70656EC6
:10447000004261636B003100320000436F6E74696B
:104480006E756F7573004D6F6D656E746172790036
:104490004C6F61642F4578747275646500556E6C5D
:1044A0006F61642F5265747261637400486F742188
:1044B0000043617574696F6E3A0048656174696E96
:1044C000670052656D6F76616C2054656D700045B4
:1044D000787472756465722053656C656374696F76
:1044E0006E00486967680041425300504C410042E9
:1044F00061636B0000FF00001006F4441806D44806
:104500002006F8482706B4482F06E4483C068C45A8
:10451000450644454D063C45530634455A062C4550
:1045200063064C456906D44572068046083C400047
:1045300000FF0000073C400000FF0000063C400078
:1045400000FF0000053C400000FF000000000800E4
:10455000533C0800553C0800543C0800523C0800FD
:1045600000000800533C0800553C0800543C08007B
:10457000523C080000000800533C0800553C08006D
:10458000543C0800523C080000FF00004141030079
:104590004143030041410300413E0300413A03000F
:1045A000000003004541030045430300454103006B
:1045B000453E0300453A030000000300422E06007A
:1045C000422E0600422E0400422E0600422E060015
:1045D00000FF00004637040046390400463B040053
:1045E000463E030000000100463C030000000100BD
:1045F000463C04004640030000000100463E020025
:1046000000000200463E0400464303000000010093
:104610004642040046430400463E020000000200F9
:10462000463B030000000100463704004639020003
:1046300000000200463B020000000200463C04006D
:10464000463E020000000200464002000000020058
:10465000463E0400463C020000000200463B0200C9
:104660000000020046390400463B02000000020040
:1046700046370200000002004637080000FF000035
:1046800044450200444302004445230000000C005E
:10469000444304004441040044400400443E0400F8
:1046A000443D1000443E200000002A00443902002E
:1046B0004437020044392300000009004434080054
:1046C000443508004431100044321B0000002A0029
:1046D000442D0200442B0200442D230000000C0056
:1046E000442B040044290400442804004426040008
:1046F0004425100044262000000034004431090005
:104700004434090044370900443A0900443D090093
:1047100044400900443E140000001E00443D0400D3
:10472000443E020044400200443D0200443E020078
:1047300044400200443D0200443E02004440020066
:10474000443D0200443E0400444004004441020051
:10475000444302004440020044410200444302003A
:10476000444002004441020044430200444002002D
:10477000444104004443040044450200444602000E
:104780004443020044450200444602004443020000
:1047900044450200444602004443020044450400EC
:1047A0000000240044490400444A0200444C020032
:1047B00044490200444A0200444C020044490200B9
:1047C000444A0200444C020044490200444A0400A6
:1047D000444C0400444D0200444F0200444C02008B
:1047E000444D0200444F0200444C0200444D02007C
:1047F000444F0200444C0200444D0400444F040066
:104800004451020044520200444F0200445102004D
:1048100044520200444F020044510200445202003C
:10482000444F0200445104000000200044510400A1
:10483000444F020044520200444C0200444F020024
:1048400044520200444C0200444D02004451020014
:10485000444A0200444D0200444F0200444A020010
:10486000444C02004451020044480200444C0200FF
:104870004451020044480200444A0200444D0200F0
:1048800044460200444A0200444C020044460200EE
:1048900044480200444C020000FF0000484002006F
:1048A000483C020000FF0000483C02004840020073
:1048B00000FF0000453904000000010045390200F6
:1048C00000000100453902000000010045400A00D7
:1048D00000FF0000433C010043400100434310003F
:1048E00000FF0000453A0A0045390A0045380A0031
:1048F0004537140000FF000047370500474005001A
:10490000473C050000FF0000556E61626C65207435
:104910006F2072656164206D656469612E004D656C
:104920006469612052656D6F766564004D656469E8
:104930006120496E736572746564004D61726C69C3
:104940006E20322E302E302E31373200256C642E00
:1049500025696D002569730025696D20256973003F
:104960002569682025696D20256973002569642003
:104970002569682025696D202569730025697920DE
:10498000256964202569682025696D2025697300E3
:104990005072696E742041626F72746564004C7568
:1049A0006C7A426F74204C756C7A426F7420426945
:1049B0006F2072656164792E005072696E74696E41
:1049C000672E2E2E005072696E74205061757365CB
:1049D000640043616E6E6F7420656E74657220733F
:1049E00075626469723A20002E0A006F70656E204D
:1049F0006661696C65642C2046696C653A200061CB
:104A000075746F25632E67006572726F72207772FE
:104A10006974696E6720746F2066696C650A004E60
:104A20006F74205344207072696E74696E670A0057
:104A30005344207072696E74696E67206279746580
:104A400020002E0A0044656C6574696F6E206661F3
:104A5000696C65642C2046696C653A200046696C77
:104A6000652064656C657465643A005772697469A1
:104A70006E6720746F2066696C653A20002E0A000C
:104A80006F70656E206661696C65642C2046696C88
:104A9000653A20002E0A006F70656E206661696CB1
:104AA00065642C2046696C653A200046696C652077
:104AB00073656C65637465640A002053697A653AAE
:104AC000200046696C65206F70656E65643A200051
:104AD0002066696C653A2000667265736800646FD1
:104AE000696E67004E6F772000454E442053554253
:104AF000524F5554494E450A002220706F730022D0
:104B000020706172656E743A2200535542524F55BF
:104B100054494E452043414C4C2074617267657482
:104B20003A2200747279696E6720746F2063616C39
:104B30006C207375622D67636F64652066696C65B0
:104B400073207769746820746F6F206D616E7920AF
:104B50006C6576656C732E204D4158206C657665CA
:104B60006C2069733A310A004D3234004D323320E3
:104B700025730053442063617264206F6B0A006FD9
:104B800070656E526F6F74206661696C65640A00AF
:104B9000766F6C756D652E696E6974206661696CDF
:104BA00065640A00534420696E6974206661696C0B
:104BB0000A00286E6F2066696C65290043616E6E7D
:104BC0006F74206F70656E20737562646972200067
:104BD0007C3C3E5E2B3D3F2F5B5D3B2C2A225C00E4
:104BE00066616C73650074727565006563686F3A21
:104BF000004572726F723A004572726F722077725E
:104C00006974696E6720746F20454550524F4D217D
:104C10000A004C4F570048494748004F4B00457227
:104C2000726F723A20416C6C200020636F6E6E656B
:104C30006374696F6E2E2E2E200054657374696E36
:104C40006720004C4F570048494748004F4B0045EC
:104C500072726F723A20416C6C200020636F6E6E2E
:104C6000656374696F6E2E2E2E200054657374690F
:104C70006E6720004C4F570048494748004F4B0093
:104C80004572726F723A20416C6C200020636F6E27
:104C90006E656374696F6E2E2E2E200054657374DA
:104CA000696E6720004C4F570048494748004F4BFA
:104CB000004572726F723A20416C6C200020636F65
:104CC0006E6E656374696F6E2E2E2E2000546573B0
:104CD00074696E672000544D4320434F4E4E454348
:104CE00054494F4E204552524F52004452565F5342
:104CF0005441545553090050574D5F5343414C455F
:104D0000090050574D434F4E460900434F4F4C4307
:104D10004F4E46090043484F50434F4E46090054FA
:104D20004849474809090054434F4F4C544852538F
:104D300009005450574D5448525309005453544598
:104D40005009090054504F574552444F574E0900DF
:104D5000494F494E09090047535441540909004934
:104D6000484F4C445F4952554E090047434F4E4609
:104D70000909000900092042616420726573706F9F
:104D80006E73652100092042616420726573706F43
:104D90006E73652100092042616420726573706F33
:104DA0006E73652100092042616420726573706F23
:104DB0006E73652100303D2E33323500313D2E318A
:104DC00038006D6178002F3331002F3331002F33DD
:104DD0003100303D2E33323500313D2E3138006DFB
:104DE0006178002F3331002F3331002F3331003001
:104DF0003D2E33323500313D2E3138006D61780063
:104E00002F3331002F3331002F333100303D2E331B
:104E1000323500313D2E3138006D6178002F33314D
:104E2000002F3331002F33310044726976657220D0
:104E30007265676973746572733A0A006F7409006A
:104E40006F747077090073326761090073326762AB
:104E500009006F6C6109006F6C62090073747374F0
:104E600009006673616374697665090073675F7230
:104E70006573756C74007374616C6C6775617264D2
:104E80000900445256535441545553005374616CB5
:104E90006C67756172642074687273002D7374613D
:104EA00072740900687973746572657369730A2D89
:104EB000656E640900626C616E6B2074696D6500DB
:104EC0006F66662074696D65004F54207072657757
:104ED00061726E206861730A6265656E2074726922
:104EE000676765726564004F542070726577617200
:104EF0006E005B6D6D2F735D090070776D0A7468CD
:104F0000726573686F6C6400747374657009006D0A
:104F100073746570730900737465616C74684368B9
:104F20006F70007673656E7365090050574D20737E
:104F300063616C650043532061637475616C004864
:104F40006F6C642063757272656E740052756E20AA
:104F500063757272656E74004D415820637572728C
:104F6000656E7400524D532063757272656E7400E5
:104F70005365742063757272656E7400456E61626C
:104F80006C656409000900617869733A70776D5F38
:104F90007363616C652F637572725F7363616C65B7
:104FA0002F6D6563685F6C6F61647C666C616773AD
:104FB0007C7761726E636F756E740A006D41290AA9
:104FC0000020647269766572206F76657274656D13
:104FD0007065726174757265207761726E696E6753
:104FE000212028003A20002063757272656E7420BB
:104FF00064656372656173656420746F20006D4140
:10500000290A0020647269766572206F7665727471
:10501000656D7065726174757265207761726E6915
:105020006E67212028003A20002063757272656E39
:10503000742064656372656173656420746F200019
:105040006D41290A0020647269766572206F766569
:105050007274656D706572617475726520776172C6
:105060006E696E67212028003A20002063757272F5
:10507000656E742064656372656173656420746F26
:10508000200025753A2530327500253032753A25D5
:105090003032750025756420253032753A2530325E
:1050A00075006D41290A0020647269766572206F6F
:1050B00076657274656D706572617475726520775E
:1050C00061726E696E67212028003A2000206375A6
:1050D0007272656E742064656372656173656420C5
:1050E000746F2000447269766572206572726F7207
:1050F00000636F696C2073686F72742063697263F8
:105100007569740A006F76657274656D7065726199
:10511000747572650A002064726976657220657222
:10512000726F722064657465637465643A203078C8
:105130000063616E63656C00726573756D65007008
:105140006175736500706F7765726F6666002F2FEB
:10515000616374696F6E3A0020573A00202F002077
:1051600042403A0020403A00546865726D616C20FC
:1051700052756E6177617900486F74656E64205472
:105180004845524D414C2052554E415741590042DD
:10519000454420544845524D414C2052554E4157AC
:1051A000415900202D20496E76616C696420657834
:1051B000747275646572206E756D62657220210A65
:1051C0000048656174696E67206661696C6564009A
:1051D0004265642048656174696E67204661696C48
:1051E000656400546865726D616C2052756E6177FC
:1051F00061790042454420544845524D414C20526B
:10520000554E415741590048656174696E67206683
:1052100061696C656400486F74656E6420486561FF
:1052200074696E67204661696C65640054686572D4
:105230006D616C2052756E6177617900486F74659D
:105240006E6420544845524D414C2052554E4157B2
:105250004159004D494E54454D502074726967675D
:105260006572656400486F74656E64204572723AB9
:10527000204D494E54454D50004572723A204D49DB
:105280004E54454D5020424544004D415854454DE3
:10529000502074726967676572656400486F746551
:1052A0006E64204572723A204D415854454D50006D
:1052B0004572723A204D415854454D502042454464
:1052C00000626564002C2073797374656D207374BB
:1052D0006F7070656421204865617465725F494430
:1052E0003A200023646566696E6520444546415551
:1052F0004C545F004B6420004B6920004B70200031
:105300000062656400504944204175746F74756E85
:10531000652066696E697368656421205075742024
:10532000746865206C617374204B702C204B69206D
:10533000616E64204B6420636F6E7374616E74736E
:105340002066726F6D2062656C6F7720696E746F76
:1053500020436F6E66696775726174696F6E2E683F
:105360000A00504944204175746F74756E6520665B
:1053700061696C6564212074696D656F75740A00DC
:10538000546865726D616C2052756E617761790049
:10539000486F74656E6420544845524D414C20520C
:1053A000554E415741590042454420544845524DBD
:1053B000414C2052554E415741590048656174692E
:1053C0006E67206661696C656400486F74656E6421
:1053D0002048656174696E67204661696C65640088
:1053E0004265642048656174696E67204661696C36
:1053F000656400504944204175746F74756E652072
:105400006661696C6564212054656D7065726174B4
:1054100075726520746F6F20686967680A00204B99
:10542000643A2000204B693A2000204B703A20005B
:105430000A20436C617373696320504944200A0059
:10544000204B643A2000204B693A2000204B703AF0
:1054500020000A204E6F206F76657273686F6F743C
:105460000A002054753A2000204B753A2000206D28
:1054700061783A2000206D696E3A200020643A205D
:105480000020626961733A200050494420417574DC
:105490006F74756E652073746172740A00504944AC
:1054A000204175746F74756E65206661696C656402
:1054B000212054656D706572617475726520746F1A
:1054C0006F20686967680A001000AD0330016A0147
:1054D00050022B0170030A019004F500B005E500AD
:1054E000D006D800F007CE001009C500300ABE0073
:1054F000500BB700700CB100900DAB00B00EA600C1
:10550000D00FA200F0109D001012990030139500EA
:105510005014920070158E0090168B00B017870003
:10552000D0188400F0198100101B7E00301C7B0015
:10553000501D7900701E7600901F7300B02070001F
:10554000D0216E00F0226B00102469003025660027
:10555000502663007027610090285E00B0295C002F
:10556000D02A5900F02B5600102D5400302E510037
:10557000502F4E0070304B0090314800B032450043
:10558000D0334200F0343E0010363B003037370055
:105590005038330070392E00903A2900B03B230078
:1055A000D03C1B00F03D1100103F0100F03F000017
:1055B0001000C90210012C014001220170011801E4
:1055C000B0010E01F00104015002FA00B002F00037
:1055D0003003E600D003DC009004D2007005C80060
:1055E000A006BE000008B400B009AA00D00BA000BD
:1055F000600E960060118C00001582002019780062
:10560000C01D6E00A0226400B0275A00902C5000EC
:1056100000314600E0343C0010383200903A280057
:10562000603C1E00A03D1400803E0A00203F0000A8
:105630006F70656E00545249474745524544003AE1
:1056400020007A5F6D6178007A5F6D696E00795F26
:105650006D617800785F6D617800785F6D696E00CC
:105660005265706F7274696E6720656E6473746FD3
:1056700070207374617475730A00205A3A002059BF
:105680003A0020583A00656E6473746F7073206836
:1056900069743A2000486F6D696E67204661696CD5
:1056A0006564000A53746174733A2046696C616DD5
:1056B000656E7420757365643A20002C204C6F6E03
:1056C00067657374206A6F623A2000546F74616C6E
:1056D0002074696D653A200053746174733A200038
:1056E0002C204661696C65643A20002C2046696E66
:1056F00069736865643A20005072696E74733A2069
:105700000053746174733A2000496E76616C696469
:105710002065787472756465720A00205A3A002018
:10572000593A0020436F756E7420583A00C2310018
:10573000001C260000F4190000D80F0000EB080040
:1057400000C0040000750200004001000024F4D4F1
:105750003050C38E20C2A24017828B7011127A91F2
:105760000D816CD90AA861E108C7586607615143E9
:10577000061E4B5D05C145A7041A411104093D9859
:1057800003713931034036DB0265339102D4305462
:1057900002802E1D02632CEE01752AC501B028A0DF
:1057A00001102781018F2564012B244B01E0223455
:1057B00001AC211F018D200D01801FFC00841EED16
:1057C00000971DDF00B81CD200E61BC600201BBCE2
:1057D00000641AB200B219A8000A19A0006A189948
:1057E00000D117910040178B00B516840031167E4A
:1057F00000B31579003A157300C7146F0058146A86
:1058000000EE1366008813630025135E00C7125B69
:10581000006C12570015125400C111510070114F45
:105820000021114B00D61049008D1047004610444E
:105830000002104200C00F4000800F3E00420F3CAB
:1058400000060F3B00CB0E3800930E37005C0E3580
:1058500000270E3400F30D3200C10D3100900D30E1
:1058600000600D2E00320D2D00050D2C00D90C2BE3
:1058700000AE0C2900850C29005C0C2700350C2794
:10588000000E0C2600E80B2400C40B2400A00B2300
:10589000007D0B23005A0B2100390B2100180B202F
:1058A00000F80A1F00D90A1E00BB0A1E009D0A1D2F
:1058B00000800A1D00630A1C00470A1B002C0A1BFB
:1058C00000110A1A00F7091A00DD091900C40919A4
:1058D00000AB091900920917007B0918006309172A
:1058E000004C09160036091600200916000A091591
:1058F00000F5081500E0081400CC081400B80814DE
:1059000000A4081400900813007D0812006B08130F
:10591000005808120046081200340811002308112C
:10592000001208110001081100F0071000E0071034
:1059300000D0071000C0071000B0070F00A107102B
:105940000091070E0083070F0074070F0065070E14
:105950000057070E0049070E003B070D002E070EEB
:105960000020070D0013070D0006070D00F9060CB7
:1059700000ED060D00E0060C00D4060C00C8060C75
:1059800000BC060C00B0060C00A4060B0099060C27
:10599000008D060B0082060B0077060B006C060BD1
:1059A0000061060A0057060B004C060A0042060A70
:1059B0000038060A002E060A0024060A001A060A03
:1059C000001006090007060A00FD050900F4050994
:1059D00000EB050900E2050900D9050900D0050919
:1059E00000C7050900BE050900B5050800AD05089A
:1059F00000A50509009C050800940508008C050811
:105A000000840508007C050800740508006C050783
:105A100000650508005D050700560508004E0507EE
:105A20000047050700400508003805070031050755
:105A3000002A050700230507001C050600160507B8
:105A4000000F0507000805060002050700FB040615
:105A500000F5040700EE040600E8040600E204076F
:105A600000DB040600D5040600CF040600C90406C6
:105A700000C3040600BD040600B7040600B1040517
:105A800000AC040600A6040600A00405009B040662
:105A90000095040500900406008A040500850405AD
:105AA00000800406007A04050075040500700405F2
:105AB000006B04050066040500610405005C040534
:105AC0000057040500520405004D04050048040574
:105AD00000430405003E0404003A040500350405B3
:105AE00000300404002C04050027040400230405EE
:105AF000001E0404001A0404001604050011040426
:105B0000000D04040009040500040404000004045A
:105B100000FC030400F8030400F4030400F0030491
:105B200000EC030400E8030400E4030400E00304C1
:105B300000DC030400D8030400D4030400D00304F1
:105B400000CC030400C8030300C503030024F404CD
:105B5000D9201BC40C5C0E9804C4095F0265077150
:105B600001F405F900FB04B30048048700C1036990
:105B7000005803550003034500BE023A0084023179
:105B80000053022A002902250004022000E4011C1F
:105B900000C8011900AF0117009801140084011317
:105BA00000710110006101100051010E0043010D50
:105BB0000036010B002B010B0020010B0015010921
:105BC000000C01090003010800FB000800F30008B5
:105BD00000EB000700E4000600DE000600D8000627
:105BE00000D2000600CC000500C7000500C2000579
:105BF00000BD000400B9000400B5000400B10004B9
:105C000000AD000400A9000400A5000300A20003E9
:105C1000009F0004009B0003009800030095000211
:105C20000093000300900003008D0002008B00032E
:105C30000088000200860002008400030081000248
:105C4000007F0002007D0002007B0002007900025C
:105C5000007700010076000200740002007200016B
:105C600000710002006F0002006D0001006C000274
:105C7000006A00010069000200670001006600017F
:105C80000065000100640002006200010061000183
:105C900000600001005F0002005D0001005C000187
:105CA000005B0001005A000100590001005800018A
:105CB000005700010056000100550001005400018A
:105CC0000053000000530001005200010051000188
:105CD00000500001004F0001004E0000004E000186
:105CE000004D0001004C0001004B0000004B000182
:105CF000004A00010049000100480000004800017E
:105D00000047000100460000004600010045000079
:105D10000045000100440001004300000043000171
:105D2000004200000042000100410000004100016B
:105D300000400001003F0000003F0001003E000065
:105D4000003E0001003D0000003D0001003C00005D
:105D5000003C0000003C0001003B0000003B000153
:105D6000003A0000003A000100390000003900014B
:105D70000038000000380000003800010037000043
:105D80000037000100360000003600000036000138
:105D9000003500000035000000350001003400002F
:105DA0000034000000340001003300000033000024
:105DB0000033000100320000003200000032000118
:105DC000003100000031000000310001003000000F
:105DD0000030000000300001002F0000002F000004
:105DE000002F0000002F0001002E0000002E0000F8
:105DF000002E0001002D0000002D0000002D0000ED
:105E0000002D0001002C0000002C0000002C0000E0
:105E1000002C0001002B0000002B0000002B0000D4
:105E2000002B0001002A0000002A0000002A0000C8
:105E3000002A0001002900000029000000290000BC
:105E400000290000002900010028000000280000AF
:105E500000280000002800000028000100270000A2
:105E60000027000000270000002700000027000195
:105E7000002600000026000000260000002600008A
:105E8000002600010025000000250000002500007C
:105E9000002500000025000000250001002400006E
:105EA0000024000000240000002400000024000161
:105EB0000023000000230000002300000023000056
:105EC0000023000000230000002300010022000046
:105ED000002200000022000000220000002200003A
:105EE000002200010021000000210000002100002C
:105EF000002100000021000000210000002100011D
:105F00000020000000200000002000000020000011
:105F10000020000000200000002000000020000100
:105F2000001F0000001F0000001F0000001F0000F5
:105F3000001F0000001F0000001F0001001E0000E5
:105F4000001E0000001E0000001E00000020204D6A
:105F50003931340020204D3931330020204D393083
:105F6000360020286D6D2900205300205A0020594A
:105F70000020580020204D34323520460042616315
:105F80006B6C61736820636F6D70656E73617469AB
:105F90006F6E3A0A0020204D393030204B004C699A
:105FA0006E65617220416476616E63653A0A0054E1
:105FB00030204500205A00205900205800447269C2
:105FC000766572207374657070696E67206D6F649A
:105FD000653A0A002059002058005374616C6C47E0
:105FE00075617264207468726573686F6C643A0AD4
:105FF00000205430204500205A002059002058002D
:10600000487962726964205468726573686F6C6461
:106010003A0A00205430204500205A002059002020
:106020005800537465707065722064726976657289
:106030002063757272656E743A0A0020440020492C
:106040000020204D333034205000204400204900EF
:1060500020204D3330312050005049442073657466
:1060600074696E67733A0A00204500205A0020596F
:106070000020580020540020530020204D3230359D
:1060800020420020453C6D61785F655F6A65726BF8
:106090003E0020583C6D61785F785F6A65726B3EA8
:1060A00020593C6D61785F795F6A65726B3E205A5A
:1060B0003C6D61785F7A5F6A65726B3E0041647621
:1060C000616E6365643A20423C6D696E5F7365671B
:1060D0006D656E745F74696D655F75733E20533CCA
:1060E0006D696E5F66656564726174653E20543CDF
:1060F0006D696E5F74726176656C5F66656564720A
:106100006174653E0020540020520020204D323042
:1061100034205000416363656C65726174696F6E11
:106120002028756E6974732F7332293A20503C70A1
:1061300072696E745F616363656C3E20523C726588
:1061400074726163745F616363656C3E20543C7478
:10615000726176656C5F616363656C3E0A00204521
:1061600000205A0020590020204D323031205800A4
:106170004D6178696D756D20416363656C65726111
:1061800074696F6E2028756E6974732F7332293AA3
:106190000A00204500205A0020590020204D3230AE
:1061A000332058004D6178696D756D2066656564B2
:1061B00072617465732028756E6974732F73293A40
:1061C0000A0053746570732070657220756E69746F
:1061D0003A0A002020473231202020203B20556EF3
:1061E00069747320696E206D6D0020204D3536393D
:1061F0002053310048617264636F646564204465B4
:106200006661756C742053657474696E6773204C95
:106210006F616465640A002823000028230000C819
:10622000000000E8030000000096430000964300D1
:10623000009643000020420000C8420000C842000F
:1062400000484333A31346454550524F4D20496EF5
:10625000697469616C697A65640A00290A002062C0
:10626000797465733B2063726320002073746F72CE
:1062700065642073657474696E67732072657472E7
:106280006965766564202800202863616C63756CFD
:106290006174656429210A0020213D200045455094
:1062A000524F4D20435243206D69736D6174636892
:1062B000202D202873746F72656429200020536993
:1062C0007A653A2000496E6465783A2000204D6175
:1062D000726C696E3D563639290A00454550524F59
:1062E0004D2076657273696F6E206D69736D617490
:1062F00063682028454550524F4D3D004E6F204564
:106300004550524F4D2E0A00290A002062797465CB
:10631000733B20637263200053657474696E677306
:106320002053746F7265642028004E6F20454550DD
:10633000524F4D2E0A00454550524F4D2064617416
:106340006173697A65206572726F722E0A005761F7
:10635000726E696E673A20486F6D696E672042758C
:106360006D702044697669736F72203C20310A0099
:1063700002020420746F6F206C6F6E672065787462
:10638000727573696F6E2070726576656E74656480
:106390000A0020636F6C6420657874727573696F8E
:1063A0006E2070726576656E7465640A0020453AE9
:1063B00000205A3A0020593A00583A00000048425A
:1063C0000000484200002042FF01010000000000E0
:1063D0000000000000004000003043000045430082
:1063E000003743000040C000004043000037432016
:1063F000746F6F206C6F6E67206578747275736947
:106400006F6E2070726576656E7465640A00206335
:106410006F6C6420657874727573696F6E2070722A
:106420006576656E7465640A00627573793A2070EA
:10643000617573656420666F7220696E7075740A89
:1064400000627573793A2070617573656420666FB8
:106450007220757365720A00627573793A207072E2
:106460006F63657373696E670A0020496E76616CAD
:10647000696420657874727564657220004D302FF0
:106480003120427265616B2043616C6C656400224F
:106490000A00556E6B6E6F776E20636F6D6D616E67
:1064A000643A202200454550524F4D204F4B0A0080
:1064B0004E6F204D6F76652E004543484F00494E84
:1064C000464F004552524F52530044525952554E76
:1064D00000434F4D4D554E49434154494F4E006F77
:1064E000666600B964BE64C364CA64D1644445424C
:1064F00055473A005072696E742074696D653A2090
:10650000004D3131332053002F2F20004361703A6A
:10651000004348414D4245525F54454D504552411C
:1065200054555245004D4F54494F4E5F4D4F4445D1
:106530005300544845524D414C5F50524F544543CF
:1065400054494F4E004155544F5245504F52545F9D
:1065500053445F5354415455530050524F4D50547F
:106560005F535550504F525400454D455247454E8C
:1065700043595F50415253455200434153455F4C8C
:10658000494748545F4252494748544E4553530087
:10659000544F47474C455F4C494748545300534F6D
:1065A0004654574152455F504F5745520042554956
:1065B0004C445F50455243454E54004C4556454C63
:1065C000494E475F44415441005A5F50524F424543
:1065D000004155544F4C4556454C005052494E547D
:1065E0005F4A4F420050524F475245535300415566
:1065F000544F5245504F52545F54454D5000564FE2
:106600004C554D455452494300454550524F4D005D
:1066100042494E4152595F46494C455F5452414EA2
:10662000534645520053455249414C5F584F4E5FC7
:10663000584F4646004649524D574152455F4E41DC
:106640004D453A4D61726C696E20322E302E302EDF
:1066500031373220284769746875622920534F55B5
:106660005243455F434F44455F55524C3A687474FA
:1066700070733A2F2F636F64652E616C6570686F5D
:10668000626A656374732E636F6D2F6469666675E5
:1066900073696F6E2F4D41524C494E2050524F54EA
:1066A0004F434F4C5F56455253494F4E3A312E306F
:1066B000204D414348494E455F545950453A4C7529
:1066C0006C7A426F742042696F2045585452554489
:1066D00045525F434F554E543A3120555549443A3F
:1066E00039613164386565652D373131382D343085
:1066F00061372D393432642D3935343166333536CE
:10670000363764640A0020284E6F7420796574203F
:106710006D6561737572656429002020417665722C
:10672000616765206D656173757265642062616380
:106730006B6C61736820286D6D293A002020536DC1
:106740006F6F7468696E6720286D6D293A2020206C
:106750002020202020202020202020202020530026
:1067600020204261636B6C617368204469737461BB
:106770006E636520286D6D293A202020202020207E
:106780002000202846312E30203D2066756C6C2C70
:106790002046302E30203D206E6F6E65290A002085
:1067A00020436F7272656374696F6E20416D6F75FF
:1067B0006E742F466164652D6F75743A2020202019
:1067C0002046006163746976653A0A00696E00428A
:1067D00061636B6C61736820436F72726563746987
:1067E0006F6E200043757272656E742066696C6509
:1067F0003A2000456E642066696C65206C6973748C
:106800000A00426567696E2066696C65206C697371
:10681000740A00416476616E6365204B3D003F4B16
:106820002076616C7565206F7574206F66207261CB
:106830006E67652028302D3130292E0A0073707262
:106840006561644379636C6500737465616C746839
:1068500043686F700020647269766572206D6F64A2
:10686000653A09007370726561644379636C650011
:10687000737465616C746843686F7000206472693A
:10688000766572206D6F64653A0900737072656198
:10689000644379636C6500737465616C7468436804
:1068A0006F700020647269766572206D6F64653A5E
:1068B00009007370726561644379636C6500737479
:1068C00065616C746843686F7000206472697665F6
:1068D00072206D6F64653A090020686F6D696E679C
:1068E0002073656E73697469766974793A20002043
:1068F000686F6D696E672073656E73697469766918
:1069000074793A200020737465616C746843686F11
:1069100070206D61782073706565643A2000207383
:106920007465616C746843686F70206D6178207362
:10693000706565643A200020737465616C74684307
:10694000686F70206D61782073706565643A20000F
:1069500020737465616C746843686F70206D617832
:106960002073706565643A200020707265776172EB
:106970006E20666C616720636C65617265640A00F5
:10698000207072657761726E20666C616720636C3F
:1069900065617265640A00207072657761726E20AD
:1069A000666C616720636C65617265640A002070C3
:1069B00072657761726E20666C616720636C6561D9
:1069C0007265640A002074656D7065726174757219
:1069D00065207072657761726E2074726967676591
:1069E0007265643A20002074656D7065726174751B
:1069F0007265207072657761726E20747269676764
:106A0000657265643A20002074656D70657261740A
:106A1000757265207072657761726E207472696735
:106A200067657265643A20002074656D70657261F7
:106A300074757265207072657761726E2074726908
:106A40006767657265643A200020647269766572D2
:106A50002063757272656E743A20002064726976E4
:106A600065722063757272656E743A2000206472DC
:106A7000697665722063757272656E743A200020C3
:106A80006472697665722063757272656E743A20FD
:106A9000004D6163726F20746F6F206C6F6E672E94
:106AA0000A0020466C6F773A200020643A00206983
:106AB0003A0020703A00204500205A00205900205A
:106AC0004D393220580043290A0061626C65642008
:106AD000286D696E2074656D7020006469730065AF
:106AE0006E00436F6C642065787472756465732002
:106AF0006172652000205400205200416363656C80
:106B000065726174696F6E3A205000496E76616CEF
:106B100069642065787472756465720A0020643A4D
:106B20000020693A0020703A00536C6565702E2E83
:106B30002E0047322F4733206261642070617261FA
:106B40006D65746572730A00446F6E6520736176BB
:106B5000696E672066696C652E0A00534420726571
:106B60006164206572726F720A00446F6E652070F6
:106B700072696E74696E672066696C650A004D32D1
:106B8000390053544F505045442E20005072696EC6
:106B90007465722073746F7070656420647565200D
:106BA000746F206572726F72732E2046697820743C
:106BB0006865206572726F7220616E6420757365FE
:106BC000204D39393920746F207265737461727485
:106BD0002E202854656D7065726174757265206928
:106BE000732072657365742E205365742069742058
:106BF00061667465722072657374617274696E6720
:106C0000290A004E6F20436865636B73756D2077AA
:106C1000697468206C696E65206E756D6265722C92
:106C2000204C617374204C696E653A20004E6F20D1
:106C3000436865636B73756D2077697468206C6950
:106C40006E65206E756D6265722C204C61737420C8
:106C50004C696E653A2000636865636B73756D20DF
:106C60006D69736D617463682C204C617374204C82
:106C7000696E653A20004C696E65204E756D6265DF
:106C800072206973206E6F74204C617374204C699C
:106C90006E65204E756D6265722B312C204C6173D0
:106CA00074204C696E653A20004D313130005265D8
:106CB00073656E643A20002042002050006F6B0024
:106CC000220A00656E7175657565696E6720220020
:106CD000504944204175746F74756E652066616912
:106CE0006C65642120426164206578747275646506
:106CF00072206E756D6265720A0042656420436F92
:106D00006F6C696E672E2E2E0042656420486561A7
:106D100074696E672E2E2E006F6B0030780047323C
:106D200038205A0A4D313137205072696E74206113
:106D3000626F727465642E004D3137205A00202036
:106D4000506C616E6E6572427566666572427974EA
:106D500065733A20002046726565204D656D6F723F
:106D6000793A2000436F6D70696C65643A204F6317
:106D70007420203820323031390A00207C204175BF
:106D800074686F723A2028416C657068204F626A9F
:106D90006563747320496E632E2C204C756C7A42A7
:106DA0006F7420476974205265706F7369746F72D5
:106DB00079290A004F63742020382032303139316C
:106DC000363A30333A343000204C617374205570B9
:106DD00064617465643A2000322E302E302E3137D3
:106DE000320A004D61726C696E0020536F667477D1
:106DF0006172652052657365740A0020576174637F
:106E000068646F672052657365740A002042726F70
:106E1000776E206F75742052657365740A00204583
:106E2000787465726E616C2052657365740A0050E7
:106E30006F77657255700A0073746172740A004B43
:106E4000494C4C45442E20005072696E7465722086
:106E500068616C7465642E206B696C6C28292063F2
:106E6000616C6C6564210A004B494C4C2063617570
:106E7000736564206279204B494C4C2062757474B0
:106E80006F6E2F70696E0A004B494C4C2063617520
:106E900073656420627920746F6F206D756368205C
:106EA000696E6163746976652074696D65202D2053
:106EB00063757272656E7420636F6D6D616E643A96
:106EC000200050726F7465637465642050696E0AA7
:106ED0000025311D40512924301C4527232F1B0A32
:106EE0000743222B1A42043803FF3604060600012A
:106EF000D7524C5BB15D1D667F68B669186EB8737A
:106F00004C7A867C8A7E53806781A282A685DC8744
:106F10001888FD8A958C7A8EB68E898FB491F192FD
:106F200064938395C096EF989399EB9AAD9BB8A024
:106F3000E8A09AA12BA2C2A4EEA59DA60CB583B58C
:106F4000CCB507B6A2B6DBB618B819B95CBAC4C1DD
:106F5000E8C27DC3DBCA42D1F9D884D96CEE2703DD
:106F6000350389033903A302AB03A9028CEE112474
:106F70001FBECFEFD1E2DEBFCDBF00E00CBF17E0F8
:106F8000A0E0B2E0EAE5FEE403E00BBF02C0079038
:106F90000D92A833B107D9F72CE1A8E3B7E001C0FF
:106FA0001D92A637B207E1F717E3C6EBD7E300E07F
:106FB00006C021970109802FFE010F94539CC8370A
:106FC000D10780E00807A9F70E94F5440D941BA79C
:106FD0000C9400001F920F920FB60F9211242F9362
:106FE0003F938F939F93AF93BF9380913907909175
:106FF0003A07A0913B07B0913C073091380723E056
:10700000230F2D3720F40196A11DB11D05C026E8E0
:10701000230F0296A11DB11D2093380780933907D5
:1070200090933A07A0933B07B0933C0780913D07AC
:1070300090913E07A0913F07B09140070196A11D96
:10704000B11D80933D0790933E07A0933F07B093F7
:107050004007BF91AF919F918F913F912F910F90DA
:107060000FBE0F901F9018952FB7F89460913907B5
:1070700070913A0780913B0790913C072FBF08958C
:107080003FB7F89480913D0790913E07A0913F074C
:10709000B091400726B5A89B05C02F3F19F0019677
:1070A000A11DB11D3FBFBA2FA92F982F8827820F8E
:1070B000911DA11DB11DBC01CD0142E0660F771FDE
:1070C000881F991F4A95D1F708958F929F92AF928A
:1070D000BF92CF92DF92EF92FF926B017C01D0DFE3
:1070E0004B015C01C114D104E104F104F1F09CD323
:1070F000C7DFDC01CB0188199909AA09BB09883EC1
:107100009340A105B10570F321E0C21AD108E1084E
:10711000F10888EE880E83E0981EA11CB11CC114F2
:10712000D104E104F10421F7DDCFFF90EF90DF906F
:10713000CF90BF90AF909F908F900895823091052F
:1071400038F0880F991F880F991F05970197F1F75D
:107150000895789484B5826084BD84B5816084BDCF
:1071600085B5826085BD85B5816085BDEEE6F0E0C0
:10717000808181608083E1E8F0E01082808182601C
:107180008083808181608083E0E8F0E0808181609D
:107190008083E1EBF0E0808184608083E0EBF0E0CD
:1071A000808181608083E1E9F0E08081826080837A
:1071B000808181608083E0E9F0E08081816080836C
:1071C000E1EAF0E080818260808380818160808359
:1071D000E0EAF0E0808181608083E1E2F1E080819B
:1071E00082608083808181608083E0E2F1E0808141
:1071F00081608083EAE7F0E0808184608083808121
:1072000082608083808181608083808180688083C8
:107210001092C10008951F93CF93DF93182FEB01B5
:1072200061E016D1209711F460E004C0CF3FD10592
:1072300031F461E0812FDF91CF911F9145C1E12FA2
:10724000F0E0E15FF64FE4914E2F50E0FA01319704
:10725000E231F10508F09DC08827EE58FF4F8F4FAF
:107260000D94539C84B5806884BDC7BD97C084B518
:10727000806284BDC8BD92C0809180008068809388
:107280008000D0938900C093880088C080918000DE
:10729000806280938000D0938B00C0938A007EC070
:1072A00080918000886080938000D0938D00C0938F
:1072B0008C0074C08091B00080688093B000C0934F
:1072C000B3006CC08091B00080628093B000C09326
:1072D000B40064C080919000806880939000D09347
:1072E0009900C09398005AC080919000806280936A
:1072F0009000D0939B00C0939A0050C08091900062
:10730000886080939000D0939D00C0939C0046C0FD
:107310008091A00080688093A0008091A0008F7B66
:107320008093A000D093A900C093A80037C080919B
:10733000A00080628093A000D093AB00C093AA000D
:107340002DC08091A00088608093A000D093AD00F4
:10735000C093AC0023C080912001806880932001FD
:10736000D0932901C093280119C080912001806227
:1073700080932001D0932B01C0932A010FC08091EC
:107380002001886080932001D0932D01C0932C01AF
:1073900005C0C038D1050CF04CCF46CFDF91CF915E
:1073A0001F91089590E0FC013197E231F10508F05A
:1073B0004EC08827EC57FF4F8F4F0D94539C809100
:1073C00080008F7703C0809180008F7D8093800044
:1073D000089580918000877FF9CF84B58F7702C0B0
:1073E00084B58F7D84BD08958091B0008F7703C0F0
:1073F0008091B0008F7D8093B000089580919000BF
:107400008F7707C0809190008F7D03C0809190009E
:10741000877F8093900008958091A0008F7707C0A8
:107420008091A0008F7D03C08091A000877F809312
:10743000A0000895809120018F7707C080912001DE
:107440008F7D03C080912001877F80932001089564
:10745000CF93DF9390E0FC01EB5AF64F2491FC01AF
:10746000E556F64F8491882361F190E0880F991FCB
:10747000FC01EB5EF54FC591D491FC01E550F64F50
:10748000A591B491611109C09FB7F89488812095A6
:1074900082238883EC912E230BC0623061F49FB766
:1074A000F8943881822F809583238883EC912E2B4A
:1074B0002C939FBF06C08FB7F894E8812E2B2883AA
:1074C0008FBFDF91CF9108951F93CF93DF93282F24
:1074D00030E0F901E15FF64F8491F901EB5AF64F84
:1074E000D491F901E556F64FC491CC23C1F0162F83
:1074F000811158DFEC2FF0E0EE0FFF1FE550F64F43
:10750000A591B4918FB7F894111105C09C91ED2FFE
:10751000E095E92302C0EC91ED2BEC938FBFDF9156
:10752000CF911F910895CF93DF93282F30E0F90179
:10753000E15FF64F8491F901EB5AF64FD491F901CE
:10754000E556F64FC491CC2389F081112BDFEC2F47
:10755000F0E0EE0FFF1FEF51F64FA591B491EC91C3
:10756000ED2381E090E021F480E002C080E090E033
:10757000DF91CF91089508951F920F920FB60F9249
:1075800011240BB60F922F933F934F935F936F93FA
:107590007F938F939F93AF93BF93EF93FF93E0916C
:1075A0000802F09109021995FF91EF91BF91AF91F7
:1075B0009F918F917F916F915F914F913F912F910B
:1075C0000F900BBE0F900FBE0F901F9018951F923B
:1075D0000F920FB60F9211240BB60F922F933F9379
:1075E0004F935F936F937F938F939F93AF93BF93CB
:1075F000EF93FF93E0910A02F0910B021995FF912E
:10760000EF91BF91AF919F918F917F916F915F911A
:107610004F913F912F910F900BBE0F900FBE0F9087
:107620001F9018951F920F920FB60F9211240BB650
:107630000F922F933F934F935F936F937F938F930B
:107640009F93AF93BF93EF93FF93E0910C02F09160
:107650000D021995FF91EF91BF91AF919F918F917D
:107660007F916F915F914F913F912F910F900BBE42
:107670000F900FBE0F901F9018951F920F920FB68C
:107680000F9211240BB60F922F933F934F935F935A
:107690006F937F938F939F93AF93BF93EF93FF93DA
:1076A000E0910E02F0910F021995FF91EF91BF91B9
:1076B000AF919F918F917F916F915F914F913F918A
:1076C0002F910F900BBE0F900FBE0F901F9018952B
:1076D0001F920F920FB60F9211240BB60F922F9399
:1076E0003F934F935F936F937F938F939F93AF934A
:1076F000BF93EF93FF93E0910402F0910502199577
:10770000FF91EF91BF91AF919F918F917F916F9179
:107710005F914F913F912F910F900BBE0F900FBE35
:107720000F901F9018951F920F920FB60F92112471
:107730000BB60F922F933F934F935F936F937F936B
:107740008F939F93AF93BF93EF93FF93E0910602C4
:10775000F09107021995FF91EF91BF91AF919F9121
:107760008F917F916F915F914F913F912F910F90EA
:107770000BBE0F900FBE0F901F9018951F920F9287
:107780000FB60F9211240BB60F922F933F934F9386
:107790005F936F937F938F939F93AF93BF93EF9379
:1077A000FF93E0911002F09111021995FF91EF9172
:1077B000BF91AF919F918F917F916F915F914F9109
:1077C0003F912F910F900BBE0F900FBE0F901F9007
:1077D00018951F920F920FB60F9211240BB60F92AD
:1077E0002F933F934F935F936F937F938F939F93C9
:1077F000AF93BF93EF93FF93E0911202F0911302C6
:107800001995FF91EF91BF91AF919F918F917F91CA
:107810006F915F914F913F912F910F900BBE0F9001
:107820000FBE0F901F9018950895CF93DF9300D04F
:107830001F92CDB7DEB7611571058105910579F00D
:107840009B01AC0169833A834B835C830F94E39C77
:1078500029813A814B815C810F94379C03C060E0A1
:1078600070E0CB010F900F900F900F90DF91CF91B0
:1078700008954F925F926F927F92AF92BF92CF9294
:10788000DF92EF92FF920F931F93CF93DF93CDB7C9
:10789000DEB729013A019B01AC01241935094609DB
:1078A00057098A899B89AC89BD89BC01CD016A19B8
:1078B0007B098C099D090F94DF9BA801970124196E
:1078C0003509460957090F94379CCA01B9016A0D59
:1078D0007B1D8C1D9D1DDF91CF911F910F91FF90FE
:1078E000EF90DF90CF90BF90AF907F906F905F90C0
:1078F0004F900895CF93CFB7F894809144078111AA
:1079000023C0E0EDF9E08491EAE8F9E09491E82FF2
:10791000F0E0EE0FFF1FEB5EF54FA591B491EC91F7
:10792000E92319F461E085E3CFDD61E085E390DDD3
:107930008CB580618CBD8CB580648CBD61E084E3C6
:1079400087DD61E083E384DD809144078F5F80936E
:107950004407CFBFCF910895CF92DF92EF92FF926D
:10796000CF93DF93EC0170E06F5F7F4F072E000C29
:10797000880B990B0F94389920E030E040E05DE3EC
:107980000F94199B6B017C01E881F9810680F781D6
:10799000E02DCE011995811105C026E636E646EAAE
:1079A0005EE304C02CEE31E548E35EE3C701B601B7
:1079B0000F94199B6B017C012AE037ED43EA5CE3ED
:1079C00069857A858B859C850F94BD979B01AC0159
:1079D000C701B6010F949D9825ED34E045EB5FE3B8
:1079E0000F949D9820E030E04AE754E40F94199BEF
:1079F0000F940A99CB01DF91CF91FF90EF90DF9028
:107A0000CF900895CF92DF92EF92FF921F93CF9382
:107A1000DF93EC0180E090E00F94369925ED34E09F
:107A200045E352E40F94199B20E030E04AE754E428
:107A30000F949D986B017C012AE037ED43EA5CE3EB
:107A400069857A858B859C850F94BD979B01AC01D8
:107A5000C701B6010F94199B26E636E646EA5EE3B7
:107A60000F949D9820E030E040E85FE30F94BC97CE
:107A70000F940A99162FE881F9810480F581E02D91
:107A8000603118F561E0CE0119952AE037ED43EA3F
:107A90005CE369857A858B859C850F94BD979B01F6
:107AA000AC01C701B6010F94199B2CEE31E548E3F8
:107AB0005EE30F949D9820E030E040E85FE30F9490
:107AC000BC970F940A99162F03C060E0CE01199558
:107AD000612FCE0177D2612F70E080E090E00F94AB
:107AE00038992D853E854F8558890F94199B0F94A1
:107AF0000A99CE01DF91CF911F91FF90EF90DF9017
:107B0000CF9043C2FC01258736874787508B7ACFB9
:107B1000CF93DF93EC0193D2682FCE01DF91CF9109
:107B20001BCFDC01ED91FC910084F185E02D1995CE
:107B3000611571058105910539F06F3F7F4F8F4FBA
:107B40009F4F21F080E0089582E0089581E008953C
:107B5000DC01ED91FC910484F585E02D19958350AD
:107B60000895DC01ED91FC910088F189E02D1995D3
:107B70008F5F08956031710509F441C088F4623067
:107B8000710509F454C020F4672B09F458C0089516
:107B90006430710509F443C068307105C1F108957E
:107BA00060347105E1F020F46032710501F108954F
:107BB0006038710561F06115714009F048C0DC0161
:107BC000ED91FC910288F389E02D60E03FC0DC017B
:107BD000ED91FC910288F389E02D61E037C0DC0172
:107BE000ED91FC910288F389E02D62E02FC0DC0169
:107BF000ED91FC910288F389E02D63E027C0DC0160
:107C0000ED91FC910288F389E02D64E01FC0DC0156
:107C1000ED91FC910288F389E02D65E017C0DC014D
:107C2000ED91FC910288F389E02D66E00FC0DC0144
:107C3000ED91FC910288F389E02D67E007C0DC013B
:107C4000ED91FC910288F389E02D68E01994089584
:107C5000DC01ED91FC910488F589E02D19958930BE
:107C600048F4E82FF0E0EE0FFF1FE25FFC4F808149
:107C70009181089580E090E00895DC01ED91FC9100
:107C8000008CF18DE02D1995843030F4E82FF0E070
:107C9000E65FFC4F8081089580E00895DC01ED915E
:107CA000FC910280F381E02D61E01995862F089503
:107CB000FC0185810895DC0115966C931597ED9173
:107CC000FC91262F30E040E050E00190F081E02D63
:107CD00061E11994DC01ED91FC910280F381E02DCA
:107CE00062E11994FC01268137818085482F4F700D
:107CF000842FB90190E00895DC019A01462F4F705E
:107D000016962C93169717963C931797942F9F705F
:107D100018968C911897807F892B18968C931897BA
:107D2000ED91FC91119750E00190F081E02D63E11D
:107D3000CD011994FC0166A177A191A580A5917050
:107D40000895DC0196964C93969797965C93979737
:107D500098966C93989799968C91999770FB80F967
:107D600099968C939997ED91FC9111979A01AB019B
:107D700051700190F081E02D6DE6CD011994DC0188
:107D80006F7096962C919697207F262B96962C9323
:107D90009697ED91FC91119797963C9197979896AD
:107DA0004C91989799965C9151700190F081E02DDB
:107DB0006DE61994DC016F7097963C919797307F30
:107DC000362B97963C939797ED91FC911197969649
:107DD0002C91969798964C91989799965C915170A2
:107DE0000190F081E02D6DE61994DC016F77989693
:107DF0004C9198974078462B98964C939897ED9194
:107E0000FC91119796962C91969797963C919797FF
:107E100099965C9151700190F081E02D6DE6199476
:107E2000FC0190A5990F9595292F092E000C330B75
:107E300020743327220F331F892F8F77822B0895C9
:107E4000DC01ED91FC910280F381E02D6FE6199445
:107E5000DC01ED91FC910084F185E02D1995CB01B9
:107E600093700895DC01ED91FC910084F185E02D83
:107E7000199577FB882780F90895DC01ED91FC9135
:107E80000084F185E02D19958F710895DC01ED9145
:107E9000FC910084F185E02D1995892F817008955A
:107EA000DC01ED91FC910084F185E02D199591FBA9
:107EB000882780F90895DC01ED91FC910084F1851B
:107EC000E02D199592FB882780F90895DC01ED914A
:107ED000FC910084F185E02D199593FB882780F9AA
:107EE0000895DC01ED91FC910084F185E02D199558
:107EF00094FB882780F90895DC01ED91FC910084C2
:107F0000F185E02D199595FB882780F90895DC010E
:107F1000ED91FC910084F185E02D199596FB882761
:107F200080F90895DC01ED91FC910084F185E02D4C
:107F3000199597FB882780F90895FC0122813381E8
:107F40008481482F4F70842FB90190E00895DC019F
:107F50009A01462F4F7012962C93129713963C93CA
:107F60001397942F9F7014968C911497807F892B70
:107F700014968C931497ED91FC91119750E0019019
:107F8000F081E02D60E1CD011994DC016F71129652
:107F90008C911297807E682B12966C931297ED91BC
:107FA000FC911197262F13963C91139714968C9160
:107FB0001497482F4F7050E00190F081E02D60E160
:107FC000CD011994DC016F7113968C911397807E0B
:107FD000682B13966C931397ED91FC911197129661
:107FE0002C911297362F14968C911497482F4F701E
:107FF00050E00190F081E02D60E1CD011994DC01A9
:108000006F7014968C911497807F682B14966C93E4
:108010001497ED91FC91119712962C91129713964B
:108020003C911397462F4F7050E00190F081E02D66
:1080300060E1CD011994FC0182818F710895FC01EA
:1080400083818F710895DC016770962F9295907FE0
:1080500092966C9192976F78692B92966C93929707
:10806000ED91FC91119792962D913D914D915C91DE
:1080700095970190F081E02D6CE6CD011994DC011B
:1080800092968C91929760FB87F992968C93929737
:108090006695677093968C919397887F682B9396DB
:1080A0006C939397ED91FC91119792962D913D9140
:1080B0004D915C9195970190F081E02D6CE6CD019A
:1080C0001994DC0193968C91939760FB87F99396B2
:1080D0008C93939761FB882780F994966C91949781
:1080E0006E7F682B94966C939497ED91FC91119709
:1080F00092962D913D914D915C9195970190F081D3
:10810000E02D6CE6CD011994DC0194962C919497A6
:1081100060FB21F994962C939497ED91FC91119723
:1081200092962D913D914D915C9195970190F081A2
:10813000E02D6CE619946F70DC0195962C91959763
:10814000207F622B95966C939597ED91FC911197FA
:1081500092962D913D914D915C9195970190F08172
:10816000E02D6CE61994CF93DF93EC01E881F9815F
:108170000280F381E02D6CE619956AA37BA38CA3A2
:108180009DA3DF91CF910895CF93DF93EC01EBDFB7
:108190008AA182958770DF91CF910895CF93DF9365
:1081A000EC01E1DF9AA1991F9927991F8BA1877094
:1081B000880F892BDF91CF910895CF93DF93EC0146
:1081C000D2DF9BA1991F9927991F8CA18170880FDD
:1081D000892BDF91CF910895CF93DF93EC01C3DF1B
:1081E0008CA186958170DF91CF910895CF93DF9315
:1081F000EC01B9DF8DA18F70DF91CF910895DC0183
:1082000092964D935D936D937C939597ED91FC9130
:108210000190F081E02D9A01AB016CE619946F702A
:10822000DC0192962C919297207F622B92966C9310
:108230009297ED91FC91119792962D913D914D91D0
:108240005C9195970190F081E02D6CE61994CF93A5
:10825000DF93EC0188DF8AA18F70DF91CF910895C1
:10826000CF92DF92EF92CF93DF93EC01E881F98117
:108270000280F381E02D60E019956B01E82E23E088
:10828000E222CA8ADB8A2E2D23709C899C7F922B46
:108290009C8B8E2DB60190E0DF91CF91EF90DF9017
:1082A000CF900895DC019A01462F437052962C938B
:1082B000529753963C935397942F937054968C9166
:1082C00054978C7F892B54968C935497ED91FC9105
:1082D000119750E00190F081E02D60E0CD011994FC
:1082E000DC0152968C91529760FB82F952968C93E6
:1082F0005297ED91FC911197282F53963C915397EB
:1083000054968C915497482F437050E00190F0811F
:10831000E02D60E0CD011994DC0152968C915297CA
:1083200060FB84F952968C935297ED91FC911197D2
:10833000282F53963C91539754968C915497482FDD
:10834000437050E00190F081E02D60E0CD01199480
:10835000DC0153968C91539760FB80F953968C9374
:108360005397ED91FC91119752962C915297382F7B
:1083700054968C915497482F437050E00190F081AF
:10838000E02D60E0CD011994CF93DF93EC0168DF1D
:108390008A8982FB882780F9DF91CF910895FC01BB
:1083A00025A536A587A5482F4F73842FB90190E0E6
:1083B0000895DC019A01462F4F739D962C939D974B
:1083C0009E963C939E97942F9F739F968C919F9718
:1083D000807C892B9F968C939F97ED91FC911197B0
:1083E00050E00190F081E02D60E7CD011994CF932A
:1083F000DF93EC0161E088812BD861E08C8128D883
:1084000062E08A8125D861E08C81DF91CF915CC8E0
:10841000BF92CF92DF92EF92FF920F931F93CF9371
:10842000DF93EC01E62E60E08C814ED807E010E08F
:10843000F12CCE2CD12CB02EC601002E02C0959569
:1084400087950A94E2F780FF02C061E001C060E016
:1084500088813AD861E08C8137D88A8164D821E05C
:1084600030E0892B11F420E030E001C0220FBA94F3
:10847000EAF7F22A60E08C8127D801501109D9F679
:10848000E0FE02C061E001C060E088811DD861E0CB
:108490008C811AD88A8147D821E0892B09F420E001
:1084A0008F2D822BDF91CF911F910F91FF90EF9035
:1084B000DF90CF90BF9008950F931F93CF93DF93DA
:1084C0008C01D62F672FA4DFC82F6D2FC801A0DF26
:1084D0002C2F30E0322F2227A901482BCA01DF912F
:1084E000CF911F910F9108950F93FC0130E080E030
:1084F00092E1AAE7B0E0481759076A077B0740F402
:10850000B695A795979587953F5F3630A1F737E0E9
:1085100091E09327222311F020E501C020E7892F65
:1085200086950C70082B022B0083917091830F911C
:10853000089520914307222399F04FB7F894209192
:108540004307213059F42DB3209341073DB32091C7
:108550004207209523232DBB4FBF02C04093410704
:108560008CBD9DBD08958EBD00000DB407FEFDCFEE
:108570008EB508950CB405FC0DC09EBD00000DB471
:1085800007FEFDCF9EB58EBD00000DB407FEFDCFEA
:108590008EB508958EBD00000DB407FEFDCF8EB5DB
:1085A0009EBD00000DB407FEFDCF9EB508958091DD
:1085B0004307882361F09FB7F89420914307809187
:1085C0004107213019F48DBB9FBF08958FBF0895D7
:1085D000FC01128213828481807F8483158216823B
:1085E00017828085807F80872187328743875487E1
:1085F00080E090E0A0E0BFE385879687A787B08BF7
:1086000084E293E091838083128A138A84898C7F29
:10861000848B158A168A8789807F878B108E118EAE
:10862000828D807F828F138E148E158E868D8E7F25
:10863000868F178E10A281A1807881A312A213A227
:1086400014A215A216A217A210A681A58E7F81A73B
:1086500012A613A614A680A98C7F80AB72AB61AB67
:1086600014AA13AA80E885A784E086A787A5807C42
:10867000856087A70895FC0181A90C94643AAF92A4
:10868000BF92CF92DF92EF92FF920F93CF93DF933F
:108690001F921F92CDB7DEB75C01F62EFC0183A9B5
:1086A00094A9892B09F448C060E0C501E4DF6F2D6F
:1086B000F50183A994A9ACDE60E070E0F50183A91F
:1086C00094A9FADE60E070E0F50183A994A9F4DED4
:1086D00061E0C501D0DF60E0C501CDDF6F2DF501A0
:1086E00083A994A995DEF501818B60E083A994A903
:1086F0008FDEC82ED12CE12CF12CFE2CED2CDC2CA5
:10870000CC2460E0F50183A994A982DEC82AFE2C5E
:10871000ED2CDC2CCC2460E0F50183A994A978DE53
:10872000C82AFE2CED2CDC2CCC2460E0F50183A9BA
:1087300094A96EDEC82A41C04091140250911502DE
:1087400060911602709117020CE021E0CE010196B3
:10875000CBDE89819A81EDDE60E0C5018CDF8F2D53
:1087600002DF80E090E006DF80E090E003DF61E080
:10877000C50181DF60E0C5017EDF8F2DF4DEF501EC
:10878000818B80E0F0DEC82ED12CE12CF12CFE2C68
:10879000ED2CDC2CCC2480E0E6DEC82AFE2CED2C6F
:1087A000DC2CCC2480E0DFDEC82AFE2CED2CDC2C77
:1087B000CC2480E0D8DEC82AFADE61E0C5015BDFA8
:1087C000C701B6010F900F90DF91CF910F91FF90ED
:1087D000EF90DF90CF90BF90AF9008954F925F924F
:1087E0006F927F928F929F92AF92BF92EF92FF9281
:1087F0000F931F93CF93DF931F921F92CDB7DEB7D6
:108800007C0149015A01162F1068FC0183A994A923
:10881000250166247724892BA1F060E0C7012BDFB6
:10882000612FF70183A994A9F3DDF701818BB201D0
:1088300083A994A941DEB401F70183A994A93CDE80
:108840001CC0409114025091150260911602709163
:1088500017020CE021E0CE01019646DE89819A8163
:1088600068DE60E0C70107DF812F7DDEF701818BC5
:10887000C20180DEC4017EDE9ADE61E0C701FBDE5C
:108880000F900F90DF91CF911F910F91FF90EF907C
:10889000BF90AF909F908F907F906F905F904F9020
:1088A0000895CF93DF93EC0161E089A90E94283AF3
:1088B00061E0CE01E0DE8BA99CA9009709F097DD6D
:1088C0008A899B892C89A22FA370AC016A2F70E042
:1088D000CE01E8DC4AA15BA16CA17DA1CE018FDCB9
:1088E0004EA15FA168A579A57170CE012ADA8DA588
:1088F0009EA52FA5A22FAF73AC016A2F70E0CE0109
:1089000058DD8A819B812C81A22FAF70AC016A2F28
:1089100070E0CE011CDB68E0CE0181DCE881F981EA
:108920000688F789E02D61E0CE01DF91CF9119949F
:10893000DC01ED91FC910280F381E02D64E019945B
:10894000F7DF64FB882780F90895CF93DF93EC016C
:10895000F7DF811105C0CE017ADC91E0811101C001
:1089600090E0892FDF91CF910895FC012589368908
:108970008789482F4F70842FB90190E00895DC015A
:108980009A01462F4F7055962C93559756963C93C7
:108990005697942F9F7057968C915797807F892B6D
:1089A00057968C935797ED91FC91119750E0019059
:1089B000F081E02D64E1CD011994FC01208D318D11
:1089C000828D482F4F70842FB90190E00895DC010B
:1089D000ED91FC910280F381E02D61E71995862FDE
:1089E000089580E090E0089508950E94A938FCDF82
:1089F0000F94FF96C0E0D0E00F949E972097E1F38C
:108A00000E940000F9CF80E00C94A14E1F93CF93F9
:108A1000DF931F921F92CDB7DEB7182F862F798371
:108A20009A830E94C04E7981872F0E94C04E812F69
:108A30000E94C04E9A81892F0F900F90DF91CF91A5
:108A40001F910C94C04ECF93DF93DC01FB0180E0BB
:108A500090E0219141505109222381F041155105A7
:108A600069F027FD06C0ED01C20FD11D288130E05D
:108A700002C020E030E0820F931FEBCFDF91CF9157
:108A80000895CF93DF93DC01FB0180E090E0249117
:108A900041505109222389F04115510571F027FDFC
:108AA00006C0ED01C20FD11D288130E002C020E0D8
:108AB00030E0820F931F3196EACFDF91CF91089576
:108AC000CF93DF931F921F92CDB7DEB781118064E1
:108AD0006A8389830E94ED4E89810E94C04E6A811B
:108AE000862F0E94C04E80E00E94C04E0F900F90D3
:108AF000DF91CF910C94F24ECF93DF931F921F9290
:108B0000CDB7DEB78F736A8379830E94C04E7981B7
:108B1000872F0E94C04E6A81862F0E94C04E80E03F
:108B20000F900F90DF91CF910C94C04EEF92FF9277
:108B30000F931F93CF93DF9300D01F92CDB7DEB773
:108B40007A01890169837A838B839C830E94ED4E2D
:108B500069817A818B819C81CFDFB801C7010E9436
:108B6000D94E0F900F900F900F90DF91CF911F91E2
:108B70000F91FF90EF900C94F24ECF93DF9300D0C3
:108B80001F92CDB7DEB769837A838C839B830E9463
:108B9000ED4E69817A818C819B81AEDF34DF8C83DD
:108BA0000E94F24E8C810F900F900F900F90DF91EA
:108BB000CF91089564ED70E280E390E0DECF0F93F3
:108BC0001F93CF93DF9300D01F92CDB7DEB7698399
:108BD0007A838B839C830E94ED4E69817A818B819D
:108BE0009C818ADF10DF182F0EDF012F10E0182B79
:108BF0000E94F24EC8010F900F900F900F90DF91DE
:108C0000CF911F910F910895CF92DF92EF92FF9233
:108C1000CF93DF9300D01F92CDB7DEB769837A83FD
:108C20008B839C830E94ED4E69817A818B819C812C
:108C300063DFE9DEF82EE7DEE82EE5DE90E0A0E077
:108C4000B0E0DC01992788279E299C01AD012F29DE
:108C500069017A01D8DEA7019601582BCA01B90132
:108C600029837A838B839C830E94F24E69817A8167
:108C70008B819C810F900F900F900F90DF91CF917F
:108C8000FF90EF90DF90CF9008950F931F93CF93B5
:108C9000DF93EC01162F6CEF7FEF8FE290E0B4DFF3
:108CA000212F30E0A9014051510924E9249F80017E
:108CB000259F100D1124012E000C220B330B600F89
:108CC000711F821F931F24E930E0AE01DF91CF9125
:108CD0001F910F912BCFCF93DF931F921F92CDB790
:108CE000DEB780686A8379830E94C04E7981872FBE
:108CF0000E94C04E6A81862F0F900F90DF91CF9116
:108D00000C94C04ECF92DF92EF92FF920F93CF93CD
:108D1000DF9300D000D0CDB7DEB779014D835E83FD
:108D200069837A838B839C830E94ED4E69817A816B
:108D30008B819C81D0DF4D81C42E5E81D52EEC0CC1
:108D4000FD1CCE14DF0431F0F60181916F010E9409
:108D5000C04EF7CF002329F080E00E94C04E0150A2
:108D6000F9CF26960FB6F894DEBF0FBECDBFDF91C8
:108D7000CF910F91FF90EF90DF90CF900C94F24E37
:108D8000CF93DF9300D01F921F92CDB7DEB74D83F4
:108D900069837A838B839C830E94ED4E69817A81FB
:108DA0008B819C8198DF4D81842FEAD70F900F90A3
:108DB0000F900F900F90DF91CF910C94F24E81386D
:108DC00008F080E8482F64ED70E280E390E0D8CFAF
:108DD00040E864ED70E280E390E0D2CF0F931F9300
:108DE000CF93DF9300D01F92CDB7DEB78A0169839E
:108DF0007A838B839C83F1D769817A818B819C8173
:108E00006ADFB80180E090E001DE0F900F900F90D4
:108E10000F90DF91CF911F910F91E4C7CF93DF9314
:108E2000CDB7DEB728970FB6F894DEBF0FBECDBF23
:108E30002D833E834F83588769837A838B839C83FA
:108E4000CCD769817A818B819C8145DF2D813E81E0
:108E50004F815885CA01B901D9DD28960FB6F8941B
:108E6000DEBF0FBECDBFDF91CF91BCC7CF92DF92E7
:108E7000EF92FF9268EF70E280E390E0C5DE6B0155
:108E80007C016CEF70E280E390E0BEDEC626D72660
:108E9000E826F9268FE0D822EE24FF2481E0CD28B1
:108EA000CE28CF2809F480E0FF90EF90DF90CF909C
:108EB000089568EF70E280E390E0A6DE7F7081E0C5
:108EC0006F3F7F4009F080E00895AF92BF92CF924C
:108ED000DF92EF92FF920F93CF93DF937C01EB0130
:108EE000E8DF882311F080E028C00C2F0D5F0C7F95
:108EF0000C1B64E775E280E390E086DE6E01C00E35
:108F0000D11C7F706C157D0560F09E01A70168E79C
:108F100075E280E390E0F6DE81E00FC0AC14BD04A2
:108F2000A0F764E775E280E390E06EDE5B012FE07E
:108F3000B222BFDF882391F3D6CFDF91CF910F917B
:108F4000FF90EF90DF90CF90BF90AF900895CF93B8
:108F5000DF9300D01F92CDB7DEB749835A836B836E
:108F60007C8364E070E0CE010196AFDF0F900F903C
:108F70000F900F90DF91CF910895CF92DF92EF92F3
:108F8000FF92CF93DF93CDB7DEB728970FB6F89453
:108F9000DEBF0FBECDBF6A017B0189E09FEFAFEF5F
:108FA000BFEF8D839E83AF83B88764E070E0CE010E
:108FB00005968BDFC982DA82EB82FC8264E070E086
:108FC000CE01019682DF28960FB6F894DEBF0FBE61
:108FD000CDBFDF91CF91FF90EF90DF90CF900895BC
:108FE000CF92DF92EF92FF92CF93DF93CDB7DEB7B0
:108FF00028970FB6F894DEBF0FBECDBF6A017B0184
:109000008AE09FEFAFEFBFEF8D839E83AF83B8877A
:1090100064E070E0CE01059658DFC982DA82EB8207
:10902000FC8264E070E0CE0101964FDF28960FB617
:10903000F894DEBF0FBECDBFDF91CF91FF90EF90D0
:10904000DF90CF900895CF92DF92EF92FF92CF936F
:10905000DF93CDB7DEB728970FB6F894DEBF0FBE0B
:10906000CDBF6A017B0184E39FEFAFEFBFEF8D833C
:109070009E83AF83B88764E070E0CE01059625DF5C
:10908000C982DA82EB82FC8264E070E0CE01019654
:109090001CDF28960FB6F894DEBF0FBECDBFDF9160
:1090A000CF91FF90EF90DF90CF900895CF92DF9215
:1090B000EF92FF920F931F93CF93DF93CDB7DEB75D
:1090C00060970FB6F894DEBF0FBECDBF8DE09FEF67
:1090D000AFEFBFEF89839A83AB83BC837E836D83BD
:1090E00058874F833A8729871C870B87FE86ED8632
:1090F000D88ACF8660E170E0CE010196E6DE609608
:109100000FB6F894DEBF0FBECDBFDF91CF911F9198
:109110000F91FF90EF90DF90CF9008950F931F93E2
:10912000CF93DF93CDB7DEB72C970FB6F894DEBFA1
:109130000FBECDBF8CE09FEFAFEFBFEF89839A8367
:10914000AB83BC837E836D8358874F833A8729879F
:109150001C870B876CE070E0CE010196B6DE2C9682
:109160000FB6F894DEBF0FBECDBFDF91CF911F9138
:109170000F910895CF92DF92EF92FF920F931F937A
:10918000CF93DF93CDB7DEB760970FB6F894DEBF0D
:109190000FBECDBF82E19FEFAFEFBFEF89839A8310
:1091A000AB83BC837E836D8358874F833A8729873F
:1091B0001C870B87FE86ED86D12CD194C194D108F3
:1091C000D88ACF8660E170E0CE0101967EDE60969F
:1091D0000FB6F894DEBF0FBECDBFDF91CF911F91C8
:1091E0000F91FF90EF90DF90CF900895CF92DF9294
:1091F000EF92FF920F931F93CF93DF93CDB7DEB71C
:1092000060970FB6F894DEBF0FBECDBF8EE09FEF24
:10921000AFEFBFEF89839A83AB83BC837E836D837B
:1092200058874F833A8729871C870B87FE86ED86F0
:10923000D88ACF8660E170E0CE01019646DE609666
:109240000FB6F894DEBF0FBECDBFDF91CF911F9157
:109250000F91FF90EF90DF90CF9008958F929F92A3
:10926000AF92BF92CF92DF92EF92FF920F931F9334
:10927000CF93DF93CDB7DEB764970FB6F894DEBF18
:109280000FBECDBF84E19FEFAFEFBFEF89839A831D
:10929000AB83BC837E836D8358874F833A8729874E
:1092A0001C870B87FE86ED86D88ACF86BA8AA98A64
:1092B0009C8A8B8A64E170E0CE01019606DE64969A
:1092C0000FB6F894DEBF0FBECDBFDF91CF911F91D7
:1092D0000F91FF90EF90DF90CF90BF90AF909F9055
:1092E0008F9008958F929F92AF92BF92CF92DF920C
:1092F000EF92FF920F931F93CF93DF93CDB7DEB71B
:1093000064970FB6F894DEBF0FBECDBF83E19FEF29
:10931000AFEFBFEF89839A83AB83BC837E836D837A
:1093200058874F833A8729871C870B87FE86ED86EF
:10933000D88ACF86BA8AA98A9C8A8B8A64E170E02F
:10934000CE010196C2DD64960FB6F894DEBF0FBE63
:10935000CDBFDF91CF911F910F91FF90EF90DF90E4
:10936000CF90BF90AF909F908F900895EF92FF9213
:109370000F931F93CF93DF93CDB7DEB72E970FB622
:10938000F894DEBF0FBECDBF8DE29FEFAFEFBFEF12
:1093900089839A83AB83BC837E836D8358874F8395
:1093A0003A8729871C870B87FE86ED866EE070E082
:1093B000CE0101968ADD2E960FB6F894DEBF0FBE61
:1093C000CDBFDF91CF911F910F91FF90EF90089546
:1093D0008F929F92AF92BF92CF92DF92EF92FF92C5
:1093E0000F931F93CF93DF93CDB7DEB764970FB67C
:1093F000F894DEBF0FBECDBF81E19FEFAFEFBFEFAF
:1094000089839A83AB83BC837E836D8358874F8324
:109410003A8729871C870B87FE86ED86D88ACF86F8
:10942000BA8AA98A9C8A8B8A64E170E0CE0101968F
:109430004CDD64960FB6F894DEBF0FBECDBFDF9152
:10944000CF911F910F91FF90EF90DF90CF90BF9041
:10945000AF909F908F900895AF92BF92CF92DF927E
:10946000EF92FF920F931F93CF93DF93CDB7DEB7A9
:1094700062970FB6F894DEBF0FBECDBF8FE09FEFAF
:10948000AFEFBFEF89839A83AB83BC837E836D8309
:1094900058874F833A8729871C870B87FE86ED867E
:1094A000D88ACF86BA8AA98A62E170E0CE01019695
:1094B0000CDD62960FB6F894DEBF0FBECDBFDF9114
:1094C000CF911F910F91FF90EF90DF90CF90BF90C1
:1094D000AF900895AF92BF92CF92DF92EF92FF923A
:1094E0000F931F93CF93DF93CDB7DEB762970FB67D
:1094F000F894DEBF0FBECDBF80E19FEFAFEFBFEFAF
:1095000089839A83AB83BC837E836D8358874F8323
:109510003A8729871C870B87FE86ED86D88ACF86F7
:10952000BA8AA98A62E170E0CE010196CEDC629629
:109530000FB6F894DEBF0FBECDBFDF91CF911F9164
:109540000F91FF90EF90DF90CF90BF90AF90089574
:109550008F929F92AF92BF92CF92DF92EF92FF9243
:109560000F931F93CF93DF93CDB7DEB764970FB6FA
:10957000F894DEBF0FBECDBF8BE09FEFAFEFBFEF24
:1095800089839A83AB83BC837E836D8358874F83A3
:1095900009871A872B873C87FE86ED86D88ACF8677
:1095A000898A9A8AAB8ABC8A64E170E0CE0101960E
:1095B0008CDC64960FB6F894DEBF0FBECDBFDF9192
:1095C000CF911F910F91FF90EF90DF90CF90BF90C0
:1095D000AF909F908F900895CF92DF92EF92FF927D
:1095E0000F931F93CF93DF93CDB7DEB760970FB67E
:1095F000F894DEBF0FBECDBF8DE19FEFAFEFBFEFA1
:1096000089839A83AB83BC834D835E836F83788722
:1096100009871A872B873C87CD86DE86EF86F88AF6
:1096200060E170E0CE01019650DC60960FB6F894D0
:10963000DEBF0FBECDBFDF91CF911F910F91FF9085
:10964000EF90DF90CF9008950F931F93CF93DF9308
:10965000CDB7DEB72C970FB6F894DEBF0FBECDBFE7
:109660008EE19FEFAFEFBFEF89839A83AB83BC831B
:109670004D835E836F83788709871A872B873C87A2
:109680006CE070E0CE01019620DC2C960FB6F894C9
:10969000DEBF0FBECDBFDF91CF911F910F91089517
:1096A000EF92FF920F931F93CF93DF93CDB7DEB767
:1096B0002E970FB6F894DEBF0FBECDBF8CE29FEFA2
:1096C000AFEFBFEF89839A83AB83BC837E836D83C7
:1096D00058874F833A8729871C870B87FE86ED863C
:1096E0006EE070E0CE010196F0DB2E960FB6F89496
:1096F000DEBF0FBECDBFDF91CF911F910F91FF90C5
:10970000EF9008950F931F93CF93DF93CDB7DEB7FC
:109710002C970FB6F894DEBF0FBECDBF86E19FEF4A
:10972000AFEFBFEF89839A83AB83BC837E836D8366
:1097300058874F833A8729871C870B876CE070E036
:10974000CE010196C2DB2C960FB6F894DEBF0FBE99
:10975000CDBFDF91CF911F910F9108950F931F936C
:10976000CF93DF93CDB7DEB72C970FB6F894DEBF5B
:109770000FBECDBF89E39FEFAFEFBFEF89839A8321
:10978000AB83BC834D835E836F83788709871A8799
:109790002B873C876CE070E0CE01019696DB2C961F
:1097A0000FB6F894DEBF0FBECDBFDF91CF911F91F2
:1097B0000F910895CF93DF93CDB7DEB728970FB6FB
:1097C000F894DEBF0FBECDBF8AE39FEFAFEFBFEFD0
:1097D00089839A83AB83BC834D835E836F83788751
:1097E00068E070E0CE01019670DB28960FB6F89421
:1097F000DEBF0FBECDBFDF91CF910895CF93DF9332
:10980000CDB7DEB728970FB6F894DEBF0FBECDBF39
:1098100086E39FEFAFEFBFEF89839A83AB83BC836F
:10982000862F90E0A0E0B0E08D839E83AF83B88761
:1098300068E070E0CE01019648DB28960FB6F894F8
:10984000DEBF0FBECDBFDF91CF910895089508957B
:1098500064E670E080E090E00E942EFC21E030E0C1
:1098600040E050E060E270E280E390E0D7DA20E090
:1098700030E0A9016CEF70E280E390E0CFDA20E005
:1098800030E0A90168EF70E280E390E0C7DA20E001
:1098900030E0A90160E270E280E390E0BFDA6CE2C0
:1098A00071E080E090E00C942EFCAF92BF92CF92DA
:1098B000DF92EF92FF920F93CF93DF937B01EB0147
:1098C00009900020E9F72197C61BD70BF2DA811126
:1098D00027C021960C2F0D5F0C7F0C1B64E775E2EF
:1098E00080E390E091D96E01C00ED11C7F706C15A1
:1098F0007D0558F09E01A70168E775E280E390E0DE
:1099000001DA0EC0AC14BD04A8F764E775E280E389
:1099100090E07AD95B012FE0B222CBDA882391F371
:10992000DF91CF910F91FF90EF90DF90CF90BF909C
:10993000AF90089520E030E0A90168E570E280E38F
:1099400090E06CDA20E031E840E050E060E571E260
:1099500080E390E063DA20E030E0A90164E571E2A1
:1099600080E390E05BDA20E030E841EF5FEF68E50C
:1099700071E280E390E052DA20E030E0A9016CE58A
:1099800071E280E390E04ADA20E031EB4FEF5FEFE5
:1099900060E671E280E390E041DA20E030ED40E201
:1099A00051E064E671E280E390E038CACF93DF9340
:1099B0001F92CDB7DEB762E0CE0101961FDF0F9098
:1099C000DF91CF910895CF939ED10ED260E088E4CD
:1099D00077D860E080E074D8CAEF60E070E280E39E
:1099E00090E0CBD88C3709F0AEC040E064ED70E277
:1099F00080E390E0C5D94DE052E06CE270E280E394
:109A000090E0ECD94CE250E060E370E280E390E05B
:109A1000E5D94AE250E068E370E280E390E0DED905
:109A200043E550E06CE370E280E390E0D7D94EE18B
:109A300051E060E470E280E390E0D0D94DE050E086
:109A400064E470E280E390E0C9D94BE050E06CE45C
:109A500070E280E390E0C2D945E150E060E570E259
:109A600080E390E0BBD940EE51E064E370E280E334
:109A700090E0B4D940E151E068E470E280E390E026
:109A8000ADD940E064E670E280E390E079D941E04E
:109A90006CE670E280E390E073D940E068E670E243
:109AA00080E390E06DD920E030E040E052E060E0FB
:109AB00070E080E390E0B2D927E030E040E056E289
:109AC00064E070E080E390E0A9D920E030E0A901F3
:109AD00068E070E080E390E0A1D942E064E570E2E4
:109AE00080E390E04DD940ED57E068E171E280E31A
:109AF00090E074D940E064E870E280E390E040D9FF
:109B000041E860E970E280E390E03AD941E864E935
:109B100070E280E390E034D947E060E770E280E3F0
:109B200090E02ED94AEF50E060ED70E280E390E0E3
:109B300055D940E060E670E280E390E021D988DE0C
:109B4000F9DECF9133CF61E070E080E090E00E94D9
:109B50006538C15009F041CF48CFEF92FF920F9383
:109B60001F93CF93DF931F92CDB7DEB78C01060F03
:109B7000171F7C01E016F10649F0F7018491498333
:109B8000FFD0FFEFEF1AFF0A4981F4CF142F112302
:109B900021F080E0F5D01150FACF0F90DF91CF91F6
:109BA0001F910F91FF90EF900895CF92DF92EF9267
:109BB000FF920F93CF93DF9300D01F92CDB7DEB704
:109BC0006A01790169837A838B839C8306D16981D9
:109BD0007A818B819C817FD8402FB701C601BDDF80
:109BE0000F900F900F900F90DF91CF910F91FF90FA
:109BF000EF90DF90CF90F6C0AF92BF92CF92DF92FE
:109C0000EF92FF920F93CF93DF937B01EA0151D93B
:109C1000882311F080E02AC00C2F0D5F0C7F0C1BF5
:109C200064E775E280E390E00E9404466E01C00E96
:109C3000D11C7F706C157D0560F09E01A70168E75F
:109C400075E280E390E0B1DF81E010C0AC14BD04A8
:109C5000A0F764E775E280E390E00E9404465B01B0
:109C60002FE0B22226D9882389F3D4CFDF91CF9178
:109C70000F91FF90EF90DF90CF90BF90AF9008953D
:109C80000F931F93CF93DF931F921F92CDB7DEB731
:109C90008C01CB0169837A830F94E5A0AC014F5FFF
:109CA0005F4F69817A81C8010F900F90DF91CF914A
:109CB0001F910F91A1CFCF92DF92EF92FF920F935E
:109CC000CF93DF9300D01F92CDB7DEB76A01790141
:109CD00069837A838B839C8380D069817A818B812D
:109CE0009C810E946B46402FB701C60136DF0F9062
:109CF0000F900F900F90DF91CF910F91FF90EF9009
:109D0000DF90CF906FC0CF93DF93539A5B98529AB6
:109D10005A9A9C9AA49AE1E0F1E080818064808361
:109D2000C2E0D1E088818074A0E0B1E08C938081B2
:109D30008B7F80838881809584708C93DF91CF9115
:109D40000895482FF89438E080E020E8922F94237B
:109D500011F0A49A01C0A49890910201909590747A
:109D60009093000190910201907490930001909162
:109D7000000192FD822B2695315041F77894089589
:109D8000F89428E030E8932F982311F0A49A01C0AA
:109D9000A4989091020190959074909300019091F5
:109DA00002019074909300013695215061F77894E8
:109DB00008950F931F93CF93DF93EC018C01060F4F
:109DC000171FC017D10721F080E0BBDF8993F9CFBF
:109DD000DF91CF911F910F9108955A9881E090E003
:109DE0000C949E385A9A08955B9866E070E080E083
:109DF00090E00E9465385B9A65E170E080E090E059
:109E00000C946538FC018081F2E18F9FC001112420
:109E100085519F4B092E000CAA0BBB0BABBFFC015D
:109E200087919691FC01199480913E038093460797
:109E3000089580913F03909146078923089590915A
:109E40003F0389238093460708959091460780FB3E
:109E500090F980FB91F980FB92F990934607089561
:109E600090914607977081E009F480E00895909101
:109E7000460780FB93F99093460708958091460723
:109E800083FB882780F9089580914507089581E034
:109E900090914507911101C080E00895CF93DF9321
:109EA00061E087E497E00E949158882309F4B9C0E3
:109EB0000E9436478111B5C06CE271E280E390E008
:109EC0000E94BD45C82F90914507911132C088234B
:109ED00009F452C08093450782E597E093DFD09163
:109EE000520722E1D29FC001112481519F4B092EBC
:109EF000000CAA0BBB0BABBFFC01279136918C2F3A
:109F0000F9011995882359F087E497E00E94B05829
:109F10008091460780FF03C06CE388E560D2909192
:109F2000520780914607D91711F0806243C08F7D98
:109F300041C08091460784FD3AC0C9132EC064E039
:109F400087E497E00E949158882309F46AC0409101
:109F50005207F2E14F9FA00111244F505F4B052E95
:109F6000000C660B770B6BBFFA01479156918C2F53
:109F7000FA011995811106C087E497E0DF91CF912E
:109F80000C94B05882E597E03DDF8091460782FF50
:109F9000F3CF6CE388E523D2EFCFC11142C087E451
:109FA00097E00E94B05880914607806103C0C913B2
:109FB00004C08F7E8093460734C063E087E497E057
:109FC0000E949158882369F1809146078F7E809383
:109FD000460785FF06C08F7D809346071092450790
:109FE00020C081FF03C06CE386E5F9D1809145076D
:109FF0001092450740915207F2E14F9FA0011124B2
:10A000004D505F4B052E000C660B770B6BBFFA01B2
:10A0100047915691FA01199582E597E0DF91CF912A
:10A02000F1CEDF91CF910895CEDCABD0FDDE82E59D
:10A0300097E00C94FA5A89E497E03BD28091460766
:10A0400086FD1BC08064809346078091520722E101
:10A05000829FC001112487519F4B092E000CAA0B2F
:10A06000BB0BABBFFC0187919691FC01199516DFE4
:10A07000809146078F7B8093460708950F931F9327
:10A08000CF93662351F08901C62FFEDE8C1305C0E5
:10A0900080E091E0F8019183808380E0CF911F916F
:10A0A0000F91089521E0FC0185819681892B09F4A7
:10A0B00020E0822F0895CF92DF92EF92FF920E94CC
:10A0C00034386B017C010E943438DC01CB018C19DF
:10A0D0009D09AE09BF098B3F9105A105B10548F067
:10A0E0000E9460FC8FE29AE00E9452FCB1DB80E0AB
:10A0F00007C00E94D3DA0E9436478111E4CF81E085
:10A10000FF90EF90DF90CF9008954F925F926F9203
:10A110007F928F929F92AF92BF92CF92DF92EF92F7
:10A12000FF920F931F932A013B014801590128E038
:10A13000829FC00111246C01990FEE08FF08C7012E
:10A14000B6016F5F7F4F804F9F4FA30192010E9426
:10A150000E47C701B6016B5F7F4F804F9F4FA50130
:10A1600094011F910F91FF90EF90DF90CF90BF90DF
:10A17000AF909F908F907F906F905F904F900C94D6
:10A180000E470F931F93CF9325ED37E04FE050E03C
:10A1900061ED77E08FE090E00E940E47C0E000E0C4
:10A1A00010E0980140E050E0BA018C2FAEDFCF5FA5
:10A1B000CA3FA9F7CF911F910F9108954F925F92D7
:10A1C0006F927F929F92AF92BF92CF92DF92EF9267
:10A1D000FF920F931F93CF93DF931F92CDB7DEB7FC
:10A1E0005C012A013B01CE01019630DBCE010196D4
:10A1F0002EDBC50160DF982E811102C0912C81C039
:10A2000060E071E280E390E00E9404466B017C0113
:10A210002FE1D222EE24FF24F50181819281A381D6
:10A22000B481892B8A2B8B2B01F561ED77E08FE0D0
:10A2300090E00E940446F5016183728383839483D6
:10A2400020E030E040E150E0261B370B480B590B73
:10A25000DA01C901411451046104710411F42601A9
:10A260003701F501D682C58212C041145104610440
:10A27000710429F4F50145805680612C712CF5019B
:10A28000D682C582D301C201412C512C3201F50185
:10A29000C580D680E12CF12C8C159D05AE05BF053F
:10A2A00008F4ACCF418152816381748100E010E0F9
:10A2B00020E330E0CE0101968FD9CE010196C7DAB6
:10A2C000F5010581168120E030E0418152816381F2
:10A2D000748180811ADF411451046104710489F092
:10A2E000F50181819281A381B481A3019201280F9C
:10A2F000391F4A1F5B1F61ED77E08FE090E00E94FD
:10A300000E47892D0F90DF91CF911F910F91FF90F4
:10A31000EF90DF90CF90BF90AF909F907F906F9025
:10A320005F904F900895CF93DF93EC01688188E0B0
:10A33000689FB0011124CB01770FAA0BBB0BBC01A6
:10A34000CD016F5F7F4F804F9F4F0E94044669830E
:10A350007A838B839C83688188E0689FB001112495
:10A36000CB01770FAA0BBB0BBC01CD016B5F7F4FFD
:10A37000804F9F4F0E9404467E836D83DF91CF9173
:10A380000895EF92FF920F931F93CF93DF931F9245
:10A39000CDB7DEB77C01CE01019658DAF701058111
:10A3A000168120E030E04181528163817481CE01C9
:10A3B00001964AD90F90DF91CF911F910F91FF9095
:10A3C000EF900895482F64E870E280E390E00C94E9
:10A3D000C04664E870E280E390E00C94BD456623DB
:10A3E00021F0482F50E0562B02C040E050E068E8D2
:10A3F00070E280E390E00E94EE4641E06CE870E29B
:10A4000080E390E00C94C04680E090E00F94369991
:10A410000F94A99A2CED36EC42EC50E40F94BC97C3
:10A4200020E030E040E451E40F94199B28E132E74A
:10A4300041E35FE30F949D9820E030E04AE852E466
:10A440000F94BD9720E030E040E05FE30F94BD97AC
:10A450000F940A99862F08950F931F93CF93DF933C
:10A46000EC018A01D1DF682F84E4B9DF87E59AE047
:10A470009A838983B80180E090E00F94369920E0B8
:10A4800030E040E85CE30F94199B0F9483980F949D
:10A490000A996C83CE010396DF91CF911F910F91A2
:10A4A0005FC66CE870E280E390E00E94BD45817079
:10A4B00008950F931F93CF93DF93FC012181328185
:10A4C000232B09F44BC0EC016481611104C0E9DF66
:10A4D00091E0892702C0039624D6882309F43EC060
:10A4E00029813A81F9010491319614913196249190
:10A4F00030E0A8EEB3E00F945B9C24E0969587953E
:10A50000779567952A95D1F76115710581059105B4
:10A5100069F401110BC01F3F49F41A82198260E0EF
:10A5200080E0DF91CF911F910F9159CF0F94369911
:10A5300020E030E040E85CE30F94199B0F9483988F
:10A540000F940A996C83CE0103960AD6612F802F4F
:10A5500046DF89819A8104969A838983DF91CF911E
:10A560001F910F9108950F931F93CF93DF931F9225
:10A57000CDB7DEB78C01FC017283618384E08483F4
:10A58000C80103964983ECD54981442351F0F80171
:10A5900081819281892B29F0C8018BDF0E94D3DA57
:10A5A000F6CF0F90DF91CF911F910F910895E9E4BD
:10A5B000F7E0108214820895E82F880FFF0BE55C06
:10A5C000F54F8491089508950F931F93CF93DF93D0
:10A5D000CDB7DEB7C459D1090FB6F894DEBF0FBEB0
:10A5E000CDBF8C016FE1CE0101960E9445464FE13F
:10A5F000BE016F5F7F4FC8016FD2CC56DF4F0FB6E1
:10A60000F894DEBF0FBECDBFDF91CF911F910F91A8
:10A610000895EF92FF920F931F93CF93DF93EB0177
:10A620007901B8019801205231092036310508F02E
:10A630000FE3E02FF0E0E55CF54F14916930710510
:10A6400021F4EBE5FAE0149100E2009739F0FA0109
:10A6500040815181688179812FE1F0D2812F90E092
:10A66000A0E0B0E06627782F892F9A2F970140E06D
:10A6700050E00F94379C88819981820F911D9983B6
:10A68000888381E0DF91CF911F910F91FF90EF9030
:10A690000895E82FF0E0E555F54F649170E080E013
:10A6A00091E30F94EE9BCB010895FC012081318151
:10A6B00040E050E060E071E380E090E00F94379C70
:10A6C000822F0895FC019191992329F0907C903874
:10A6D000D1F781E0089580E00895FC0194919923D9
:10A6E00031F03196907C9038C9F781E0089580E090
:10A6F0000895FC01A081B181CD01019691838083F1
:10A700009C91892F90E0A081B1812C91207C2038F0
:10A7100051F4982F88279D012F5F3F4F318320836D
:10A720002C91822BF0CF08958F929F92AF92BF927F
:10A73000CF92DF92EF92FF920F931F93CF93DF930D
:10A7400000D000D0CDB7DEB76C017A8369835C831B
:10A750004B833E832D835801E62EF72EED81FE813B
:10A7600080818823C9F0CE010596C3DF8C01950155
:10A77000AE014D5F5F4FBE016F5F7F4FC601DDD3FE
:10A780008111ECCF9501AE014D5F5F4FBE016F5F50
:10A790007F4FC6013EDFE2CF89819A818E199F09E2
:10A7A00026960FB6F894DEBF0FBECDBFDF91CF91D6
:10A7B0001F910F91FF90EF90DF90CF90BF90AF90DF
:10A7C0009F908F900895CF92DF92EF92FF926C014D
:10A7D000E12CF12CC701B601BAD2C701B601FF9036
:10A7E000EF90DF90CF90EFCECF93DF93EC0147D384
:10A7F000CE01DF91CF91E8CECF92DF92EF92FF9220
:10A800000F931F93CF93DF9300D01F92CDB7DEB786
:10A810007B011C821B821A8219828C019B01AE0172
:10A820004F5F5F4FBE016D5F7F4F80E090E085D34B
:10A8300081110AC09701AE014F5F5F4FBE016D5F8E
:10A840007F4F80E090E0E5DE8B819C810F900F9040
:10A850000F900F90DF91CF911F910F91FF90EF908C
:10A86000DF90CF9008950F931F938B019C0140E0E0
:10A8700050E060E070E080E090E056DF1F910F91C3
:10A880000895AF92BF92CF92DF92EF92FF920F9313
:10A890001F93CF93DF93CDB7DEB77C015B01CDB6BD
:10A8A000DEB60F94E5A001962DB73EB7281B390BF5
:10A8B0000FB6F8943EBF0FBE2DBF0DB71EB70F5F8A
:10A8C0001F4FB701C8010F94DEA0B501C801CBDF4F
:10A8D0000FB6F894DEBE0FBECDBEDF91CF911F91B3
:10A8E0000F91FF90EF90DF90CF90BF90AF900895C1
:10A8F0006F927F928F929F92AF92BF92CF92DF9290
:10A90000EF92FF920F931F93CF93DF931F921F92AB
:10A91000CDB7DEB76C015B014A0139011A830983A7
:10A9200040E050E060E072E20E94A74749815A810E
:10A9300060E070E07561C6010E94A74749815A81B5
:10A9400060E070E07961C6010E94A74741E050E0F5
:10A9500060E07FE1C6010E94A747F1FE07C0698160
:10A960007A81C30180DF9695879506C0F3FE06C005
:10A9700069817A81C30177DFA81AB90AF2FE06C09D
:10A98000CE01019692DE8695881A910809811A8176
:10A990009301A401B501C601C7DE40E050E060E0CC
:10A9A00073E2C6010E94A7470F900F90DF91CF91ED
:10A9B0001F910F91FF90EF90DF90CF90BF90AF90DD
:10A9C0009F908F907F906F9008954F925F926F92BB
:10A9D0007F928F929F92AF92BF92CF92DF92EF922F
:10A9E000FF920F931F93CF93DF931F921F92CDB7C8
:10A9F000DEB75C014B0129016DB67EB6C901498302
:10AA00005A830F94E5A001962DB73EB7281B390B4A
:10AA10000FB6F8943EBF0FBE2DBF8DB79EB70196FF
:10AA20006C01B2010F94DEA0960149815A81B401F4
:10AA3000C5015EDF0FB6F8947EBE0FBE6DBE0F90EF
:10AA40000F90DF91CF911F910F91FF90EF90DF90CA
:10AA5000CF90BF90AF909F908F907F906F905F90BE
:10AA60004F9008959F92AF92BF92CF92DF92EF9254
:10AA7000FF920F931F93CF93DF93EC018B017A0129
:10AA8000E2E0EE16F104E0F0F801A4900E5F1F4F33
:10AA90003196B490BE019C2E9A0C961659F06B011B
:10AAA000FFEFCF1ADF0A80E090E04B2D0E94C046F6
:10AAB000B601F3CFCA0DD11D82E0E81AF108E0CF4C
:10AAC000DF91CF911F910F91FF90EF90DF90CF908A
:10AAD000BF90AF909F900895AF92BF92CF92DF92B8
:10AAE000EF92FF920F931F93CF93DF93EC018B01B3
:10AAF0004F7150E060E070E075600E94A747F80178
:10AB0000E057FF4F40815181628173817160CE01B6
:10AB10000E94A74778018CE8E80EF11CF701A0809D
:10AB2000B1803897C080D180C5019170A0E0B0E0BD
:10AB3000AC01BD017760349790819F71892F90E0BF
:10AB4000A0E0B0E023E1880F991FAA1FBB1F2A9540
:10AB5000D1F7842B952BA62BB72BA601537060E061
:10AB600070E039E0440F551F661F771F3A95D1F703
:10AB7000482B592B6A2B7B2BCE010E94A7474B2DCC
:10AB80004695437050E060E070E078628D2D8695C8
:10AB90008695837090E0A0E0B0E0E2E0880F991F16
:10ABA000AA1FBB1FEA95D1F7482B592B6A2B7B2B89
:10ABB000CE010E94A747F701E080F1803497008121
:10ABC0001181A701517060E070E060617860C80198
:10ABD0009170A0E0B0E0F9E0880F991FAA1FBB1F99
:10ABE000FA95D1F7482B592B6A2B7B2BCE010E946B
:10ABF000A7474F2D4695437050E060E070E07962C2
:10AC0000812F8695837090E0A0E0B0E012E0880F7D
:10AC1000991FAA1FBB1F1A95D1F7482B592B6A2BD6
:10AC20007B2BCE01DF91CF911F910F91FF90EF9081
:10AC3000DF90CF90BF90AF900C94A747AF92BF9298
:10AC4000CF92DF92EF92FF920F931F93CF93DF93F8
:10AC5000E22FEF71102F1F77611522E0720720F4A9
:10AC6000411522E05207A8F17A01EB015C014E2F59
:10AC700050E060E070E075600E94A747412F50E00F
:10AC800060E070E07660C5010E94A747F701B4E07C
:10AC9000EE0FFF1FBA95E1F7FF77AF0160E070E0BC
:10ACA0007064CE01C4E0880F991FCA95E1F7EC01EA
:10ACB000DF77CE01A0E0B0E0DFE0880F991FAA1F88
:10ACC000BB1FDA95D1F7482B592B6A2B7B2BC5017B
:10ACD00032C0012F10E020E030E03068CE2ED12CC1
:10ACE000E12CF12CE7E0CC0CDD1CEE1CFF1CEA95FE
:10ACF000D1F70C291D292E293F296A01E12CF12CBD
:10AD0000FCE0CC0CDD1CEE1CFF1CFA95D1F70C29E5
:10AD10001D292E293F296B01E12CF12CA5E1CC0C3A
:10AD2000DD1CEE1CFF1CAA95D1F7B901A8014C2926
:10AD30005D296E297F29DF91CF911F910F91FF909F
:10AD4000EF90DF90CF90BF90AF900C94A747CF9239
:10AD5000DF92EF92FF920F93CF93DF93CDB7DEB7E1
:10AD6000C459D1090FB6F894DEBF0FBECDBF6B0139
:10AD70007C01DC01CB018C569F4FAF4FBF4FCF56AC
:10AD8000DF4F88839983AA83BB83C159D04082E077
:10AD900090E0A0E0B0E0CF57DF4F88839983AA838B
:10ADA000BB83C158D04083E190E0A0E0B0E0CB5736
:10ADB000DF4F88839983AA83BB83C558D04086E23E
:10ADC00090E0A0E0B0E0C757DF4F88839983AA8363
:10ADD000BB83C958D04081E390E0A0E0B0E0C35706
:10ADE000DF4F88839983AA83BB83CD58D040AE01BF
:10ADF0004F5F5F4FFA018FE7840F11928E13FDCFE3
:10AE000080E090E0FC01E053F54F3491FC01EF52FB
:10AE1000F54F2491FC01EE52F54FE491311104C03D
:10AE2000DA01A20FB11DEC9305968C3221E0920756
:10AE300049F700E024E930E0C701B6010E948246EC
:10AE4000C6018C569F4F40ED59E06AEF7BE00ADE69
:10AE5000C0924E07D0924F07E0925007F0925107F0
:10AE6000CC56DF4F0FB6F894DEBF0FBECDBFDF91DB
:10AE7000CF910F91FF90EF90DF90CF900895CF93F7
:10AE8000DF93CDB7DEB7C459D1090FB6F894DEBF52
:10AE90000FBECDBF40914E0750914F0760915007B4
:10AEA000709151074C565F4F6F4F7F4FCF56DF4F1A
:10AEB000488359836A837B83C159D04042E050E084
:10AEC00060E070E0CF57DF4F488359836A837B830C
:10AED000C158D04043E150E060E070E0CB57DF4F15
:10AEE000488359836A837B83C558D04046E250E04B
:10AEF00060E070E0C757DF4F488359836A837B83E4
:10AF0000C958D04041E350E060E070E0C357DF4FE4
:10AF1000488359836A837B83CD58D04041E0BE018A
:10AF20006F5F7F4FD9DDCC56DF4F0FB6F894DEBF91
:10AF30000FBECDBFDF91CF9108954F925F926F9278
:10AF40007F928F929F92AF92BF92CF92DF92EF92B9
:10AF5000FF920F931F93CF93DF932901F801E15ADA
:10AF6000F24CEF31F14008F070C0FCE3DF2ED0E08E
:10AF7000A5E0CA2EED2E0D2E000CFF0837016D0C3A
:10AF8000711CD7FC7A9477FE03C03FEF631A730AF3
:10AF900075946794C62D2C2D362D3203F0011124A3
:10AFA000E253F54FA591B491A017B10759F0DD1503
:10AFB00009F44BC0A017B10710F0D62CDFCFD1E0B9
:10AFC000D60DD8CFCF3F09F440C0D8015A017B013C
:10AFD0006C0185E0689EB0011124FB01E053F54F40
:10AFE000D491FB01EF52F54F0491FB01EE52F54F66
:10AFF000C491612C712CD11113C0A03BB24C39F516
:10B0000060E079E080E090E0A30192010F94379C2A
:10B01000F70180819181821B91099183808317C000
:10B0200060EF862E8C0E8D2F90E00F94B1A0892BAF
:10B0300011F4912C02C059EF952E8D2FBDDAC82F37
:10B04000D93659F4D02F07E002C080E059C0C114AE
:10B05000D10409F441C021E008C0C114D10409F4AD
:10B060003BC0802F0D2FD82F2FE1F501408151815A
:10B07000F70160817181C601E1DDDD2369F1892D70
:10B08000990C990BAA0BBB0B6627782F892F9A2F47
:10B09000A30192010F94379CF501A080B180A20E0C
:10B0A000B11C27FDBA94882D880C990BAA0BBB0BF9
:10B0B0006627782F892F9A2FA30192010F94379C2E
:10B0C000F70160817181620F711D27FD7A950D2F47
:10B0D00021E0A501C601B2DD8C2F90E0A0E0B0E038
:10B0E0006627782F892F9A2FA30192010F94379CFE
:10B0F000F70180819181820F911D9183808381E08E
:10B10000DF91CF911F910F91FF90EF90DF90CF9043
:10B11000BF90AF909F908F907F906F905F904F9077
:10B1200008950F931F93CF938C01C62F0E9434383C
:10B130000F94369920E030E040E85CE30F94199BCF
:10B140000F9483980F940A99F8018081962F981B89
:10B1500081E09C1708F480E0CF911F910F91089532
:10B16000CF93DF93EC010E9434380F94369920E09E
:10B1700030E040E85CE30F94199B0F9483980F94A0
:10B180000A996883DF91CF9108956F927F928F9291
:10B190009F92AF92BF92CF92DF92EF92FF920F9366
:10B1A0001F93CF93DF931F921F92CDB7DEB75C0141
:10B1B0006B014A017901FC016081718180E290E0BC
:10B1C0001BDBC81AD90A9A828982F7019182808290
:10B1D000612C712C00E010E0CE0101968ADA8032F9
:10B1E000910509F18A309105F1F0009771F40C1581
:10B1F0001D05A0F0F701208131812815390561F086
:10B200000097D9F08A309105C1F0F5016081718114
:10B21000F3DA080F191FE0CF009741F429813A8132
:10B220002150310905C00C151D0520F729813A81EF
:10B23000F701318320833801E3CFF70180819181C9
:10B240008815990531F489819A81019791838083CA
:10B250003801C3010F900F90DF91CF911F910F9193
:10B26000FF90EF90DF90CF90BF90AF909F908F9026
:10B270007F906F9008952F923F924F925F926F92BE
:10B280007F928F929F92AF92BF92CF92DF92EF9276
:10B29000FF920F931F93CF93DF93CDB7DEB72C9719
:10B2A0000FB6F894DEBF0FBECDBF9E838D837A8725
:10B2B000698758874F8319012DB73EB73C872B8785
:10B2C00080E091E09C838B838A2DE3D99C838B83E0
:10B2D0004701412C512C612C712C9E012F5F3F4F57
:10B2E000A401B101CE01039650DF29813A812815CE
:10B2F000390561F06816790608F43C01CE01039621
:10B30000D4D9480E511C89809A80E7CF261437047F
:10B3100018F00415150540F4AA948A2DBAD99C8317
:10B320008B833AE1A312D4CFD3FC0FC0460188240B
:10B3300082E09822D1FE0AC0410137FE03C09FEF90
:10B34000891A990A9594879401C0410136016624AF
:10B3500024E07222D2FE05C0041915093801769442
:10B360006794E894D2F889859A85880E991E2A2DCB
:10B3700030E03A8729879E012F5F3F4FA701B10137
:10B38000CE01039602DF09811A810E151F0509F40B
:10B3900057C00E191F0909F447C04DB65EB6C80163
:10B3A00001962DB73EB7281B390B0FB6F8943EBF58
:10B3B0000FBE2DBF8DB79EB701965C01A801B701E6
:10B3C0000F9483A1F501E00FF11F108201501109C4
:10B3D000F501E00FF11F80818A3011F0803209F40D
:10B3E0001082C5016FD94F815885460D571D88239E
:10B3F00049F00B811C8176019501B4018D819E81FC
:10B4000077DA0DC0860129853A85B4018D819E8148
:10B410000E948E48B5018D819E810E94554C0FB6C9
:10B42000F8945EBE0FBE4DBECE0103963ED92F816D
:10B430003885280F311D38872F83E980FA809BCF0C
:10B440008B859C850FB6F8949EBF0FBE8DBF2C9642
:10B450000FB6F894DEBF0FBECDBFDF91CF911F9125
:10B460000F91FF90EF90DF90CF90BF90AF909F90A3
:10B470008F907F906F905F904F903F902F900895A6
:10B480002F923F924F925F926F927F928F929F92F4
:10B49000AF92CF92DF92EF92FF920F931F93CF93D1
:10B4A000DF9300D01F92CDB7DEB74C013B011701EF
:10B4B0004DB65EB6C7012B833C8349835A830F94F4
:10B4C000E5A001966DB77EB7681B790B0FB6F894AF
:10B4D0007EBF0FBE6DBF8DB79EB701967C01B101D7
:10B4E0000F94DEA02B813C8149815A81B301C401B4
:10B4F000C2DE0FB6F8945EBE0FBE4DBE0F900F9029
:10B500000F900F90DF91CF911F910F91FF90EF90CF
:10B51000DF90CF90AF909F908F907F906F905F90D3
:10B520004F903F902F900895FC018081F2E18F9F12
:10B53000C00111248B519F4B092E000CAA0BBB0B91
:10B54000ABBFFC0187919691FC011994FC018081AD
:10B55000F2E18F9FC001112489519F4B092E000CED
:10B56000AA0BBB0BABBFFC0187919691FC01199410
:10B57000DB019091C8052DEE30E480E0891781F061
:10B58000A901032E000C660B770B6BBFFA014791E4
:10B5900056912E5E3F4FA417B50719F08F5FEECF7F
:10B5A0008FEF0895CF93DF93EC01E2DF8F3F09F037
:10B5B0008883DF91CF9108951F93CF93DF93C0E0ED
:10B5C000D091C80512E1CD1788F41C9FC001112449
:10B5D0008D519F4B092E000CAA0BBB0BABBFFC017E
:10B5E00087919691FC011995CF5FEDCFDF91CF91B7
:10B5F0001F910895CF93DF93EC01DEDFCE01DF9141
:10B60000CF9192CFCF93DF93EC018B818C838A8192
:10B610008B8389818A83CE01ABDF8983DF91CF91D0
:10B620000895FC0183818483828183838181828365
:10B63000808181830895FC0182818183838182835B
:10B640008481838314820895FC0121812083F3CFB8
:10B650000F931F93CF93DF931F921F92CDB7DEB747
:10B660008C0169837A83DDDFC80170DF69817A81AB
:10B67000C80198DFC8010F900F90DF91CF911F9103
:10B680000F9152CFCF93DF93EC0160DFCE01DCDF6F
:10B69000CE01DF91CF9148CF1092520708958F923B
:10B6A0009F92AF92BF92CF92DF92EF92FF920F9351
:10B6B0001F93CF93DF93CDB7DEB7C459D1090FB62F
:10B6C000F894DEBF0FBECDBF182F6B015A01790170
:10B6D000C90103D8082F1A3184F1002399F0812F72
:10B6E0000E944953BC01C701CCD84C01812F0E9454
:10B6F00049539A838983CE0101960E945553E82FBE
:10B70000F0E013C0612FCE0101960E9445464FEF35
:10B710005FE7B701CE0101960E9441454C01C35736
:10B72000DF4FE881F981CD58D0408C149D041CF482
:10B73000EA15FB0514F01150CECF812FCC56DF4F08
:10B740000FB6F894DEBF0FBECDBFDF91CF911F9132
:10B750000F91FF90EF90DF90CF90BF90AF909F90B0
:10B760008F9008954F925F926F927F928F929F92E7
:10B77000AF92BF92CF92DF92EF92FF92CF93DF937F
:10B78000EC01FB01C080D180E280F3808084918451
:10B79000A284B38444805580668077804485558533
:10B7A0006685778574600E94A747B301A201CE0128
:10B7B0000E942348B501A401CE010E94F047B701C1
:10B7C000A601CE010E94BD47CE01DF91CF91FF902F
:10B7D000EF90DF90CF90BF90AF909F908F907F9031
:10B7E0006F905F904F900895813041F0833059F40D
:10B7F00062E276EB82E597E02BDF03C082E597E01B
:10B8000041DF81E0089580E008952F923F924F92AA
:10B810005F926F927F928F929F92AF92BF92CF92E0
:10B82000DF92EF92FF920F931F93CF93DF9300D09D
:10B8300000D0CDB7DEB75C013B012A01222E3B834D
:10B840000C831E834701DA82C982E0911802F091CD
:10B850001902309769F000E09E012F5F3F4FAC0165
:10B860004E5F5F4FDC0111966C9119958D8301C07D
:10B870001D8289819A8195FF03C0F501308009C03E
:10B8800094014C815E81622D7B81D5018C9107DF13
:10B89000382EC980DA80E32C032C000CFF080C81C1
:10B8A0001E81222D3B81A201B301C5010E94564891
:10B8B000C4010E946D53882309F44BC06AEC75E102
:10B8C000C5010E94404E822D9B8197FD0196959562
:10B8D0008795680E791E8C819E8197FD01969595BE
:10B8E0008795480E591E89819A8190FD25C040E0B8
:10B8F00050E060E072E2C5010E94A74740E050E0DE
:10B9000060E074E0C5010E94A747832D0E9449535F
:10B91000E12C36E0F32E8C019401A2014150510933
:10B92000B30161507109C50150D840E050E060E0BA
:10B9300073E2C5010E94A747832D0E944953E12C61
:10B9400026E0F22E8C019401A201B301C5013DD87D
:10B9500004C0B401C5010E94404EE0911802F0916C
:10B960001902309779F0BD81BB2361F001E09E019F
:10B970002F5F3F4FA5014E5F5F4FD50111966C9130
:10B98000C5011995C50126960FB6F894DEBF0FBE06
:10B99000CDBFDF91CF911F910F91FF90EF90DF907E
:10B9A000CF90BF90AF909F908F907F906F905F905F
:10B9B0004F903F902F900895AF92BF92CF92DF9219
:10B9C000EF92FF920F931F93CF93DF9300D0CDB7E9
:10B9D000DEB7B82E80FF21C0CE0101960E94264C12
:10B9E0008AE189831A821B824FEF5FEF6FEF72E06B
:10B9F000CE0101960E94A74747E050E060E076E262
:10BA0000CE0101960E94A7471A8240E050E060E014
:10BA100073E0CE0101960E94A747B1FE94C0CE010B
:10BA200001960E94264C1A821B828CE1898328EEA3
:10BA300035E14FE250E06AE071E031DEB82E88EE89
:10BA400095E10E946D53882391F08B2D0E944953FC
:10BA5000E12C36E0F32E8C0128EE35E14AE150E08E
:10BA600068E870E0CE0101960E94E55413C02B2DCA
:10BA7000BB0C330B00E016E04AE150E068E870E0F0
:10BA8000CE0101960E948E4868EE75E1CE010196C6
:10BA90000E94404E8BE1898360E573E0CE01019600
:10BAA00061DE5C01FC0182818068828382E08183A7
:10BAB00042E050E060E073E0C5010E94A747C12C5E
:10BAC000D12C8AEDE82E85E1F82E0FE210E02AE075
:10BAD00031E048E350E063E070E0C50196DE5C01D0
:10BAE000FC0182818F77828383E0818343E050E091
:10BAF00060E073E0C5010E94A7479BECE92E95E149
:10BB0000F92E2AE031E04DE650E063E070E0C50137
:10BB10007CDE60E473E026DE5C0181E0F501818378
:10BB200041E050E060E073E0C5010E94A74721EFCB
:10BB3000E22E25E1F22E2AE031E04DEA51E063E009
:10BB400070E0C50162DE0F900F900F90DF91CF91F2
:10BB50001F910F91FF90EF90DF90CF90BF90AF902B
:10BB60000895E3E6F7E01082118212821382EFE576
:10BB7000F7E01082118290E892831382EBE5F7E000
:10BB8000108291838FEF82831382E7E5F7E0908341
:10BB900081838283138208958F929F92AF92BF9286
:10BBA000CF92DF92EF92FF920F931F93CF93DF9389
:10BBB000CDB7DEB7C459D1090FB6F894DEBF0FBEBA
:10BBC000CDBF182F6B015A017901C9010E946D5335
:10BBD000082F1A318CF10023A1F0812F0E944953C4
:10BBE000BC01C7010E9441544C01812F0E9449535E
:10BBF0009A838983CE0101960E945553E82FF0E085
:10BC000013C0612FCE0101960E9445464FEF5FE7BA
:10BC1000B701CE0101960E9441454C01C357DF4F49
:10BC2000E881F981CD58D0408C149D041CF4EA15AC
:10BC3000FB0514F01150CDCF812FCC56DF4F0FB63E
:10BC4000F894DEBF0FBECDBFDF91CF911F910F9152
:10BC5000FF90EF90DF90CF90BF90AF909F908F902C
:10BC60000895CF93DF93EC010E94264C8AE18883EC
:10BC700019821A82DF91CF9108952F923F924F92AD
:10BC80005F926F927F928F929F92AF92BF92CF926C
:10BC9000DF92EF92FF920F931F93CF93DF93CDB775
:10BCA000DEB728970FB6F894DEBF0FBECDBF3C01BC
:10BCB0009B01542EDC0119969C91941709F4A9C09C
:10BCC000EFEFE90FE33048F4F0E0EE0FFF1FE2582A
:10BCD000FC4F0190F081E02D02C0E4EAF3E04FEF69
:10BCE000450D433048F450E0440F551F48585C4F11
:10BCF000DA010D911C9102C004EA13E0D8011C96F0
:10BD00004D915D916D917C911F97C484D584E6849B
:10BD1000F78481E0C416D506E606F70651F495309F
:10BD200021F4B5E05B1205C003C0A5E0CA2E5C108B
:10BD300080E0C480D580E680F780C982DA82EB8219
:10BD4000FC82D8011496CD90DD90ED90FC90179771
:10BD5000CD82DE82EF82F88680849184A284B384CF
:10BD60001896CD90DD90ED90FC901B9722242394A3
:10BD70008C149D04AE04BF0419F4943009F0212CF6
:10BD8000352C790163014080518062807380F80115
:10BD900080809180A280B380882359F0F5E03F1223
:10BDA00004C043E655E461E270E07460C7010E949C
:10BDB000A74729813A814B815C818D819E81AF812A
:10BDC000B885281739074A075B0751F0D801149640
:10BDD0004D915D916D917C911797C7010E94234809
:10BDE000222041F0F8014085518562857385C701A5
:10BDF0000E94F047481459046A047B0441F0D801BA
:10BE00004D915D916D917C91C7010E94BD47F601F6
:10BE1000318628960FB6F894DEBF0FBECDBFDF91F6
:10BE2000CF911F910F91FF90EF90DF90CF90BF9037
:10BE3000AF909F908F907F906F905F904F903F90CA
:10BE40002F900895FC01668320916A0A211104C095
:10BE50004D50461B40936A0A0895CF93DF9300D05C
:10BE6000CDB7DEB710926A0A0E941D9BCE010196E3
:10BE7000F8DE8EE390E590931902809318020F90FC
:10BE80000F900F90DF91CF910895813041F058F0DD
:10BE900090E1980F963038F480936A0A16C082E5D4
:10BEA00097E0F0DB12C04091520792E1499FA00158
:10BEB00011244F505F4B052E000C660B770B6BBFA8
:10BEC000FA0147915691FA01199481E00895E091A1
:10BED0006A0AE05FE63058F484E0E89FF00111243C
:10BEE000E05AFC4F6081718182819381089560E006
:10BEF00070E0CB0108952F923F924F925F926F9224
:10BF00007F928F929F92AF92BF92CF92DF92EF92E9
:10BF1000FF920F931F93CF93DF9300D01F92CDB763
:10BF2000DEB72C013B01942E3A8329831C830B83BB
:10BF3000170186017501DA8CFC018081811003C034
:10BF4000F82FF1708F2E80FD0BC0892D0E94069B6B
:10BF5000811106C0D11004C081101FC043E003C08E
:10BF60008820E1F34D2DB301C20187DE882011F056
:10BF7000492D01C040E0F301418350E060E070E0F2
:10BF80007360C3010E94A747C12CD12C91014B8142
:10BF90005C8169817A81C30138DC0F900F900F902A
:10BFA0000F90DF91CF911F910F91FF90EF90DF9055
:10BFB000CF90BF90AF909F908F907F906F905F9049
:10BFC0004F903F902F9008956F927F928F929F9203
:10BFD000AF92BF92CF92DF92EF92FF920F931F9397
:10BFE000CF93DF9300D01F92CDB7DEB73C01FC01A9
:10BFF0006083CE0101966C8334DE6C8160FF41C0AA
:10C000004FEF5FEF6FEF72E0CE0101960E94A747FE
:10C0100047E050E060E076E2CE0101960E94A7473B
:10C020004FEF5FEF6FEF74E0CE0101960E94A747DC
:10C030004FEF5FEF6FEF70E0CE0101960E94234853
:10C0400043E655E461E270E0CE0101960E94F047BC
:10C0500042ED59EA69E770E0CE0101960E94BD47C2
:10C0600043E655E461E274E0CE0101960E94A747E1
:10C070001A8240E050E060E073E0CE0101960E9439
:10C08000A7478BE18983992493949F928824839472
:10C090008DE2A82E86E1B82E9AE2C92ED12C2AE094
:10C0A000E22EFF24F39403EB11E023E030E041E0C3
:10C0B000BE016F5F7F4FC3011EDFF301918283E1F9
:10C0C00096E1908787830F900F900F900F900F90BD
:10C0D000DF91CF911F910F91FF90EF90DF90CF9064
:10C0E000BF90AF909F908F907F906F9008958F92A8
:10C0F000AF92BF92CF92DF92EF92FF920F931F9376
:10C10000CF93DF93FC01EB01422F80916A0A8111EA
:10C1100002C020936A0A9681423FA9F040F4403F52
:10C1200071F0413FB9F492502AE036E116C0433F26
:10C1300071F0443F79F49F5F21E036E10EC09350E7
:10C140002EE036E10AC0915026E036E106C024E038
:10C1500036E103C09E5F2DEF35E1808181FF04C091
:10C1600011E080916A0A841310E0913009F446C00E
:10C1700020F1923009F066C0618170E06150710970
:10C18000A0EEB1E06A9FC0016B9F900D7A9F900D69
:10C1900011246AE070E00F94EE9B6D5F7F4F1F9358
:10C1A0008824839459018AE2C82ED12C92E2E92E88
:10C1B000F12C8B0124EA30E041C0618170E06150D4
:10C1C0007109A0EEB1E06A9FC0016B9F900D7A9F4C
:10C1D000900D11246AE070E00F94EE9B6D5F7F4F2D
:10C1E0001F938824839459015AE2C52ED12CA2E2D0
:10C1F000EA2EF12C8B0123E530E020C0618170E054
:10C2000061507109A0EEB1E06A9FC0016B9F900D73
:10C210007A9F900D11246AE070E00F94EE9B6D5FA1
:10C220007F4F1F938824839459012AE2C22ED12C78
:10C2300032E2E32EF12C8B012BE730E0BE01CF017F
:10C240005ADE0F90DF91CF911F910F91FF90EF90E9
:10C25000DF90CF90BF90AF908F9008956F927F92B4
:10C260008F929F92AF92BF92CF92DF92EF92FF9206
:10C270000F931F93CF93DF9300D0CDB7DEB73C0170
:10C28000962E5A01822ECE010196EBDC8AE189833B
:10C29000D3011196EC91F0E0319720EE31E0E29F6E
:10C2A000C001E39F900DF29F900D11246AE070E0B1
:10C2B0000F94EE9B8B010D5F1F4F1F928AE2C82ED9
:10C2C000D12C9FEAE92EF12C23E530E0492DBE0167
:10C2D0006F5F7F4FC3010FDEF30181818F5F818329
:10C2E0000F900F900F900F90DF91CF911F910F91B2
:10C2F000FF90EF90DF90CF90BF90AF909F908F9086
:10C300007F906F9008956F927F928F929F92AF92DD
:10C31000BF92CF92DF92EF92FF920F931F93CF9332
:10C32000DF934C01C90137017601D1FE06C0E90156
:10C3300037FD2196D595C79506C0D3FE02C0E90109
:10C3400002C0C0E0D0E0C60FD71F5801F2FE07C000
:10C3500017FF03C02FEFA21AB20AB594A794A40E38
:10C36000B51EF5FE03C0F401108107C09301A801BA
:10C37000BC01F401808110DC182FC3010E946D53B1
:10C38000882359F0812F0E9449538C019301A50104
:10C39000BE01C4010E94E5540DC0212F110F330BC3
:10C3A0008701A501BE01C4010E948E48B301C401EA
:10C3B0000E94404EC401DF91CF911F910F91FF90D9
:10C3C000EF90DF90CF90BF90AF909F908F907F9035
:10C3D0006F9008958F929F92AF92BF92CF92DF920B
:10C3E000EF92FF920F931F93CF93DF9300D0CDB7BF
:10C3F000DEB75C017B01FC01808180FF37C0CE018C
:10C4000001962FDC45E0BE016F5F7F4FC50135DC33
:10C41000F501218130E02150310940EE51E0249FA7
:10C42000C001259F900D349F900D11246AE070E0AB
:10C430000F94EE9B4B01F3E08F0E911C8BE18983EF
:10C440001A8240E050E060E073E0CE0101960E9465
:10C45000A747C12C86E0D82E0AE210E025EF30E095
:10C46000A40163E070E0CE0101964DDFF50181810A
:10C470008F5F81830F900F900F90DF91CF911F916D
:10C480000F91FF90EF90DF90CF90BF90AF909F9073
:10C490008F9008958F929F92AF92BF92CF92DF922A
:10C4A000EF92FF920F931F93CF93DF9300D0CDB7FE
:10C4B000DEB75C01CE010196D4DB8AE18983F50108
:10C4C000808180FF36C045E0BE016F5F7F4FC501B0
:10C4D000D4DBF501218130E02150310940EE51E0FB
:10C4E000249FC001259F900D349F900D11246AE078
:10C4F00070E00F94EE9B4B01F3E08F0E911C1A82BB
:10C5000040E050E060E073E0CE0101960E94A74752
:10C51000C12C86E0D82E94E1E92E96E1F92E0AE2AC
:10C5200010E02AE430E0A40163E070E0CE0101965F
:10C53000EADEF501868125EF281B41814F5FBE01B0
:10C540006F5F7F4FC501D3DDF501868124EF281B86
:10C5500041814F5FBE016F5F7F4FC501C8DDF501AF
:10C56000868123EF281B41814F5FBE016F5F7F4FA4
:10C57000C501BDDDF50181818F5F81830F900F9033
:10C580000F90DF91CF911F910F91FF90EF90DF906F
:10C59000CF90BF90AF909F908F9008952F923F9231
:10C5A0004F925F926F927F928F929F92AF92BF92C3
:10C5B000CF92DF92EF92FF920F931F93CF93DF936F
:10C5C00000D0CDB7DEB73C01962ECE01019649DBF7
:10C5D000F301808180FF2DC045E0BE016F5F7F4F7A
:10C5E000C3014BDBF301218130E02150310940EEE2
:10C5F00051E0249FC001259F900D349F900D112480
:10C600006AE070E00F94EE9BAB014D5F5F4F8AE1F3
:10C610008983C12CA6E0DA2EBEE1EB2EB6E1FB2E1B
:10C620000AE210E02AE430E063E070E0CE01019617
:10C630006ADE8AE18983F301218130E021503109EA
:10C6400080EE282E33243394229DC001239D900D2B
:10C65000329D900D11242AE0422E512CB2010F94EC
:10C66000EE9B8B010D5F1F4F1F92882483943BE24A
:10C67000A32E36E1B32E4AE2C42ED12C52E2E52E8F
:10C68000F12C23E530E0492DBE016F5F7F4FC301E0
:10C6900032DCF301218130E021503109229DC001BB
:10C6A000239D900D329D900D1124B2010F94EE9BAD
:10C6B0008B010D5F1F4F41E0490D1F9269E2A62ECD
:10C6C00066E1B62E2BE730E0BE016F5F7F4FC301FE
:10C6D00012DCF301218130E021503109229DC0019B
:10C6E000239D900D329D900D1124B2010F94EE9B6D
:10C6F0008B010D5F1F4F42E0490D1F9277E2A72E7D
:10C7000076E1B72E24EA30E0BE016F5F7F4FC301B0
:10C71000F2DBF301218130E021503109229DC0017B
:10C72000239D900D329D900D1124B2010F94EE9B2C
:10C730008B010D5F1F4F43E0490D1F92E3E2AE2EC8
:10C74000E6E1BE2EF6E3EF2EF12C2CEC30E0BE013C
:10C750006F5F7F4FC301CFDBF30181818F5F8183E7
:10C760000F900F900F900F900F900F900F90DF9100
:10C77000CF911F910F91FF90EF90DF90CF90BF90DE
:10C78000AF909F908F907F906F905F904F903F9071
:10C790002F9008952F923F924F925F926F927F92C7
:10C7A0008F929F92AF92BF92CF92DF92EF92FF92C1
:10C7B0000F931F93CF93DF93CDB7DEB7C659D1093F
:10C7C0000FB6F894DEBF0FBECDBF5C013901470143
:10C7D0007601D1FE09C0290137FF03C08FEF481A47
:10C7E000580A5594479406C0D3FE02C0290102C0DE
:10C7F000412C512C460E571E6801F2FE07C017FF50
:10C8000003C0EFEFCE1ADE0AD594C794C40ED51E2E
:10C81000F5013080F5FC4CC0C4010E946253282E03
:10C82000F9E1F3150CF044C0222039F1832D0E9468
:10C830004953BC01C4010E9433549C01832DCB5643
:10C84000DF4F2883C559D040CA56DF4F3883C659B9
:10C85000D0400E9449539A838983CE0101960E9459
:10C86000555390E0CB56DF4F2881C559D040CA566A
:10C87000DF4F3881C659D04013C0632DCE010196D9
:10C880000E9445464FEF5FE7B401CE0101960E943A
:10C8900023459C01C357DF4F88819981CD58D040F3
:10C8A000261537051CF48017910714F03A94B8CF79
:10C8B000C4010E946253882359F0832D0E9449537A
:10C8C0008C019401A601B201C5010E9478540DC0EB
:10C8D000232D330C330B8701A601B201C5010E9441
:10C8E0008E48B401C5010E94554CC501CA56DF4FA0
:10C8F0000FB6F894DEBF0FBECDBFDF91CF911F9171
:10C900000F91FF90EF90DF90CF90BF90AF909F90EE
:10C910008F907F906F905F904F903F902F900895F1
:10C920002F923F924F925F926F927F928F929F923F
:10C93000AF92BF92CF92DF92EF92FF920F931F932D
:10C94000CF93DF9300D000D0CDB7DEB73C016C832E
:10C950007A013E832D83902ECE01019682D9F30178
:10C96000808180FF6AC045E0BE016F5F7F4FC301D9
:10C9700084D9F301218130E02150310970EEA72ED6
:10C98000BB24B3942A9DC0012B9D900D3A9D900D20
:10C990001124EAE02E2E312CB1010F94EE9B2B01D5
:10C9A000F3E04F0E511C1A8240E050E060E073E06B
:10C9B000CE0101960E94A7478AE18983C12CF6E047
:10C9C000DF2E0AE210E02AE430E0A20163E070E02A
:10C9D000CE01019698DC44E0BE016F5F7F4FC3013A
:10C9E0004CD9F301218130E0215031092A9DC00149
:10C9F0002B9D900D3A9D900D1124B1010F94EE9B4B
:10CA00005B01F3E0AF0EB11CF301428153816481FD
:10CA10007581CE0101960E94F047C12CDD24D3948C
:10CA2000BCEFEB2EB5E1FB2E2EE530E0A50163E572
:10CA300070E0CE0101960E94055C8BE18983F301D1
:10CA4000218130E02150310990EE292E3324339496
:10CA5000229DC001239D900D329D900D11242AE04E
:10CA6000422E512CB2010F94EE9B8B010D5F1F4F94
:10CA70001F92892C3AEFA32E35E1B32E4AE2C42E41
:10CA8000D12C52E2E52EF12C28EB30E04C81BE0196
:10CA90006F5F7F4FC3012FDAF301218130E0215016
:10CAA0003109229DC001239D900D329D900D1124CE
:10CAB000B2010F94EE9B8B010D5F1F4F4C814F5FB6
:10CAC0001F9268EFA62E65E1B62E20EE30E0BE0183
:10CAD0006F5F7F4FC3010FDAF30180810F900F90DA
:10CAE00081FF35C0992099F140E0BE016F5F7F4F13
:10CAF000C301C3D8F301218130E021503109229DC7
:10CB0000C001239D900D329D900D1124B2010F9410
:10CB1000EE9B5B01F3E0AF0EB11C1A8240E050E0E7
:10CB200060E073E0CE0101960E94A7478AE1898305
:10CB3000C12C86E0D82EED80FE800AE210E02EE5C2
:10CB400030E0A50163E570E0CE01019623DEF3013C
:10CB500081818F5F818326960FB6F894DEBF0FBE6A
:10CB6000CDBFDF91CF911F910F91FF90EF90DF909C
:10CB7000CF90BF90AF909F908F907F906F905F907D
:10CB80004F903F902F9008954F925F926F927F92B7
:10CB9000AF92BF92CF92DF92EF92FF920F931F93CB
:10CBA000CF93DF93CDB7DEB7A0970FB6F894DEBF73
:10CBB0000FBECDBF6C01F62E5A0128013901FC01D0
:10CBC000808180FF05C001E020E030E0C601A8DEE2
:10CBD000F601808181FF1CC08E010F5F1F4F2681EF
:10CBE00045E0C301B2010F947A9C66EF75E1C8017C
:10CBF0000F94D3A0F60167817085C8010F94D3A06C
:10CC00000E2D9E012F5F3F4FA5016F2DC60188DEBF
:10CC1000A0960FB6F894DEBF0FBECDBFDF91CF91C7
:10CC20001F910F91FF90EF90DF90CF90BF90AF904A
:10CC30007F906F905F904F900895E3E7F7E0108248
:10CC4000118212821382EFE6F7E01082118290E8DF
:10CC500092831382EBE6F7E0108291838FEF828359
:10CC60001382E7E6F7E0908381838283138208953D
:10CC70008F929F92AF92BF92CF92DF92EF92FF92EC
:10CC80000F931F93CF93DF93CDB7DEB7C459D1096C
:10CC90000FB6F894DEBF0FBECDBF182F6B015A013F
:10CCA0007901C9010E946D53082F1A318CF10023BC
:10CCB000A1F0812F0E944953BC01C7010E94415439
:10CCC0004C01812F0E9449539A838983CE0101969A
:10CCD0000E945553E82FF0E013C0612FCE0101965A
:10CCE0000E9445464FEF5FE7B701CE0101960E94D3
:10CCF00041454C01C357DF4FE881F981CD58D04001
:10CD00008C149D041CF4EA15FB0514F01150CDCFD2
:10CD1000812FCC56DF4F0FB6F894DEBF0FBECDBFCC
:10CD2000DF91CF911F910F91FF90EF90DF90CF9007
:10CD3000BF90AF909F908F900895CF93DF9300D0D6
:10CD4000CDB7DEB7CE0101960E94264C8AE18983D9
:10CD50001A821B8240E05FEF6FEF7FEFCE010196FA
:10CD60000E94A747CE0101960E94F453809152077A
:10CD700022E1829FC001112483519F4B092E000C98
:10CD8000AA0BBB0BABBFFC012791369183E0F901E5
:10CD9000199540E050E0BA01CE0101960E94A747E4
:10CDA00041E05FEF6FEF7FEFCE0101960E94A74752
:10CDB000CE0101960E94274C0F900F900F90DF91AB
:10CDC000CF9108950E941D9B81E00C9425FC80E08A
:10CDD0000C9425FC813031F482E597E00E94425B9F
:10CDE00081E0089580E0089562E082E79AE00E9481
:10CDF0009158882339F0A1DF82E79AE00E94B05869
:10CE00000E94129B0C948A9BAF92BF92CF92DF92AA
:10CE1000EF92FF920F931F93CF93DF9300D0CDB784
:10CE2000DEB7CE0101960E94264C8AE189831A82E0
:10CE30001B824FEF5FEF6FEF72E0CE0101960E9411
:10CE4000A74743E655E461E274E0CE0101960E94F3
:10CE5000A74747E050E060E076E2CE0101960E94ED
:10CE6000A7471A8240E050E060E073E0CE010196EF
:10CE70000E94A7478CE1898320E736E14EE350E02A
:10CE80006AE071E0F5DE182F80E796E10E946D53AD
:10CE9000882391F0812F0E944953E12C16E0F12E56
:10CEA0008C0120E736E142E250E068E870E0CE0114
:10CEB00001960E94E55413C0212F110F330B00E09F
:10CEC00016E042E250E068E870E0CE0101960E9470
:10CED0008E4860E776E1CE0101960E94404E8AE1DD
:10CEE00089834C9B03C064EC73E002C064ED73E083
:10CEF0008B818F778B83CE0101960E94B25BC12C10
:10CF0000D12CBAE6EB2EB6E1FB2E0EE310E024E5C1
:10CF100030E047E450E063E070E00E94055C8091FF
:10CF2000060187FF03C064ED73E002C064EC73E0A8
:10CF30008B818F778B83CE0101960E94B25BC12CCF
:10CF4000D12CAEE5EA2EA6E1FA2E0EE310E024E5A0
:10CF500030E047E450E06DE570E00E94055C8091B0
:10CF6000000184FD03C064ED73E002C064EC73E073
:10CF70008B818F778B83CE0101960E94B25BC12C8F
:10CF8000D12CF2E5EF2EF6E1FF2E0EE310E024E5C2
:10CF900030E047E450E068EB70E00E94055C80916F
:10CFA000060182FF03C064ED73E002C064EC73E02D
:10CFB0008B818F778B83CE0101960E94B25BC12C4F
:10CFC000D12C74E6E72E76E1F72E0EE310E024E58F
:10CFD00030E04CE850E063E070E00E94055C8B813B
:10CFE00080688B83E8E5EE2EE6E1FE2E24E530E056
:10CFF0004CE850E06DE570E0CE0101960E94055CC2
:10D000001C9B03C064ED73E002C064EC73E08B8191
:10D010008F778B83CE0101960E94B25BC12CD12CFD
:10D020002CE4E22E26E1F22E0EE310E024E530E0BF
:10D030004CE850E068EB70E00E94055C8B818068F2
:10D040008B833BE3E32E36E1F32E24E530E040ED25
:10D0500050E063E070E0CE0101960E94055C8B8198
:10D0600080688B8342E3E42E46E1F42E24E530E031
:10D0700040ED50E06DE570E0CE0101960E94055C48
:10D080008B8180688B8354E4E52E56E1F52E24E5F0
:10D0900030E040ED50E068EB70E0CE0101960E9478
:10D0A000055C8BE1898364EC73E0CE0101960E94FC
:10D0B000B25B5C0181E0F501818341E050E060E01A
:10D0C00073E0C5010E94A74769E7E62E66E1F62EE8
:10D0D0002AE031E04EE951E063E070E0C5010E94D2
:10D0E000055C0F900F900F90DF91CF911F910F91E2
:10D0F000FF90EF90DF90CF90BF90AF900895E3E85E
:10D10000F7E01082118212821382EFE7F7E01082BB
:10D11000118290E892831382EBE7F7E0108291830B
:10D120008FEF82831382E7E7F7E090838183828326
:10D1300013820895EF920F931F93CF93DF93CDB790
:10D14000DEB72A970FB6F894DEBF0FBECDBF682FAB
:10D15000CE0101960E94E45F42E060E0CE010196BC
:10D160000E94225F8EE796E19987888769E876E1D9
:10D17000CE0101962FD980E00E9444DD8B019C01F5
:10D1800080E090E0AFEFB0E08B839C83AD83BE8303
:10D19000EE24E39447E856E162E0CE010196F4DC28
:10D1A00081E00E9444DD8B019C0180E09BEBA0E0CC
:10D1B000B0E08B839C83AD83BE8345E856E164E099
:10D1C000CE010196E1DC82E00E9444DD8B019C01EE
:10D1D0008FEB90E0A0E0B0E08B839C83AD83BE83B7
:10D1E00043E856E166E0CE010196CEDC80E00E9485
:10D1F00066DD8B019C0181E794E6A6E5B0E08B83B8
:10D200009C83AD83BE8341E856E168E0CE01019680
:10D21000BBDCCE0101963ED92A960FB6F894DEBF4C
:10D220000FBECDBFDF91CF911F910F91EF90089569
:10D230001F93CF93DF9300D01F92CDB7DEB7182F87
:10D240000E94675F9B01AC01812F90E0FC01329747
:10D25000E830F10508F081C08827EA56FF4F8F4F6C
:10D260000D94539C80E029833A834B835C830E9416
:10D2700044DD29813A814B815C810F94BC970DC0BC
:10D2800080E029833A834B835C830E9444DD2981BB
:10D290003A814B815C810F94BD9740E00E9475DD1F
:10D2A00058C081E029833A834B835C830E9444DD2C
:10D2B00029813A814B815C810F94BC970DC081E03C
:10D2C00029833A834B835C830E9444DD29813A8120
:10D2D0004B815C810F94BD9741E0E0CF82E02983D0
:10D2E0003A834B835C830E9444DD29813A814B81E0
:10D2F0005C810F94BC970DC082E029833A834B83F5
:10D300005C830E9444DD29813A814B815C810F94CA
:10D31000BD9742E0C3CF80E029833A834B835C838F
:10D320000E9466DD29813A814B815C810F94BC9714
:10D330000DC080E029833A834B835C830E9466DDC5
:10D3400029813A814B815C810F94BD9740E00E9416
:10D35000F5DD81E08093C90901C080E00F900F9056
:10D360000F900F90DF91CF911F910895E3E9F7E0BF
:10D370001082118212821382EFE8F7E0108211828C
:10D3800090E892831382EBE8F7E0108291838FEFAD
:10D3900082831382E7E8F7E090838183828313829C
:10D3A0000895CF92DF92EF92FF92CF93DF93DC014B
:10D3B0002D913C9111972115310509F468C01496FF
:10D3C0008D919C9115971696CD91DC911797281702
:10D3D0003907B1F4CF3F2FEFD20779F01B96DC93DA
:10D3E000CE931A9718968D919C9119971D969C93A0
:10D3F0008E931C978FEF9FEF26C01D921C9247C003
:10D40000A9014E5F5F4F11965C934E936901032E05
:10D41000000CEE08FF08EBBEF601879196911B9673
:10D420009C938E931A978F3F6FEF9607A9F41B96E4
:10D43000DC93CE931A9718962D913C9119971D96CF
:10D440003C932E931C9717969C938E931697199640
:10D450009C938E9318971BC02C5F3F4F11963C9363
:10D460002E93052E000C660B770B6BBFFA014791CC
:10D4700056911D965C934E931C97219641F41796F6
:10D480009C938E93169719965C934E931897DF9101
:10D49000CF91FF90EF90DF90CF900895CF92DF92E1
:10D4A000EF92FF920F931F93CF93DF93FC01C285FE
:10D4B000D38544855585A685B785008911899E0148
:10D4C0000F946A9C6B017C019A01D8010F946A9CAD
:10D4D000DC01CB018C0D9D1DAE1DBF1DCD01BB27F9
:10D4E00097FDB095AB2F02891389012E000C220BFA
:10D4F000330B800F911FA21FB31F4096A11DB11DBA
:10D5000035E0B595A795979587953A95D1F7938F7F
:10D51000828FA489B589068917899E010F946A9C18
:10D520006B017C019A01D8010F946A9CDC01CB014C
:10D530008C0D9D1DAE1DBF1DCD01BB2797FDB09568
:10D54000AB2F408D518D052E000C660B770B840F91
:10D55000951FA61FB71F4096A11DB11D55E0B5959B
:10D56000A795979587955A95D1F7958F848FDF91D9
:10D57000CF911F910F91FF90EF90DF90CF90089582
:10D58000CF93DF9300D0CDB7DEB7CE0101960E94D6
:10D59000264C8AE189831A821B8240E050E060E0D9
:10D5A00072E0CE0101960E94A74747E050E060E09C
:10D5B00076E2CE0101960E94A7470E94E8468FEFCF
:10D5C0000E94E2510F900F900F90DF91CF9108953C
:10D5D000CF93DF93EC017B836A83440F551F460F83
:10D5E000571F5D834C83798368838FEF9FEF9F8301
:10D5F0008E83CE01D6DE80E092E29F878E87198AE5
:10D60000188A1B8A1A8A1D8A1C8A80E09CE39F8BD9
:10D610008E8B198E188ECE0141DF8A8D9B8D9F8F48
:10D620008E8F8C8D9D8D99A388A3DF91CF910895C6
:10D63000CF93DF93EC0188819981892B39F1CE0159
:10D64000B0DECE012BDF2A8D3B8D4E8D5F8D8E811E
:10D650009F812417350759F46C8D7D8D48A159A100
:10D660006417750721F48F3F4FEF940721F78F3F21
:10D670004FEF940729F499A388A39F8F8E8F06C03C
:10D680003F8F2E8F8C8D9D8D99A388A3DF91CF9195
:10D6900008956F927F928F929F92BF92CF92DF9266
:10D6A000EF92FF920F931F93CF93DF93CDB7DEB727
:10D6B000A2970FB6F894DEBF0FBECDBF7C01669671
:10D6C000BFAC6697BB2009F47BC082E2FE01F396F3
:10D6D000DE01119601900D928A95E1F78B819C8174
:10D6E0009A8389838FEF9FEF98878F83CE0101966E
:10D6F00058DEC12CA0E8DA2E00E010E866246A9417
:10D70000BFE77B2E88248A948FE7982E89819A819F
:10D71000892BC1F08B8D9C8D881599050CF44C01DB
:10D72000081719070CF48C018D8D9E8D86159705B1
:10D730000CF43C01C816D9060CF46C01CE0101961C
:10D7400077DFE4CF08191909C618D70840E050E080
:10D7500060E072E2F701808191810E94A747A301F6
:10D76000577060E070E07B61C4019770A0E0B0E0AA
:10D77000EBE0880F991FAA1FBB1FEA95D1F7482B32
:10D78000592B6A2B7B2BF701808191810E94A7473F
:10D79000A6015F7060E070E07C611F7020E030E007
:10D7A000FCE0000F111F221F331FFA95D1F7402B09
:10D7B000512B622B732BF701808191810E94A74727
:10D7C000F7010081118140E050E060E072E2C801A1
:10D7D0000E94A74740E050E060E074E1C8010E9469
:10D7E000A74742E050E060E076E2C8010E94A74708
:10D7F00040E050E060E070E2C8010E94A7474DE0C1
:10D8000050E060E07CE0C8010E94A7474FEF5FEF67
:10D8100067E07AE0C8010E94A74748E050E060E076
:10D820007FE1C8010E94A7478DA99EA99CAB8BAB45
:10D830008FEF9FEF9AAF89AFCE01C396B2DD8BA970
:10D840009CA9892BB1F161964EAD5FAD619784E0E3
:10D85000440F551F8A95E1F75F7760E070E07064D0
:10D860002F968EAD9FAD2F9724E0880F991F2A9594
:10D87000E1F79F77A0E0B0E03FE0880F991FAA1F73
:10D88000BB1F3A95D1F7482B592B6A2B7B2BC8012C
:10D890000E94A74789AD9AAD019639F448E050E05F
:10D8A00060E07FE1C8010E94A747CE01C396C0DEB9
:10D8B000C6CF40E050E060E073E2C8010E94A74795
:10D8C00040E050E060E072E2C8010E94A7474FEFDD
:10D8D00050E066E07AE0C8010E94A74749E050E0C6
:10D8E00060E07FE1C8010E94A74740E050E060E0AF
:10D8F00070E4C8010E94A74740E05EE160E878E478
:10D90000C8010E94A74740E050E060E073E2C80110
:10D910000E94A747BB2049F040E050E060E073E27E
:10D92000F701808191810E94A747A2960FB6F894D3
:10D93000DEBF0FBECDBFDF91CF911F910F91FF9042
:10D94000EF90DF90CF90BF909F908F907F906F90DF
:10D950000895FF920F931F93CF93DF93CDB7DEB758
:10D96000E6970FB6F894DEBF0FBECDBF8E010C5CFC
:10D970001F4FC8010E94264C8AE18CAB1DAA1EAA2B
:10D9800040E05FEF6FEF7FEFC8010E94A7474FEFC6
:10D990005FEF6FEF72E0C8010E94A74747E050E0D9
:10D9A00060E076E2C8010E94A7471CA30BA31DA25A
:10D9B0001EA21FA218A680EE90EEA3EFB0E089A7EA
:10D9C0009AA7ABA7BCA785E08DA71EA61FA618AA7D
:10D9D00019AA8CE18AAB83E08BAB4FEF5FEF6FEF5F
:10D9E00074E0C8010E94A74746E050E06BE07FE288
:10D9F000CE010196EDDDFF24F394FF928DB79EB723
:10DA000082970FB6F8949EBF0FBE8DBFADB7BEB75D
:10DA1000119682E2FE01319601900D928A95E1F70E
:10DA2000CE01839636DE0FB6F894DEBF0FBECDBFB3
:10DA300047EC5AE660E074E0C8010E94A74749E657
:10DA400055E065E970E2CE010196C2DDFF928DB727
:10DA50009EB782970FB6F8949EBF0FBE8DBFADB72D
:10DA6000BEB7119682E2FE01319601900D928A9521
:10DA7000E1F7CE0183960DDE0FB6F894DEBF0FBE40
:10DA8000CDBF41E651E067E67BE2CE010196A0DD25
:10DA9000FF928DB79EB782970FB6F8949EBF0FBEC8
:10DAA0008DBFADB7BEB7119682E2FE0131960190EF
:10DAB0000D928A95E1F7CE018396EBDD0FB6F894CF
:10DAC000DEBF0FBECDBF41E750E069E27EE2CE018E
:10DAD00001967EDDFF928DB79EB782970FB6F894C0
:10DAE0009EBF0FBE8DBFADB7BEB7119682E2FE01DD
:10DAF000319601900D928A95E1F7CE018396C9DDAA
:10DB00000FB6F894DEBF0FBECDBF4FEF5FEF6FEFE4
:10DB100074E0C8010E94A7474AEF54E061EA76E149
:10DB2000CE01019655DDFF928DB79EB782970FB655
:10DB3000F8949EBF0FBE8DBFADB7BEB7119682E2FF
:10DB4000FE01319601900D928A95E1F7CE01839600
:10DB5000A0DD0FB6F894DEBF0FBECDBF40E050E0B1
:10DB6000BA01C8010E94A74741E05FEF6FEF7FEF66
:10DB7000C8010E94A747C8010E94274C64EC79E0C5
:10DB800080E090E00E94B8DAE6960FB6F894DEBF27
:10DB90000FBECDBFDF91CF911F910F91FF900895E0
:10DBA0006CE871E280E390E00E94044697FD11C0AA
:10DBB0000E94E3750E94A1A76FE670E882E597E0F6
:10DBC0000E94285B82E597E00E941B5B61ED74EB8D
:10DBD0002BC00E94D9D981110AC00E94A1A782E955
:10DBE00096E10E9404C30E94DBD90E9435C30E94C3
:10DBF0003E4F882329F00E944F8E811101C0A9DE7B
:10DC00000E94A1A767EF77E882E597E00E94285B72
:10DC100082E597E00E941B5B61ED74EB82E597E083
:10DC20000E94025B65E97EE882E597E00C94025B66
:10DC3000E3EAF7E01082118212821382EFE9F7E043
:10DC40001082118290E892831382EBE9F7E0108250
:10DC500091838FEF82831382E7E9F7E090838183DA
:10DC6000828313820895FC01862F408192E1499FAF
:10DC7000A001112443515F4B052E000C660B770B5E
:10DC80006BBFFA0147915691FA011994E82FF0E021
:10DC9000E955F84FE08184E0E89FF0011124E85055
:10DCA000FB4B859194910895CF93DF9340910F069C
:10DCB0002AEF34E490E0A82FB0E0A955B84F9417AC
:10DCC00059F0F901C591D4916C177D0709F49C9323
:10DCD0009F5F2C5F3F4FF3CFDF91CF910895462F89
:10DCE000E82FF0E0E955F84FE08184E0E89FF0018B
:10DCF0001124E650FB4B6591749189E497E00C94F4
:10DD0000B352482FE82FF0E0E955F84F208130E07A
:10DD1000C901019660910F0670E00F94029C808308
:10DD200060E0842FDCCF64ED78E480E0BDDF64EB5D
:10DD300078E481E0B9DF64EE78E482E0B5CF0E9458
:10DD4000E95180936A0A0C941D9B8430C1F058F409
:10DD5000813079F08330D9F40E94304F91E08927E7
:10DD60000E94254F10C0853061F0863081F482E03A
:10DD700009C082E597E00E94425B81E0089580E05F
:10DD800001C081E0BEDF81E08093C909089580E091
:10DD900008954F925F926F927F928F929F92AF926F
:10DDA000BF92CF92DF92EF92FF920F931F93CF9388
:10DDB000DF93CDB7DEB7C759D1090FB6F894DEBFF0
:10DDC0000FBECDBF182FCE018B569F4F0E94315EE4
:10DDD000123009F069C0CB56DF4F6881C559D04079
:10DDE000CE0101960E944546C357DF4F6881798175
:10DDF0008A819B81CD58D0400F94369920E030E045
:10DE000040EA51E40F94199B20E030E040E85DE3E4
:10DE10000F94199B0F940A998B0116950795B801D9
:10DE200080E090E00F9436992B013C0120E030E037
:10DE300040EA50E40F94199B9B01AC0160E070E054
:10DE400086EE92E40F94BC970F9405994B015C0108
:10DE50008FE290E06C01C01AD10AD694C79488E38F
:10DE6000C80ED11C20E030E040E250E4C301B20112
:10DE70000F94199B20E030E048EF52E40F94BD97D7
:10DE80000F94059922E0E22EF12C9401A601CE0117
:10DE90008B569F4F0E94504B81E080934807CE01E4
:10DEA0008B569F4F0E94274C81E0C956DF4F0FB61B
:10DEB000F894DEBF0FBECDBFDF91CF911F910F91C0
:10DEC000FF90EF90DF90CF90BF90AF909F908F909A
:10DED0007F906F905F904F9008952F923F924F9256
:10DEE0005F926F927F928F929F92AF92BF92CF92EA
:10DEF000DF92EF92FF920F931F93CF93DF93CDB7F3
:10DF0000DEB7CA59D1090FB6F894DEBF0FBECDBF38
:10DF10005C011B01C856DF4F59834883C859D04064
:10DF2000490128013701CB56DF4FD982C882C55934
:10DF3000D040E0911802F0911902309789F000E08A
:10DF40009E012B563F4FAC014E5F5F4FDC01119697
:10DF50006C911995C656DF4F8883CA59D04005C0C9
:10DF6000C656DF4F1882CA59D040CB56DF4F888142
:10DF70009981C559D04095FF08C0F501F081C95677
:10DF8000DF4FF883C759D0403FC0D5011C91C30172
:10DF90000E946253F82E1A317CF1FF20A1F0812FEC
:10DFA0000E944953BC01C3010E9433546C01812F6C
:10DFB0000E9449539A838983CE0101960E9455534A
:10DFC000282F30E013C0612FCE0101960E944546F4
:10DFD0004FEF5FE7B301CE0101960E9423456C012C
:10DFE000C357DF4F28813981CD58D040C814D90498
:10DFF0004CF42415350534F4C956DF4F1883C7593E
:10E00000D04002C01150C7CFCB56DF4FC880D98057
:10E01000C559D040C956DF4FB881C759D040EB2E03
:10E02000BB0FFF0882019401C856DF4F4881598118
:10E03000C859D040B101C5010E945648C3010E9491
:10E040006253882309F461C067E17FE2C5010E9441
:10E05000404E97FE03C0EFEF8E1A9E0A9594879468
:10E06000280C391C57FE03C0FFEF4F1A5F0A559466
:10E070004794C856DF4F88819981C859D040480ECF
:10E08000591ECB56DF4F88819981C559D04090FDEC
:10E090002AC040E050E060E072E2C5010E94A7475C
:10E0A00040E050E060E074E0C5010E94A747C95617
:10E0B000DF4F8881C759D0400E944953E12C36E098
:10E0C000F32E8C019301A20141505109B10161501D
:10E0D0007109C5010E94785440E050E060E073E2AD
:10E0E000C5010E94A747C956DF4F8881C759D04054
:10E0F0000E944953E12C26E0F22E8C019301A201EB
:10E10000B101C5010E94785404C0B301C5010E9449
:10E11000554CE0911802F0911902309799F0C656CB
:10E12000DF4F9881CA59D040992361F001E09E01E8
:10E130002B563F4FA5014E5F5F4FD50111966C9155
:10E14000C5011995C501C656DF4F0FB6F894DEBF5D
:10E150000FBECDBFDF91CF911F910F91FF90EF9038
:10E16000DF90CF90BF90AF909F908F907F906F90F7
:10E170005F904F903F902F9008952F923F924F9233
:10E180005F926F927F928F929F92AF92BF92CF9247
:10E19000DF92EF92FF920F931F93CF93DF93CDB750
:10E1A000DEB7C55AD1090FB6F894DEBF0FBECDBF9A
:10E1B000782ECE0184569F4F0E94315E70FE8FC034
:10E1C0004FEF5FEF6FEF72E0CE0184569F4F0E94DA
:10E1D000A74747E050E060E076E2CE0184569F4FCB
:10E1E0000E94A74743E655E461E274E0CE018456FD
:10E1F0009F4F0E94A747C356DF4F1882CD59D0408A
:10E2000040E050E060E073E0CE0184569F4F0E94F2
:10E21000A7478BE1C456DF4F8883CC59D040C12C2F
:10E22000F6E0DF2EA5E2EA2EAFE2FA2E0FE210E0D2
:10E230002AE031E043E050E063E070E0CE01845634
:10E240009F4F0E9483614C018AE1F4018083118217
:10E2500040E050E060E073E0C4010E94A747C12C99
:10E26000BCE0DB2E86E3E82E8FE2F82E23E730E0D9
:10E2700048E350E063E070E0C4010E94836128E15C
:10E28000E22E2FE2F22E23E730E04DE650E063E08D
:10E2900070E00E9483613EE5E32E3FE2F32E23E728
:10E2A00030E048ED50E063E070E00E9483614FE4AD
:10E2B000E42E4FE2F42E23E730E04DE051E063E03E
:10E2C00070E00E94836153E4E52E5FE2F52E23E7C0
:10E2D00030E043E451E063E070E00E94836171FE4E
:10E2E00081C182E0D3DCC156DF4F99838883CF5947
:10E2F000D04081E0CBDCCF55DF4F99838883C15A72
:10E30000D04080E0C3DCCD55DF4F99838883C35A6A
:10E31000D0400E94304FCB55DF4F8883C55AD04044
:10E32000C0906A0AD12C8BE1C456DF4F8883CC5948
:10E33000D04066EF73E0CE0184569F4F0E94B25BDF
:10E340004C0182E0F401818342E050E060E073E040
:10E35000C4010E94A747F4016081CE0101960E948A
:10E360004546C357DF4F688179818A819B81CD58AB
:10E37000D0400F94369920E030E040EA51E40F9409
:10E38000199B20E030E040E85DE30F94199B0F9467
:10E390000A998B0116950795B801660F771F80E0E3
:10E3A00090E00F9436999B01AC0160E070E086EE3E
:10E3B00092E40F94BC970F9405991B012C016FE216
:10E3C000662E712C601A710A76946794F8E36F0ECA
:10E3D000711CB80180E090E00F94369920E030E0A5
:10E3E00048EF52E40F94BD970F940599AA24AA947C
:10E3F000B12CE12CF12C9101A301C4010E946A4AC5
:10E4000066EE73E0C4010E94B25B4C0183E0F4014C
:10E41000818343E050E060E073E0C4010E94A747BD
:10E4200062E77FE2CE018B569F4F0F94DEA064EE31
:10E4300073E0CE018B569F4F0F9458A165E77FE2A2
:10E44000CE018B569F4F0F94D3A0F4016081CE0173
:10E4500001960E944546C357DF4F488059806A8025
:10E460007B80CD58D040F4010081002E000C110BB0
:10E47000C301B2010F94369920E030E040EA51E444
:10E480000F94199B20E030E040E85DE30F94199B66
:10E490000F9405994FE250E0461B570B57FF02C0FF
:10E4A0004F5F5F4F55954795FA01E359FF4FA5E040
:10E4B000B0E0A30192010F94709CDC01CB0124E039
:10E4C000B695A795979587952A95D1F7AF01480FEF
:10E4D000591FCB55DF4FC880C55AD040E12CF12CD5
:10E4E00024E430E063E970E0C4010E94BA48BE0150
:10E4F0006B567F4FC4010E94554C0FB6F894DEBF97
:10E500000FBECDBF66E174E0C4010E94B25B4C0156
:10E5100084E0F401818344E050E060E073E0C401F2
:10E520000E94A747C12CD12CCD55DF4FE880F98040
:10E53000C35AD0400FE210E022E830E048ED50E04E
:10E540006BE870E0C401C9DC4C0185E0F401818313
:10E5500045E050E060E073E0C4010E94A747CF555A
:10E56000DF4FE880F980C15AD04022E830E04DE02A
:10E5700051E06BE870E0C401B0DC4C0186E0F401CE
:10E58000818346E050E060E073E0C4010E94A74749
:10E59000C156DF4FE880F980CF59D04022E830E003
:10E5A00043E451E06BE870E0C40197DC66E074E09E
:10E5B0000E94B25B4C0181E0F401818341E050E0B4
:10E5C00060E073E0C4010E94A7473DE6E32E3FE20E
:10E5D000F32E2AE031E04DEA51E063E070E0C4013F
:10E5E0000E94055CCB55DF4F0FB6F894DEBF0FBE1F
:10E5F000CDBFDF91CF911F910F91FF90EF90DF90F2
:10E60000CF90BF90AF909F908F907F906F905F90D2
:10E610004F903F902F900895CF93DF93CDB7DEB703
:10E620002A970FB6F894DEBF0FBECDBF89E189836C
:10E63000CE0101960E949351CE0108960E94315E50
:10E6400040E05FEF6FEF7FEFCE0108960E94A74793
:10E65000CE0101960E945250882329F0CE010196E6
:10E660000E94C1510FC0CE0108960E94F45361E090
:10E6700082E597E0F8DA40E050E0BA01CE01019679
:10E680000E94DE5062E082E597E0EDDA40E050E083
:10E69000BA01CE0108960E94A74741E05FEF6FEFF5
:10E6A0007FEFCE0108960E94A747CE0108960E94F0
:10E6B000274C2A960FB6F894DEBF0FBECDBFDF9170
:10E6C000CF910895EF92FF920F931F93CF93DF9313
:10E6D00000D0CDB7DEB761E082E79AE00E949158A2
:10E6E0008823D1F182E79AE00E94B058CE010196CA
:10E6F0000E94315E80914807882381F10E94474F34
:10E700008823A9F060E070E980E390E00E9404466D
:10E710008C0122273327623009F510936A0A812F72
:10E720000E94E25181E08093C90976DF15C0E12C97
:10E73000F12C00E010E020E030E040E050E060E04C
:10E7400070E0CE0101960E94504BCE0101960E94CE
:10E75000274C1092480702C00E948A9B0F900F908E
:10E760000F90DF91CF911F910F91FF90EF9008953F
:10E77000E6EBF7E01082118212821382E2EBF7E0FF
:10E780001082118290E892831382EEEAF7E0108201
:10E7900091838FEF82831382EAEAF7E0908381838B
:10E7A000828313820895CF93DF93CDB7DEB7C45928
:10E7B000D1090FB6F894DEBF0FBECDBF682FCE01D2
:10E7C00001960E944546C357DF4F688179818A814F
:10E7D0009B81CD58D0400F94369920E030E040EA3C
:10E7E00051E40F94199B20E030E040E85DE30F9482
:10E7F000199B0F940A99CB01CC56DF4F0FB6F894B2
:10E80000DEBF0FBECDBFDF91CF9108952F923F9213
:10E810004F925F926F927F928F929F92AF92CF9220
:10E82000DF92EF92FF920F931F93CF93DF93CDB7B9
:10E83000DEB7CC59D1090FB6F894DEBF0FBECDBFFD
:10E840003C01CB56DF4F79836883C559D0401A010C
:10E850002901C956DF4F99828882C759D0402DB708
:10E860003EB7C556DF4F39832883CB59D040C70107
:10E870000F94E5A04C01C6010F94E5A0880D991DE9
:10E880000296EDB7FEB7E81BF90B0FB6F894FEBF82
:10E890000FBEEDBF2DB73EB72F5F3F4F4901B70108
:10E8A000C9010F94DEA064EE73E0C4010F9458A177
:10E8B000B601C4010F94D3A0F3016081CE0101968B
:10E8C0000E944546C357DF4FC880D980EA80FB804D
:10E8D000CD58D040F3018081282F880F330BC756C5
:10E8E000DF4F39832883C959D040401A510AC701E4
:10E8F000B6010F94369920E030E040EA51E40F94DD
:10E90000199B20E030E040E85DE30F94199B0F94E1
:10E910000599A801461B570B57FF02C04F5F5F4F79
:10E9200055954795F101E40FF51FA5E0B0E0A7016B
:10E9300096010F94709CDC01CB0124E0B695A7955D
:10E94000979587952A95D1F7AF01480F591F17FF63
:10E9500002C00F5F1F4F15950795CB56DF4F68819B
:10E960007981C559D040600F711FCA2CC956DF4F3D
:10E97000E880F980C759D040C756DF4F0881198118
:10E98000C959D0409201C3010E94BA48B401C301E1
:10E990000E94554CC301C556DF4FE881F981CB5920
:10E9A000D0400FB6F894FEBF0FBEEDBFC456DF4F88
:10E9B0000FB6F894DEBF0FBECDBFDF91CF911F9190
:10E9C0000F91FF90EF90DF90CF90AF909F908F903E
:10E9D0007F906F905F904F903F902F900895089593
:10E9E000CF93DF930E94DA45CAE6DAE089830E947A
:10E9F000E9518883DF91CF910C941D9B843099F06D
:10EA000038F4813039F582E597E00E94425B1CC002
:10EA1000853099F08630F1F46DEB70E782E597E090
:10EA20000E94285B11C00E94EE82811103C00E94E7
:10EA3000FC820CC00E94F78209C00E943E4F91E008
:10EA400089270E94374F02C081E0089581E08093BA
:10EA5000C909089580E008954F925F926F927F9266
:10EA60008F929F92AF92BF92CF92DF92EF92FF92DE
:10EA70000F931F93CF93DF9300D0CDB7DEB7182F3E
:10EA8000CE0101960E94315E123009F43FC013306E
:10EA900009F084C0898187DE8C0116950795B8013D
:10EAA00080E090E00F9436992B013C0120E030E0AB
:10EAB00040EA50E40F94199B9B01AC0160E070E0C8
:10EAC00086EE92E40F94BC970F9405994B015C017C
:10EAD0008EE390E06C01C01AD10AD694C79480ED01
:10EAE000C80ED11C20E030E040E250E4C301B20186
:10EAF0000F94199B20E030E048EF52E40F94BD974B
:10EB00000F94059923E0E22EF12C3BC089814BDE66
:10EB10008C0116950795B80180E090E00F94369926
:10EB20002B013C0120E030E040EA50E40F94199BB7
:10EB30009B01AC0160E070E086EE92E40F94BC971C
:10EB40000F9405994B015C018EE390E06C01C01AB3
:10EB5000D10AD694C7948CE8C80ED11C20E030E0CE
:10EB600040E250E4C301B2010F94199B20E030E071
:10EB700048EF52E40F94BD970F94059952E0E52EAB
:10EB8000F12C9401A601CE0101960E94504B81E028
:10EB900080934807CE0101960E94274C81E00F9098
:10EBA0000F900F90DF91CF911F910F91FF90EF90F9
:10EBB000DF90CF90BF90AF909F908F907F906F909D
:10EBC0005F904F90089520E030E0A90168E570E281
:10EBD00080E390E00E940E470E949A4C0E94D64C1F
:10EBE0008FEF0E94DF460E94144F4CE250E060E33A
:10EBF00070E280E390E00E94EE464DE050E064E475
:10EC000070E280E390E00C94EE4610921B081092A4
:10EC10001A088FEF0E94E2518FEF0E94DF460E9498
:10EC2000144F81D84CE250E060E370E280E390E062
:10EC30000E94EE464DE050E064E470E280E390E034
:10EC40000C94EE462F923F924F925F926F927F927A
:10EC50008F929F92AF92BF92CF92DF92EF92FF92EC
:10EC60000F931F93CF93DF93CDB7DEB760970FB6A7
:10EC7000F894DEBF0FBECDBF988B8F8786E99FE2E9
:10EC80000E9452FC20911A0830911B082D873E8764
:10EC90000E94E951382E0E94DA45282E0E94194F11
:10ECA000082F60E571E280E390E00E9404466983EA
:10ECB0007A838B839C8364E571E280E390E00E9419
:10ECC00004462B013C0168E571E280E390E00E947C
:10ECD00004464B015C016CE571E280E390E00E9428
:10ECE00004466D837E838F83988760E671E280E3BC
:10ECF00090E00E94044669877A878B879C8764E648
:10ED000071E280E390E00E9404466B017C0160E3C5
:10ED100070E280E390E00E94DF45182F64E470E227
:10ED200080E390E00E94DF45E7EAF7E0A081B1814F
:10ED3000928149815A816B817C81EF85F88940837A
:10ED40005183628373834482558266827782808690
:10ED50009186A286B3864D815E816F8178854487D6
:10ED600055876687778749855A856B857C85408B73
:10ED7000518B628B738BC48AD58AE68AF78A2D857C
:10ED80003E85318F208F228E1C52138F8D50848FA1
:10ED9000358E068FA78FB0A391A360960FB6F89417
:10EDA000DEBF0FBECDBFDF91CF911F910F91FF90BE
:10EDB000EF90DF90CF90BF90AF909F908F907F901B
:10EDC0006F905F904F903F902F9008952F923F92B9
:10EDD0004F925F926F927F928F929F92AF92BF926B
:10EDE000CF92DF92EF92FF920F931F93CF93DF9317
:10EDF000CDB7DEB762970FB6F894DEBF0FBECDBFBA
:10EE0000FC01278C80A1898791A19A87208131817B
:10EE100042815381448055806680778080849184CC
:10EE2000A284B384C484D584E684F78480899189DC
:10EE3000A289B38989839A83AB83BC8384899589AA
:10EE4000A689B7898D839E83AF83B887608D718DC6
:10EE5000128D938D998BA48DAA8B358C068D89E7A5
:10EE60009FE22D873E874F87588B6B877C870E9458
:10EE700052FC6B857C8570931B0860931A08832D68
:10EE80000E94E251802F0E941F4F812F0E94DF4677
:10EE90002D853E854F85588960E571E280E390E0DD
:10EEA0000E940E47A301920164E571E280E390E0C5
:10EEB0000E940E47A501940168E571E280E390E0AD
:10EEC0000E940E47A70196016CE571E280E390E095
:10EED0000E940E4729813A814B815C8160E671E294
:10EEE00080E390E00E940E472D813E814F8158853E
:10EEF00064E671E280E390E00E940E47B9894B2FEF
:10EF0000BB0F550B445D5F4F60E370E280E390E020
:10EF10000E94EE468A89482F880F550B435F5F4F4A
:10EF200064E470E280E390E00E94EE46E7EAF7E0F6
:10EF3000208299859183AA85A28362960FB6F89460
:10EF4000DEBF0FBECDBFDF91CF911F910F91FF901C
:10EF5000EF90DF90CF90BF90AF909F908F907F9079
:10EF60006F905F904F903F902F900C94AD892F92AF
:10EF70003F924F925F926F927F928F929F92AF9249
:10EF8000BF92CF92DF92EF92FF920F931F93CF9396
:10EF9000DF93CDB7DEB727970FB6F894DEBF0FBE6D
:10EFA000CDBF782ECE0101960E94315E70FE78C0F2
:10EFB0004FEF5FEF6FEF72E0CE0101960E94A7471F
:10EFC00047E050E060E076E2CE0101960E94A7475C
:10EFD00043E655E461E274E0CE0101960E94A74742
:10EFE0001A8240E050E060E073E0CE0101960E949A
:10EFF000A7478BE18983C12C26E0D22E36EFE32E82
:10F000003FE2F32E0EE310E02AE031E043E050E06F
:10F0100063E070E0CE0101960E9483614C018AE1B9
:10F02000F4018083118240E050E060E073E0C401AD
:10F030000E94A747C12C4CE0D42E57EEE52E5FE28C
:10F04000F52E23E730E047E450E063E070E0C401D0
:10F050000E9483616AEDE62E6FE2F62E23E730E030
:10F060004CE850E063E070E00E9483617EECE72EA4
:10F070007FE2F72E23E730E040ED50E063E070E000
:10F080000E948361E2ECEE2EEFE2FE2E23E730E0F9
:10F0900045E151E063E070E0CE0101960E9483619A
:10F0A00071FE13C10E943E4F8C830E94EE828D83BD
:10F0B00080916A0A282F30E03F832E83C0906B0A2C
:10F0C000D12C8BE1898366E374E0CE0101960E9426
:10F0D000B25B4C0182E0F401818342E050E060E0E9
:10F0E00073E0C4010E94A747F40180815CDB8C01BE
:10F0F00016950795B801660F771F80E090E00F9492
:10F1000036999B01AC0160E070E086EE92E40F94CA
:10F11000BC970F9405991B012C012EE3622E712CD4
:10F12000601A710A76946794F7E46F0E711CB80147
:10F1300080E090E00F94369920E030E048EF52E410
:10F140000F94BD970F94059940E8A42EB12CE12CA3
:10F15000F12C9101A301C4010E946A4A83E0F401E9
:10F16000818343E050E060E073E0C4010E94A74760
:10F17000F401808118DB8C0116950795B801660FA4
:10F18000771F80E090E00F9436999B01AC0160E01E
:10F1900070E086EE92E40F94BC970F9405992B01D2
:10F1A0003C01FEE32F2E312C201A310A369427948D
:10F1B000FCE82F0E311CB80180E090E00F943699E6
:10F1C00020E030E048EF52E40F94BD970F9405998A
:10F1D000AA24AA94B12CCE80DF809201A101C4019F
:10F1E0000E946A4A66E274E0C4010E94B25B3C017C
:10F1F00084E0F301818344E050E060E073E0C30108
:10F200000E94A747812C912CAD8011E1C12E10E303
:10F21000D12E0EE0E02E00E3F02E0EE310E023E707
:10F2200030E040ED50E06CE770E0C301EFDA3C0104
:10F2300085E0F301818345E050E060E073E0C301C5
:10F240000E94A747AC8023E730E045E151E06CE73E
:10F2500070E0C301DBDA66E574E00E94B25B4C014A
:10F2600086E0F401818346E050E060E073E0C40191
:10F270000E94A747C12CD12C81EBE82E8FE2F82EFB
:10F280002AE031E049E551E063E070E0C4010E940A
:10F29000055C66E474E00E94B25B4C0181E0F4011D
:10F2A000818341E050E060E073E0C4010E94A74721
:10F2B00099E0E92E90E3F92E2AE031E04EE951E0A1
:10F2C00063E070E0C4010E94055C27960FB6F894D5
:10F2D000DEBF0FBECDBFDF91CF911F910F91FF9089
:10F2E000EF90DF90CF90BF90AF909F908F907F90E6
:10F2F0006F905F904F903F902F900895CF93DF9342
:10F30000CDB7DEB72A970FB6F894DEBF0FBECDBFDC
:10F3100088E18983CE0101960E949351CE0108961F
:10F320000E94315E40E05FEF6FEF7FEFCE01089605
:10F330000E94A747CE0101960E945250882329F0CF
:10F34000CE0101960E94C15110C0CE0108960E94C4
:10F35000F45361E082E597E00E94336E40E050E0B4
:10F36000BA01CE0101960E94DE5062E082E597E08C
:10F370000E94336E40E050E0BA01CE0108960E9430
:10F38000A74741E05FEF6FEF7FEFCE0108960E9445
:10F39000A747CE0108960E94274C2A960FB6F894EC
:10F3A000DEBF0FBECDBFDF91CF910895CF92DF9228
:10F3B000EF92FF920F931F93CF93DF9300D0CDB7BF
:10F3C000DEB711E061E082E79AE00E94915888235D
:10F3D00009F454C082E79AE00E94B058CE01019629
:10F3E0000E94315E80914807882309F449C00E9439
:10F3F000474F882399F060E070E980E390E00E9435
:10F4000004466C01EE24FF246230E9F06330C1F55C
:10F41000D0926A0A8D2D0E94E2512DC0E12CF12C70
:10F4200000E010E020E030E040E050E060E070E01C
:10F43000CE0101960E94504BCE0101960E94274CAE
:10F44000109248071DC0B60180E090E00F943699F5
:10F4500020E030E040E053E40F94199B20E03FEFC0
:10F460004FE757E40F949D980F940A99862F609365
:10F470006B0A0E94DF461093C90940DF0E948A9BF5
:10F480000F900F900F90DF91CF911F910F91FF90F0
:10F49000EF90DF90CF900895E6ECF7E010821182B4
:10F4A00012821382E2ECF7E01082118290E89283DC
:10F4B0001382EEEBF7E0108291838FEF8283138249
:10F4C000EAEBF7E0908381838283138208951092A0
:10F4D0006B0A10926C0A10926D0A10926E0A0C94CC
:10F4E0002D5FEF920F931F93CF93DF93CDB7DEB7CE
:10F4F0002A970FB6F894DEBF0FBECDBF682FCE019E
:10F5000001960E94E45F42E061E0CE0101960E9414
:10F51000225F8BE290E39987888766E370E3CE01F0
:10F5200001960E94EA6164E1CE0101960E94CE62DA
:10F5300080E00E9423DDE82E80E00E942DDC8B011C
:10F540009C0180E090E0AFEFB0E08B839C83AD83C3
:10F55000BE8344E350E362E0CE0101960E94C4659D
:10F5600081E00E9423DDE82E81E00E942DDC8B01EA
:10F570009C0180E09BEBA0E0B0E08B839C83AD839B
:10F58000BE8342E350E364E0CE0101960E94C4656D
:10F5900082E00E9423DDE82E82E00E942DDC8B01B8
:10F5A0009C018FEB90E0A0E0B0E08B839C83AD8367
:10F5B000BE8340E350E366E0CE0101960E94C4653D
:10F5C00081E794E6A6E5B0E08B839C83AD83BE83A0
:10F5D00080E00E9429DD00916B0A10916C0A209155
:10F5E0006D0A30916E0AE82E4EE250E368E0CE01DB
:10F5F00001960E94C465CE0101960E944A622A9635
:10F600000FB6F894DEBF0FBECDBFDF91CF911F9133
:10F610000F91EF900895CF92DF92EF92FF92CF93E8
:10F62000C82F0E94675F6B017C018C2F90E0FC016A
:10F630003297E631F10508F080C08827E256FF4F87
:10F640008F4F0D94539C80E00E942DDCA701960102
:10F650000F94BC9707C080E00E942DDCA7019601A3
:10F660000F94BD9740E008C081E00E942DDCA70107
:10F6700096010F94BC9741E00E945BDC59C081E089
:10F680000E942DDCA70196010F94BD97F4CF82E074
:10F690000E942DDCA70196010F94BC9707C082E061
:10F6A0000E942DDCA70196010F94BD9742E0E4CFA4
:10F6B00080E00E9445DCA70196010F94BC9740E0D2
:10F6C0000E94F4DCA701960160916B0A70916C0AAC
:10F6D00080916D0A90916E0A0F94BC9716C080E0DD
:10F6E0000E9445DCA70196010F94BD9740E00E945F
:10F6F000F4DCA701960160916B0A70916C0A80910D
:10F700006D0A90916E0A0F94BD9760936B0A709387
:10F710006C0A80936D0A90936E0A0AC085E290E3AA
:10F7200005C08FE190E302C089E190E30E9467C3C6
:10F7300081E004C085E190E3F9CF80E0CF91FF90B4
:10F74000EF90DF90CF9008958F929F92AF92BF92EB
:10F75000CF92DF92EF92FF92CF93DF93CDB7DEB7D8
:10F7600060970FB6F894DEBF0FBECDBF6A017B0174
:10F7700090E1EEE6F2E0DE01119601900D929A958D
:10F78000E1F7E1E0F0E0EC0FFD1F94E0899FE00D70
:10F79000F11D112420E030E040E752E460817181E6
:10F7A000828193810F949D984B015C0120E030E0B1
:10F7B00040E850E4C701B6010F94199B2DEC3CECD6
:10F7C0004CE45FE30F94199B6B017C0120E030E077
:10F7D000A9010F94999AA701960118160CF0505898
:10F7E000C501B4010F94969887FD0FC020E030E06A
:10F7F000A901C701B6010F94999A4601570118163D
:10F8000024F0B7FAB094B7F8B094C501B40160968B
:10F810000FB6F894DEBF0FBECDBFDF91CF91FF9042
:10F82000EF90DF90CF90BF90AF909F908F90089512
:10F8300083E08ADF0C9474DFCF93DF93CDB7DEB71C
:10F840002A970FB6F894DEBF0FBECDBF87E089833D
:10F85000CE0101960E949351CE0108960E94264C3B
:10F860008AE1888719861A8640E05FEF6FEF7FEFA5
:10F87000CE0108960E94A747CE0101960E945250E1
:10F88000882329F0CE0101960E94C15110C0CE01FB
:10F8900008960E94F45361E082E597E00E94336E7F
:10F8A00040E050E0BA01CE0101960E94DE5062E0D5
:10F8B00082E597E00E94336E40E050E0BA01CE014D
:10F8C00008960E94A74741E05FEF6FEF7FEFCE0100
:10F8D00008960E94A747CE0108960E94274C2A96B8
:10F8E0000FB6F894DEBF0FBECDBFDF91CF91089564
:10F8F00060E182E79AE00E949158882329F09CDF1A
:10F9000082E79AE00E94B0580C948A9BE6EDF7E0FB
:10F910001082118212821382E2EDF7E010821182CE
:10F9200090E892831382EEECF7E0108291838FEFE0
:10F9300082831382EAECF7E09083818382831382CF
:10F94000089590E0FC013197EE30F10590F588279D
:10F95000EC54FF4F8F4F0D94539C0E94BAB524C0B6
:10F960006FED71EC1DC06AE978E61AC064E379EBCB
:10F9700017C064E077E614C06FEC71E911C06EE95E
:10F9800075E90EC063E378EB0BC066EF76EB08C059
:10F990006EEA79E905C062E276EB02C067EB77E7D1
:10F9A00082E597E00E94285B81E0089567EE75EBA1
:10F9B000F7CF80E00895AF92BF92CF92DF92EF929F
:10F9C000FF920F931F93CF93DF9300D0CDB7DEB795
:10F9D000B82E80FF18C0CE0101960E94264C8AE105
:10F9E00089831A821B824FEF5FEF6FEF72E0CE01C7
:10F9F00001960E94A74747E050E060E076E2CE0122
:10FA000001960E94A747B1FE77C1CE0101960E94E0
:10FA1000264C8AE189831A821B8266E774E0CE0154
:10FA200001960E94B25B5C018BE1F501808382E06C
:10FA3000818342E050E060E073E0C5010E94A74787
:10FA4000C12CD12C82E6E82E80E3F82E0FE210E0E4
:10FA500022E830E043E050E063E070E0C5010E943E
:10FA6000055C5C01FC0182818F77828383E0818366
:10FA700043E050E060E073E0C5010E94A7479FE8C3
:10FA8000E92E90E3F92E22E830E048E350E063E00D
:10FA900070E0C5010E94055C5C01FC0182818F77EA
:10FAA000828384E0818344E050E060E073E0C5013C
:10FAB0000E94A7472AE6E22E20E3F22E22E830E059
:10FAC0004DE650E063E070E0C5010E94055C5C011A
:10FAD00085E0F501818345E050E060E073E0C50119
:10FAE0000E94A74736E8E32E30E3F32E22E830E009
:10FAF00043EA50E063E070E0C5010E94055C5C01F0
:10FB0000FC0182818068828386E0818346E050E048
:10FB100060E073E0C5010E94A7474CEBE42E40E390
:10FB2000F42E22E830E048ED50E063E070E0C501DB
:10FB30000E94055C5C0187E0F501818347E050E0AD
:10FB400060E073E0C5010E94A74759ECE52E50E341
:10FB5000F52E22E830E043E050E06BE870E0C501AC
:10FB60000E94055C5C0188E0F501818348E050E07B
:10FB700060E073E0C5010E94A74763EBE62E60E3F7
:10FB8000F62E22E830E048E350E06BE870E0C50173
:10FB90000E94055C5C0189E0F501818349E050E049
:10FBA00060E073E0C5010E94A74776EAE72E70E3A4
:10FBB000F72E22E830E04DE650E06BE870E0C5013A
:10FBC0000E94055C5C018AE0F50181834AE050E017
:10FBD00060E073E0C5010E94A747E1EAEE2EE0E392
:10FBE000FE2E22E830E043EA50E06BE870E0C50109
:10FBF0000E94055C5C01FC0182818F7782838BE02F
:10FC000081834BE050E060E073E0C5010E94A747AC
:10FC1000F8E9EF2EF0E3FF2E22E830E048ED50E067
:10FC20006BE870E0C5010E94055C5C01FC0182810B
:10FC30008F7782838CE081834CE050E060E073E05A
:10FC4000C5010E94A747A0E4EA2EA0E3FA2E2AE00D
:10FC500031E04DE051E063E070E0C5010E94055CD9
:10FC60005C018DE0F50181834DE050E060E073E0E0
:10FC7000C5010E94A747BFE4EB2EB0E3FB2E2AE0AC
:10FC800031E043E451E063E070E0C5010E94055CAF
:10FC90005C018EE0F50181834EE050E060E073E0AE
:10FCA000C5010E94A74785E7E82E80E3F82E2AE0E9
:10FCB00031E048E751E063E070E0C5010E94055C77
:10FCC00066E674E00E94B25B5C0181E0F50181832D
:10FCD00041E050E060E073E0C5010E94A74792ED6B
:10FCE000E92E90E3F92E2AE031E04DEA51E063E09D
:10FCF00070E0C5010E94055C0F900F900F90DF919E
:10FD0000CF911F910F91FF90EF90DF90CF90BF9018
:10FD1000AF900895E6EEF7E010821182128213820E
:10FD2000E2EEF7E01082118290E892831382EEED0A
:10FD3000F7E0108291838FEF82831382EAEDF7E080
:10FD400090838183828313820895AF92BF92CF9272
:10FD5000DF92EF92FF920F931F93CF93DF9300D028
:10FD6000CDB7DEB77C015B01CE0101960E94315E0A
:10FD700040E05FEF6FEF7FEFCE0101960E94A74753
:10FD80004FEF5FEF6FEF72E0CE0101960E94A74741
:10FD900047E050E060E076E2CE0101960E94A7477E
:10FDA00043E655E461E274E0CE0101960E94A74764
:10FDB0001A8240E050E060E073E0CE0101960E94BC
:10FDC000A747A114B10411F49CE1A92EC12C86E02F
:10FDD000D82E0EEA10E02AE031E043E050E063E084
:10FDE00070E0CE0101960E943B5966E974E0CE01B5
:10FDF00001960E94B25B0F900F900F90DF91CF9110
:10FE00001F910F91FF90EF90DF90CF90BF90AF9038
:10FE10000895AF92BF92CF92DF92EF92FF920F932D
:10FE20001F93CF93DF9300D0CDB7DEB77C015B018A
:10FE3000CE0101960E94315E40E05FEF6FEF7FEFF1
:10FE4000CE0101960E94A7474FEF5FEF6FEF72E080
:10FE5000CE0101960E94A74747E050E060E076E2BD
:10FE6000CE0101960E94A74743E655E461E274E0A3
:10FE7000CE0101960E94A7471A8240E050E060E060
:10FE800073E0CE0101960E94A747A114B10411F4BA
:10FE90009CE1A92EC12C86E0D82E0EEA10E02AE0C3
:10FEA00031E043E050E063E070E0CE0101960E9453
:10FEB000405A66E974E0CE0101960E94B25B0F9051
:10FEC0000F900F90DF91CF911F910F91FF90EF90C6
:10FED000DF90CF90BF90AF9008950F931F93CF9373
:10FEE000DF9300D0CDB7DEB7CE0101960E94315E20
:10FEF00043E655E461E274E0CE0101960E94A74713
:10FF000000E010E020E030E04EE051E068E870E012
:10FF1000CE0101960E94824BCE0101960E94274C91
:10FF20000F900F900F90DF91CF911F910F91089537
:10FF3000813011F0823031F482E597E00E94425B1B
:10FF400081E0089580E008950C94129B8F929F9217
:10FF5000AF92BF92CF92DF92EF92FF920F931F93D7
:10FF6000CF93DF9300D0CDB7DEB7182FCE01019627
:10FF70000E94315E123041F036E9A32E34E0B32EF8
:10FF8000113049F0B50109C026E8A22E24E0B22EB6
:10FF900066E974E002C066E874E08BE18983CE0113
:10FFA00001960E94B25B4C0181E0F401818341E043
:10FFB00050E060E073E0C4010E94A747C12CD12C3F
:10FFC0008FEDE82E80E3F82E06E310E022E830E023
:10FFD00047EA51E063E070E0C4010E94055CB501AE
:10FFE0000E94B25B5C0182E0F501818342E050E057
:10FFF00060E073E0C5010E94A7479CEDE92E90E305
:020000021000EC
:10000000F92E22E830E047EA51E06BE870E0C501E4
:100010000E94055C0F900F900F90DF91CF911F9180
:100020000F91FF90EF90DF90CF90BF90AF909F9097
:100030008F900895CF92DF92EF92FF920F931F93CC
:10004000CF93DF9300D0CDB7DEB7CE0101960E94EB
:10005000315E8BE1898381E08A8341E050E060E09A
:1000600073E0CE0101960E94A747C12CD12C87EDE9
:10007000E82E80E3F82E06E310E02AE031E047EABC
:1000800051E063E070E0CE0101960E94055C0F90A4
:100090000F900F90DF91CF911F910F91FF90EF90F4
:1000A000DF90CF900895E6EFF7E010821182128280
:1000B0001382E2EFF7E01082118290E892831382BC
:1000C000EEEEF7E0108291838FEF82831382EAEEE7
:1000D000F7E0908381838283138208950895AF921D
:1000E000CF92DF92EF92FF920F931F93CF93DF9304
:1000F00000D0CDB7DEB7CE0101960E94264C8AE132
:1001000089831A821B824FEF5FEF6FEF72E0CE019F
:1001100001960E94A74747E050E060E076E2CE01FA
:1001200001960E94A74743E655E461E274E0CE01E0
:1001300001960E94A7478CE1A82EC12C96E0D92EEB
:1001400023EEE22E20E3F22E0AED11E02AE031E068
:1001500043E050E063E070E0CE0101960E94405A17
:1001600045E15FEF6FEF7FEFCE0101960E94A74759
:100170000F900F900F90DF91CF911F910F91FF90F3
:10018000EF90DF90CF90AF900895AF92CF92DF9233
:10019000EF92FF920F931F93CF93DF9300D0CDB7D1
:1001A000DEB7CE0101960E94264C8AE189831A822D
:1001B0001B820E941D9B6CE871E280E390E00E942C
:1001C000044697FF22C040E05FEF6FEF7FEFCE0164
:1001D00001960E94A74782E082DF40E050E0BA012A
:1001E000CE0101960E94A747CE0101960E94274C9E
:1001F0000F900F900F90DF91CF911F910F91FF9073
:10020000EF90DF90CF90AF90089540E05FEF6FEFF9
:100210007FEFCE0101960E94A7474FEF5FEF6FEF90
:1002200072E0CE0101960E94A74747E050E060E0EF
:1002300076E2CE0101960E94A74743E655E461E2CB
:1002400074E0CE0101960E94A7478CE1A82EC12C34
:1002500096E0D92E2FEFE22E20E3F22E0AED11E0E8
:100260002AE031E043E050E063E070E0CE01019627
:100270000E94405A40E050E0BA01CE0101960E942F
:10028000A74741E05FEF6FEF7FEFCE0101960E943D
:10029000A747CE0101960E94274C6CE871E280E3EB
:1002A00090E00E94044697FFF8CF8DCF6CE871E292
:1002B00080E390E00E94044697FF08C00E94364702
:1002C000811104C082E597E00C94425B0895E6E05A
:1002D000F8E01082118212821382E2E0F8E01082CC
:1002E000118290E892831382EEEFF7E010829183FF
:1002F0008FEF82831382EAEFF7E09083818382831A
:1003000013820895EF920F931F93CF93DF93CDB78E
:10031000DEB72A970FB6F894DEBF0FBECDBF682FA9
:10032000CE0101960E94E45F42E060E0CE010196BA
:100330000E94225F83E291E39987888767E471E3F3
:10034000CE0101960E94EA6180E00E94BADE8B0134
:100350009C0180E090E0AFEFB0E08B839C83AD83A5
:10036000BE83EE24E39440E451E362E0CE010196C3
:100370000E94C46581E00E94BADE8B019C0180E08E
:100380009BEBA0E0B0E08B839C83AD83BE8349E30D
:1003900051E364E0CE0101960E94C46582E00E94B0
:1003A000BADE8B019C018FEB90E0A0E0B0E08B8384
:1003B0009C83AD83BE8342E351E366E0CE010196A8
:1003C0000E94C46580E00E94C7DE8B019C0181E72A
:1003D00094E6A6E5B0E08B839C83AD83BE834AE2BE
:1003E00051E368E0CE0101960E94C465CE010196FA
:1003F0000E944A622A960FB6F894DEBF0FBECDBFA8
:10040000DF91CF911F910F91EF9008951F93CF939C
:10041000DF9300D01F92CDB7DEB7182F0E94675F21
:100420009B01AC01812F90E0FC013297E830F1058F
:1004300008F07FC08827EE53FF4F8F4F0D94539CD9
:1004400080E029833A834B835C830E94BADE298152
:100450003A814B815C810F94BC970DC080E0298369
:100460003A834B835C830E94BADE29813A814B81B7
:100470005C810F94BD9740E00EC081E029833A83F0
:100480004B835C830E94BADE29813A814B815C8177
:100490000F94BC9741E00E94D1DE3BC081E02983EC
:1004A0003A834B835C830E94BADE29813A814B8177
:1004B0005C810F94BD97EECF82E029833A834B8312
:1004C0005C830E94BADE29813A814B815C810F9462
:1004D000BC970DC082E029833A834B835C830E94E2
:1004E000BADE29813A814B815C810F94BD9742E04D
:1004F000D2CF80E029833A834B835C830E94C7DE9E
:1005000029813A814B815C810F94BC9740E00E9425
:10051000E2DE81E00FC080E029833A834B835C8375
:100520000E94C7DE29813A814B815C810F94BD977F
:10053000EDCF80E00F900F900F900F90DF91CF9153
:100540001F910895E6E1F8E0108211821282138271
:10055000E2E1F8E01082118290E892831382EEE0EB
:10056000F8E0108291838FEF82831382EAE0F8E053
:1005700090838183828313820895EAE6FAE08FE50F
:100580009FE5DC0180839183A283B38314820C9462
:100590001D9BEAE6FAE080E090E02191222351F0F1
:1005A000880F991F880F991F022E000C330B82278A
:1005B0009327F3CF009711F48FEF9FEF0895809169
:1005C0001A0890911B08892B41F010926E0A6BE279
:1005D00073E882E597E00C94285B089581E0209110
:1005E0001A0830911B08232B09F480E0089510921B
:1005F0001B0810921A08089510926E0A10921B0898
:1006000010921A086BE273E882E597E00C94285B7D
:10061000AF92BF92CF92DF92EF92FF920F931F9310
:10062000CF93DF93EC0157018881E82E880FFF08F4
:10063000CE010E94F648B501CE010E94404ECE0187
:10064000DF91CF911F910F91FF90EF90DF90CF90AE
:10065000BF90AF900895AF92BF92CF92DF92EF928A
:10066000FF920F931F93CF93DF93CDB7DEB7C75998
:10067000D1090FB6F894DEBF0FBECDBF182FCE0143
:100680008B569F4F0E94264C8AE1CB56DF4F8883C2
:10069000C559D040CA56DF4F1882C659D040C956F6
:1006A000DF4F1882C759D04010FF29C04FEF5FEFCE
:1006B0006FEF72E0CE018B569F4F0E94A74747E035
:1006C00050E060E076E2CE018B569F4F0E94A74734
:1006D00043E655E461E274E0CE018B569F4F0E94E1
:1006E000A747CA56DF4F1882C659D04040E050E0B5
:1006F00060E073E0CE018B569F4F0E94A74711FF29
:100700005CC180916E0A873619F0873789F005C081
:10071000A1EACA2EA1E3DA2E14C080911A089091A2
:100720001B08892B51F0F0E8CF2EF1E3DF2E09C032
:10073000E4EBCE2EE1E3DE2E04C070E9C72E71E3B8
:10074000D72E10926E0A0E94444FA82EB12C8CE135
:10075000CB56DF4F8883C559D040C6010E946D53E8
:10076000082F1CE10023A1F0812F0E944953BC01F6
:10077000C6010E9441547C01812F0E9449539A83F3
:100780008983CE0101960E945553282F30E013C073
:10079000612FCE0101960E9445464FEF5FE7B601FB
:1007A000CE0101960E9441457C01C357DF4F28814D
:1007B0003981CD58D0408AE0E81681E0F8061CF473
:1007C0002A3231051CF01150193161F6C6010E9420
:1007D0006D53882391F0812F0E944953E12C66E0EC
:1007E000F62E8C01960148E450E068E870E0CE01F6
:1007F0008B569F4F0E94E55414C0212F110F330BCD
:1008000000E016E048E450E068E870E0CE018B5666
:100810009F4F0E948E48B601CE018B569F4F0E947B
:10082000404E8DE1CB56DF4F8883C559D0408AE6D4
:100830009AE00E946253F82E1DE1FF20A9F0812F5B
:100840000E944953BC018AE69AE00E9433546C012D
:10085000812F0E9449539A838983CE0101960E9479
:100860005553282F30E014C0612FCE0101960E940D
:1008700045464FEF5FE76AE67AE0CE0101960E94B7
:1008800023456C01C357DF4F28813981CD58D040B3
:100890008AE0C81681E0D8061CF42A3231051CF023
:1008A0001150193151F68AE69AE00E94625388236A
:1008B00099F0812F0E944953E12C56E0F52E8C01CE
:1008C0002AE63AE048EA50E068E870E0CE018B564C
:1008D0009F4F0E94785415C0212F110F330B00E059
:1008E00016E048EA50E068E870E0CE018B569F4F72
:1008F0000E948E486AE67AE0CE018B569F4F0E9496
:10090000554C8CE1CB56DF4F8883C559D0404FEF13
:100910005FEF6FEF74E0CE018B569F4F0E94A747A9
:100920004FEF5FEF6FEF70E0CE018B569F4F0E944D
:10093000234843E655E461E270E0CE018B569F4FB9
:100940000E94F04742ED59EA69E770E0CE018B560C
:100950009F4F0E94BD47650184E5E82E81E3F82E94
:100960000AE210E02AE031E043E251E063E070E0A7
:10097000CE018B569F4F4CDE2FE5E22E21E3F22E67
:100980002AE031E043E551E063E070E041DE3AE621
:10099000E32E31E3F32E2AE031E043E851E063E057
:1009A00070E036DE45E7E42E41E3F42E2AE031E044
:1009B00043EB51E063E070E02BDEC956DF4F0FB62A
:1009C000F894DEBF0FBECDBFDF91CF911F910F9185
:1009D000FF90EF90DF90CF90BF90AF9008951F935E
:1009E000CF93DF93CDB7DEB72A970FB6F894DEBF6B
:1009F0000FBECDBF1AE11983CE0101960E9493511B
:100A0000CE0108960E94264C188719861A8640E067
:100A10005FEF6FEF7FEFCE0108960E94A747CE01F0
:100A200001960E945250882329F0CE0101960E941F
:100A3000C15110C0CE0108960E94F45361E082E5D6
:100A400097E00E94336E40E050E0BA01CE0101967B
:100A50000E94DE5062E082E597E00E94336E40E043
:100A600050E0BA01CE0108960E94A74741E05FEF2F
:100A70006FEF7FEFCE0108960E94A747CE01089640
:100A80000E94274C2A960FB6F894DEBF0FBECDBF4A
:100A9000DF91CF911F910895CF93DF93C0911A08F2
:100AA000D0911B08209781F410926E0A98DF41E0E4
:100AB00064ED78E489E497E00E94B3526ADD909394
:100AC0001B0880931A081FC064DDC817D90761F49A
:100AD00087E680936E0A83DF41E064ED78E489E481
:100AE00097E00E94B3520FC087E780936E0A77DFCA
:100AF00041E064EE78E489E497E00E94B35282E535
:100B000097E00E941B5B82E597E0DF91CF910C9408
:100B1000425BCF93C82F6FE570E08AE69AE00F94AE
:100B200063A1FC01892B79F0CC3341F48AE0EA36E9
:100B3000F80749F031978FE5808305C0C083818134
:100B4000811101C0A9DF81E0CF910895E8E2F8E0CA
:100B50001082118212821382E4E2F8E01082118284
:100B600090E892831382E0E2F8E0108291838FEFA5
:100B700082831382ECE1F8E0908381838283138285
:100B800008958F929F92AF92BF92CF92DF92EF9291
:100B9000FF920F931F93CF93DF93CDB7DEB7C45966
:100BA000D1090FB6F894DEBF0FBECDBF182F6B0171
:100BB0005A017901C9010E946D53082F1A318CF135
:100BC0000023A1F0812F0E944953BC01C7010E945C
:100BD00041544C01812F0E9449539A838983CE014D
:100BE00001960E945553E82FF0E013C0612FCE010B
:100BF00001960E9445464FEF5FE7B701CE0101968F
:100C00000E9441454C01C357DF4FE881F981CD581F
:100C1000D0408C149D041CF4EA15FB0514F011500F
:100C2000CDCF812FCC56DF4F0FB6F894DEBF0FBE6D
:100C3000CDBFDF91CF911F910F91FF90EF90DF908B
:100C4000CF90BF90AF909F908F90089590E0FC015F
:100C50003197EA30F105C0F58827E653FF4F8F4FF3
:100C60000D94539C82E597E00E94425B24C06BE6A2
:100C70007DE925C062E47AE882E597E00E94025BA4
:100C80008CED91E30E9468B582E597E00E941B5BC2
:100C900012C060E572EA13C040E064ED75E489E4D7
:100CA00097E00E94B35207C0A8D781110EC084EC10
:100CB00091E30E9475B581E0089564E077E682E5EE
:100CC00097E00E94285BF7CF80E00895AF92BF9233
:100CD000CF92DF92EF92FF920F931F93CF93DF9308
:100CE00000D0CDB7DEB780FF59C1CE0101960E947A
:100CF000264C8AE189831A821B824FEF5FEF6FEFE8
:100D000072E0CE0101960E94A74747E050E060E004
:100D100076E2CE0101960E94A7478BE189831A8271
:100D200040E050E060E073E0CE0101960E94A747EA
:100D300043E655E461E274E0CE0101960E94A747C4
:100D40008CE1898320E332E34AE250E06AE071E01B
:100D500018DFB82E80E392E30E946D53882391F050
:100D60008B2D0E944953E12CF6E0FF2E8C0120E3ED
:100D700032E348E150E068E870E0CE0101960E945D
:100D8000E55413C02B2DBB0C330B00E016E048E1FB
:100D900050E068E870E0CE0101960E948E4860E362
:100DA00072E3CE0101960E94404E66EB74E0CE01E4
:100DB00001960E94B25B5C0182E0F501818342E012
:100DC00050E060E073E0C5010E94A7478BE1F501A8
:100DD0008083C12CD12C8FE3E82E82E3F82E0AE227
:100DE00010E02AE031E043E350E063E070E0C50149
:100DF0000E94055C5C0183E0F501818343E050E0E3
:100E000060E073E0C5010E94A74790E5E92E92E3F8
:100E1000F92E2AE031E043E650E063E070E0C501DE
:100E20000E94055C5C0184E0F501818344E050E0B0
:100E300060E073E0C5010E94A7472CE5E22E22E3A3
:100E4000F22E2AE031E043E950E063E070E0C501B2
:100E50000E94055C5C0185E0F501818345E050E07E
:100E600060E073E0C5010E94A74731E7E32E32E35B
:100E7000F32E2AE031E043EC50E063E070E0C5017E
:100E80000E94055C5C0186E0F501818346E050E04C
:100E900060E073E0C5010E94A747F50182818F776A
:100EA00082834BE7E42E42E3F42E2AE031E043EF65
:100EB00050E063E070E0C5010E94055C5C0187E0E2
:100EC000F501818347E050E060E073E0C5010E94D6
:100ED000A747F50182818068828351E9E52E52E3BC
:100EE000F52E2AE031E043E251E063E070E0C50115
:100EF0000E94055C5C0188E0F501818348E050E0D8
:100F000060E073E0C5010E94A747F5018281806817
:100F100082836BEAE62E62E3F62E2AE031E043E5B7
:100F200051E063E070E0C5010E94055C5C0189E06E
:100F3000F501818349E050E060E073E0C5010E9463
:100F4000A747F50182818068828373ECE72E72E304
:100F5000F72E2AE031E043E851E063E070E0C5019C
:100F60000E94055C5C0181E0F501818341E050E075
:100F700060E073E0C5010E94A74766EA74E0C5011E
:100F80000E94B25BE3EDEE2EE2E3FE2E2AE031E0BA
:100F900043EB51E063E070E00E94055C0F900F901E
:100FA0000F90DF91CF911F910F91FF90EF90DF9005
:100FB000CF90BF90AF900895E8E3F8E010821182DF
:100FC00012821382E4E3F8E01082118290E89283A7
:100FD0001382E0E3F8E0108291838FEF8283138223
:100FE000ECE2F8E09083818382831382089560E0CD
:100FF00070E08BEF92E30E94097F81E00C94A67F62
:10100000813049F0823081F461ED74EB82E597E044
:101010000E94285B0BC088ED92E30E9467C382E5C3
:1010200097E00E941B5B02C00C94987F81E00895BA
:10103000E8E4F8E01082118212821382E4E4F8E01E
:101040001082118290E892831382E0E4F8E010822B
:1010500091838FEF82831382ECE3F8E090838183A6
:101060008283138208958F929F92AF92BF92CF9204
:10107000DF92EF92FF920F931F93CF93DF93CDB741
:10108000DEB7C459D1090FB6F894DEBF0FBECDBF8D
:10109000182F6B015A017901C9010E946D53082F65
:1010A0001A318CF10023A1F0812F0E944953BC0119
:1010B000C7010E9441544C01812F0E9449539A83D9
:1010C0008983CE0101960E945553E82FF0E013C0AA
:1010D000612FCE0101960E9445464FEF5FE7B701B1
:1010E000CE0101960E9441454C01C357DF4FE88174
:1010F000F981CD58D0408C149D041CF4EA15FB05F1
:1011000014F01150CDCF812FCC56DF4F0FB6F8948D
:10111000DEBF0FBECDBFDF91CF911F910F91FF902A
:10112000EF90DF90CF90BF90AF909F908F900895F9
:101130004F925F926F927F928F929F92AF92BF92E7
:10114000CF92DF92EF92FF921F93CF93DF93CDB7B1
:10115000DEB72F970FB6F894DEBF0FBECDBF7C0170
:101160006B015A012901CE0101960E94264C8AE1A9
:1011700089831A821B8214E6612C712C950140E050
:1011800050E02C833D834E835F83960140E050E026
:10119000288739874A875B87970140E050E02C8792
:1011A0003D874E875F87C301B2010E94153C4B010A
:1011B0005C016C817D818E819F810E94153C288518
:1011C00039854A855B85820E931EA41EB51E24E0D8
:1011D000880C991C2A95E1F7E89497F86401E12CB2
:1011E000F12C460157016894B6F82C853D854E8553
:1011F0005F85260F371F481F591FB90134E0660F5E
:10120000771F3A95E1F77F776B01E12CF12C4FE0E6
:10121000CC0CDD1CEE1CFF1C4A95D1F7C828D92840
:10122000EA28FB286FEF7FEF8FEF90E00E94153CDC
:101230004B015C0142E050E060E07FE1CE010196AD
:101240000E94A74740E451E060E07DE0CE010196B6
:101250000E94A747B501A4017460CE0101960E94C7
:10126000A747B701A601CE0101960E94A7471150DA
:1012700009F099CF2F960FB6F894DEBF0FBECDBF01
:10128000DF91CF911F91FF90EF90DF90CF90BF90B3
:10129000AF909F908F907F906F905F904F90089548
:1012A0000F931F9380916A0A90916B0AA0916C0A28
:1012B000B0916D0A892B8A2B8B2BD9F00E94343880
:1012C00000916A0A10916B0A20916C0A30916D0AA4
:1012D000DC01CB01801B910BA20BB30B8095909589
:1012E000A095B0958827B7FD83959927AA27BB2796
:1012F00001C080E01F910F910895811103C080E02B
:1013000090E002C08DEA9EED90931B0880931A082E
:1013100088EE93E30C94B0E11F93CF93DF9300D05A
:10132000CDB7DEB7182FCE0101960E94264C8AE178
:1013300089831A821B8280E0113041F4DEDF61ED87
:1013400074EB82E597E00E94285B81E00F900F909C
:101350000F90DF91CF911F91089580911A0890917D
:101360001B088D3A9E4D31F462E47AE882E597E0FD
:101370000C94285B0895CF92DF92EF92FF920E9427
:1013800034386B017C0160E47CE980E090E00E94ED
:10139000153CEAE6FAE020E1C20E27E2D21EE11C8B
:1013A000F11CDC01CB018C0D9D1DAE1DBF1D80838A
:1013B0009183A283B3838EEC93E39583848340E08F
:1013C00060E070E0CB010E944AE241E060E070E042
:1013D000CB010E944AE246E060E070E0CB010E944F
:1013E000E4E181E0FF90EF90DF90CF9086CFC0EBFB
:1013F000D3E3D0936F0AC0936E0A82E597E00E9410
:10140000024FF7CF82E993E390936F0A80936E0ABD
:1014100082E597E00E94024FFBCF82E597E00E94B1
:10142000024F0E94129B0E94B2E181110BC00E94E8
:10143000D9E1811103C08EE893E302C08BE593E309
:101440000E94B0E16EE582E79AE00E9491588823FD
:1014500059F064E670E080E090E00E94153C0F9443
:10146000389940E00E9484E21BDF882349F062E063
:1014700070E080E090E00E94153C60FDC3DFB7DFC4
:101480000C948A9BCF92DF92EF92FF920F931F935F
:10149000CF93DF9300D0CDB7DEB7CE0101960E9487
:1014A000264C8AE189831A821B82C0906E0AD090F2
:1014B0006F0A4FEF5FEF6FEF72E0CE0101960E946F
:1014C000A74747E050E060E076E2CE0101960E9437
:1014D000A74743E655E461E274E0CE0101960E941D
:1014E000A7478BE1898396014FE250E06AE071E003
:1014F000BADD182FC6010E946D53882389F0812F11
:101500000E944953E12C26E0F22E8C0196014AE11B
:1015100050E068E870E0CE0101960E94E55412C0E8
:10152000212F110F330B00E016E04AE150E068E88C
:1015300070E0CE0101960E948E48B601CE01019660
:101540000E94404E2FEC30E04AE051E06DE670E042
:1015500083E090E0EDDDA4DE9BE199839B81811126
:1015600002C09F7701C090689B834FEF5FEF6FEFE2
:1015700074E0CE0101960E94A7474FEF5FEF6FEF37
:1015800070E0CE0101960E94234842ED59EA69E7D6
:1015900070E0CE0101960E94F0474FEF5FEF6FEFD2
:1015A00070E0CE0101960E94BD4781E08A8341E050
:1015B00050E060E073E0CE0101960E94A747C12C85
:1015C000D12C8DEEE82E83E3F82E0FE210E022E816
:1015D00030E048E751E067E470E0CE0101960E94F8
:1015E000055C0F900F900F90DF91CF911F910F919D
:1015F000FF90EF90DF90CF900895E8E5F8E010823B
:10160000118212821382E4E5F8E01082118290E8E0
:1016100092831382E0E5F8E0108291838FEF82835A
:101620001382ECE4F8E0908381838283138208952F
:10163000EAE6FAE01782128211821482138216827D
:1016400015820C942D5F8F929F92AF92BF92CF9292
:10165000DF92EF92FF920F931F93CF93DF93CDB75B
:10166000DEB72A970FB6F894DEBF0FBECDBF682F46
:10167000CE0101960E94E45F41E062E0CE01019656
:101680000E94225F2FEF33E3FC013087278362EF54
:1016900073E3CE0101960E94EA618AE6C82E8AE0D1
:1016A000D82EF60161817281072E000C880B990BF0
:1016B0000F9438994B015C0180E00E9468DE9B0129
:1016C000AC0180E090E0AFEFB0E08B839C83AD8312
:1016D000BE83C501B4010F949D988B019C01EE243B
:1016E000E39446E054E362E0CE0101960E94C465B3
:1016F000F60163817481072E000C880B990B0F94FF
:1017000038994B015C0181E00E9468DE9B01AC01CD
:1017100080E09BEBA0E0B0E08B839C83AD83BE8335
:10172000C501B4010F949D988B019C0144E054E3E2
:1017300064E0CE0101960E94C465F6016581768160
:10174000072E000C880B990B0F9438996B017C01C4
:1017500082E00E9468DE9B01AC018FEB90E0A0E08C
:10176000B0E08B839C83AD83BE83C701B6010F9429
:101770009D988B019C01EE24E39442E054E366E0E3
:10178000CE0101960E94C465CE0101960E944A6274
:101790002A960FB6F894DEBF0FBECDBFDF91CF9172
:1017A0001F910F91FF90EF90DF90CF90BF90AF907F
:1017B0009F908F9008950F931F93CF93C82F0E94EF
:1017C000675F8B019C018C2F90E0FC013297E83021
:1017D000F10508F09BC08827EC52FF4F8F4F0D9406
:1017E000539C40E0C901B8010E94B2DF8C0141E086
:1017F00060E088279927801B910B0E94B1DF209120
:101800006B0A30916C0AC901801B910B90936C0A92
:1018100080936B0A72C040E0C901B8010E94B2DF38
:101820008C0141E060E00E94B1DF80916B0A9091F1
:101830006C0A080F191F10936C0A00936B0A5DC0A5
:1018400041E0C901B8010E94B2DF8C0141E061E0D2
:1018500088279927801B910B0E94B1DF20916D0A88
:1018600030916E0AC901801B910B90936E0A809390
:101870006D0A43C041E0C901B8010E94B2DF8C018A
:1018800041E061E00E94B1DF80916D0A90916E0AA3
:10189000080F191F10936E0A00936D0A2EC042E0C4
:1018A000C901B8010E94B2DF8C0141E062E08827E3
:1018B0009927801B910B0E94B1DF20916F0A309114
:1018C000700AC901801B910B9093700A80936F0A74
:1018D00014C042E0C901B8010E94B2DF8C0141E0AE
:1018E00062E00E94B1DF80916F0A9091700A080F48
:1018F000191F1093700A00936F0A81E008C090913D
:10190000710A81E089278093710AF7CF80E0CF9137
:101910001F910F910895813011F00C94455F0E9442
:10192000BAB581E008950C94129BE8E6F8E01082C5
:10193000118212821382E4E6F8E01082118290E8AC
:1019400092831382E0E6F8E0108291838FEF828326
:101950001382ECE5F8E090838183828313820895FB
:101960000E941D9B0E94E8468FEF0C94E25108955F
:101970002F923F924F925F926F927F928F929F929F
:10198000AF92BF92CF92DF92EF92FF920F931F938D
:10199000CF93DF93CDB7DEB7C350D2400FB6F894E4
:1019A000DEBF0FBECDBF6C011B01CE018F5F9D4F0F
:1019B0000E94264C8AE1CF5FDD4F8883C150D24020
:1019C000CE5FDD4F1882C250D240CD5FDD4F18820E
:1019D000C350D24040E05FEF6FEF7FEFCE018F5FEB
:1019E0009D4F0E94A74740E050E060E072E0CE01CA
:1019F0008F5F9D4F0E94A74747E050E060E076E28E
:101A0000CE018F5F9D4F0E94A74740E050E0BA0192
:101A1000CE018F5F9D4F0E94A74741E05FEF6FEFC0
:101A20007FEFCE018F5F9D4F0E94A747CE018F5F52
:101A30009D4F0E94274C40E05FEF6FEF7FEFCE019C
:101A40008F5F9D4F0E94A74700E014E020E030E048
:101A500040E05CEF6FE070E0CE018F5F9D4F0E9431
:101A6000AE4B4CE350E060E070E0CE018F5F9D4FE5
:101A70000E94DA4B40E050E0BA01CE018F5F9D4FEB
:101A80000E94A74741E05FEF6FEF7FEFCE018F5FCE
:101A90009D4F0E94A747CE018F5F9D4F0E94274C0C
:101AA0000E9434384B015C0181E00E94DFFC412C34
:101AB000512C320140E052E0BE016F5F7F4FC60102
:101AC000F10119957C01019639F40E9460FC88E0CF
:101AD00094E30E9452FC62C00E943438DC01CB01C6
:101AE00088199909AA09BB090B97A105B10530F01E
:101AF0000E94D3DA0E9434384B015C0100E0970168
:101B0000AE014F5F5F4FC301B2017450804F9F4FD2
:101B10000E94824614E10E943438DC01CB0188190E
:101B20009909AA09BB090B97A105B10588F00E9484
:101B3000D3DA0E9434384B015C01115049F40E9401
:101B400060FC8CE194E30E9452FC0E94284C26C069
:101B500064E170E980E390E00E9404466415750535
:101B600086059705C1F6C7010F2C000CAA0BBB0B0D
:101B7000480E591E6A1E7B1E83E058226624772475
:101B8000A301920168E170E980E390E00E940E47B2
:101B9000E114E2E0FE0609F48DCF97CF84E00E94C5
:101BA000DFFC40E05FEF6FEF7FEFCE018F5F9D4F77
:101BB0000E94A747CE018F5F9D4F0E94274C0E9435
:101BC000C1500E94A1A7CD5FDD4F0FB6F894DEBFD4
:101BD0000FBECDBFDF91CF911F910F91FF90EF907E
:101BE000DF90CF90BF90AF909F908F907F906F903D
:101BF0005F904F903F902F9008951F93CF93DF9366
:101C0000CDB7DEB7C856D1090FB6F894DEBF0FBE08
